:020000041A00E0
:20000000D8400810FDC2031AD742031A8DB8011AD942031ADB42031ADD42031AAA46E55368
:20002000000000000000000000000000DF42031AE142031A00000000B5B8011A658E001AAD
:20004000E342031A00000000E542031A0000000000000000E742031AE942031AEB42031A42
:2000600097BF011AED42031AEF42031AF142031A8D48031A9FD3011AF342031AF542031A00
:20008000F742031AF942031AFB42031AFD42031A00000000FF42031A0143031A0343031ADA
:2000A0009BC5011A27C6011A0543031A0743031A0943031A0B43031A0D43031A0F43031A41
:2000C0001143031A1343031A1543031A1743031A1943031A1B43031A1D43031A1F43031A60
:2000E0002143031A2343031A2543031A2743031A00000000000000002943031A2B43031ADC
:200100000000000067C5011A000000002D43031A2F43031AFFFFFFFFFFFFFFFFFFFFFFFF88
:20012000000000000000000000000000000000004A2D4C696E6B2056313220636F6D7069A9
:200140006C65642041707220323320323032342031303A34313A323100436F707972696720
:20016000687420323032322D32303232205345474745523A207777772E7365676765722E55
:20018000636F6D000000000000000000000000000000000000000000000000000000000020
:2001A0006C1A46A746194EB81EA08CCBAF3EEC9AF4CF0D1DF39FA25A450223C4B6F22AD58F
:2001C000A3D333BBA0EC70F45F694893ED280E881DC62659CC6F20EC9A342202ED78B8269F
:2001E000CA8D9C1AC992D7FC2B2649619091D5B8FC81BC617975C4CD4801F121D6F42C2091
:20020000FCD5D3E3B369B9722ED69D247D0BFD1110891A81BC9A132C673C6852748B83D13C
:20022000D88E69F1C034F598955EC67095FB86883711389A98EF529EFC07D374A663CADE2A
:2002400003EC5BFDEDE37708ECC2282CCE51595553251027ED14A0CE143B9C0E0D0E75C6CC
:20026000FBAE60F255EB11D142DAFC985CADB87F12DD70264ABF98CC4D690EECC8DB6A03BF
:20028000D41FD02BE8D0EB3FCE63EFD6B52F3C4038323CE55FD886444519E9E462ECD1F171
:2002A0000138FDD5704700BF30BFFDE700000000DB002DE9FF4F81B03A4C3B4D3B4E4FF4A0
:2002C00080670198013001904FF0000A10F8018D02980130029010F8019D0498082888BFE7
:2002E0000820009004980099DDF800B0401A0490012080F310885FEAC87037604FF4807027
:200300004CBF306028604FF4805028602068FFF7C7FF2F604FEA58082068FFF7C1FF3760DE
:200320005FEAC9704FF480704CBF286030602068FFF7B6FF2F604FEA59092068FFF7B0FF5B
:200340004FF48050306037602068FFF7A9FF2F602068FFF7A5FF16480068400000F0800016
:2003600040EA5A0ABBF1010BC5D100064FF480704CBF286030604FF480502860002080F317
:20038000108800980399C0F1080001312AFA00F0039101F8010D0498002892D105B0BDE876
:2003A000F08F00007838081000620F4080620F4000610F4038B541F20050C4F20500032115
:2003C000016000BF41688907FCD50022C4F208021068C0074EF21000CEF200001ED14FF490
:2003E0000031C0F87411C0F874124EF26031C0F21601516040F2FF3151610B211160AA218A
:20040000552300BF91609360D468FF2CFAD91168090742BF116841F008011160EFF3108364
:20042000012181F310884FF40031C0F874124EF2314CCEF2000C10248CF80040C0F8F4109F
:20044000AA2191605521916083F31088016821F0030101604EF60850CEF2000048F20001F5
:20046000C1F60021016046F2CB50C1F60020017808064CBF002001F0030043F67431C1F2E2
:2004800008014FF0000C086040B1012401280CD1002145F69073C0F201030AE04BF62073B1
:2004A000C0F202030021002403E04FF480714AF6C87343F67C30C1F208005A1E026043F6FB
:2004C0007830C1F2080041F26F72026045F20C20C4F200001F2202601820C4F2050040F65E
:2004E000000EC0F2001EC0F854E0C0F800C0C0F830E040F60005C0F6001505F1407282655D
:20050000C26A42F00102C26243F68032C1F2080240F6000C13604FF47A72534343F6703259
:20052000C1F20802C0F20E6C1360C0F82CC000BF826AD207FCD0C26AC26245654FF47A7242
:200540000092009A12B1009A013AF9E7002CC26A22F4407442F0800218BF44EA0102C262F5
:20056000816AC907FCD040F60401C0F200614163426B02F0F852B2F1C06FF9D1826842F061
:200580000102826014220092009AB2F5004F12D84FF48044009A0132009284EA5402C4F353
:2005A0004D0462F38E34009AB2F5004FF2D90CF5FF22144303E044F20004C0F21664C46092
:2005C00042F20002C0F230020261026942F0620202611831816000BF4168C907FCD005F116
:2005E00008010163C0F838E0C0F83CE005F184010164406D43F66C50C1F20800036038BD55
:200600002DE9F04F8BB08A468146EFF310800090012181F310883120CDE90320B9F1D05F80
:2006200038BF09F1D0590025C4F208054FEA52282868C00703D0AA20A8605520A86040F25A
:200640000010C1F240000AA9026804A89047AA2655274FF0070BCDE9019A00BF2868C007F3
:200660001CBFAE60AF600020002100BF5AF8002001320FD1002901DD013906E02968C90775
:200680001CBFAE60AF604FF480710430B0F5007FECD144E0322004904FEA196000241A28F7
:2006A00088BF0124C9F34A30082888BF0BEBD000059009F2FF10C0F34A30082888BF0BEB22
:2006C000D000CDE906042868C0071CBFAE60AF6040F20010C1F240000AA9026804A8904766
:2006E0000A9818BB4FF400700790CDE9059A3320049043F68030C1F20800099400680890BE
:200700002868C0071CBFAE60AF6040F20010C1F240000AA9026804A890470A9830B9B8F181
:2007200001080AF5007A09F5007997D1009880F3108801AA07CA32F00FFF90B14AF2201458
:20074000C0F207040120012130F06AFD204613F0AAFD0120002130F063FD204613F0A3FD37
:20076000F0E70BB0BDE8F08F03281BD801460020DFE801F01A021B2346F20020C4F20F000F
:200780004FF40041C0F880104FF60061CFF6FF71425822F0010242506FF0FF01405800F08A
:2007A000010070474FF0FF30704746F20020C4F20F000121C0F8801005E046F20020C4F2E2
:2007C0000F00012101604FF60061CFF6FF71425842F0010242504FF400410160002070478F
:2007E00003281BD801460020DFE801F01A021B2446F20020C4F20F004FF40051C0F8801068
:200800004FF60061CFF6FF71425822F4007242506FF0FF014058C0F3402070474FF0FF301A
:20082000704746F20020C4F20F004FF40071C0F8801006E046F20020C4F20F004FF4007131
:2008400001604FF60061CFF6FF71425842F4007242504FF4005101600020704703281BD89E
:2008600001460020DFE801F01A021B2446F20020C4F20F004FF48051C0F880104FF60061DF
:20088000CFF6FF71425822F4807242506FF0FF014058C0F3002070474FF0FF30704746F211
:2008A0000020C4F20F004FF48071C0F8801006E046F20020C4F20F004FF4807101604FF6FA
:2008C0000061CFF6FF71425842F4807242504FF4805101600020704703281AD8014600205E
:2008E000DFE801F019021A2346F20020C4F20F004021C0F884104FF60061CFF6FF714258A9
:2009000022F4806242506FF0FF014058C0F3802070474FF0FF30704746F20020C4F20F000A
:200920004FF48061C0F8801006E046F20020C4F20F004FF4806101604FF60061CFF6FF71E8
:20094000425842F480624250402141600020704703281AD801460020DFE801F019021A22E7
:2009600046F20020C4F20F001021C0F880104FF60061CFF6FF71425822F0020242506FF065
:20098000FF014058C0F3400070474FF0FF30704746F20020C4F20F000221C0F8801005E083
:2009A00046F20020C4F20F00022101604FF60061CFF6FF71425842F00202425010210160C7
:2009C0000020704703281AD801460020DFE801F019021A2246F20020C4F20F000421C0F8B3
:2009E00094104FF60061CFF6FF71425822F0080242506FF0FF014058C0F3C00070474FF0D0
:200A0000FF30704746F20020C4F20F000821C0F8801005E046F20020C4F20F0008210160D6
:200A20004FF60061CFF6FF71425842F008024250042141610020704740F20801C2F20001E5
:200A4000C86043F67800C1F2080001220068C1E90520BFF35F8F0420086000BF0868002825
:200A6000FCD1704738B58C4643F20414C4F205040146206D4FF0807363EA0000206000BF95
:200A8000206DC001FCD46420C4F2050040F60003C0F6001303604FF69453CFF6FF7341F2FE
:200AA0000070C4F20500C258D2070AD14FF6905ECFF6FF7E012240F80E2000BFC258D2078D
:200AC000FCD04268D20704D1012202604268D207FCD04269D20704D1012202614269D207BB
:200AE000FCD04FF080552846624613F0A3F943F20440C4F204006FF080710560206D21EAE1
:200B000000002060206DC001FCD538BD2DE9F04F43F6C407C1F208079C463F78012F40F02D
:200B2000A28046F20023C4F20F034FF480794FF60066CFF6FF76C3F800909F5947F48077DA
:200B40009F514FF480571F6043F2D87EC1F2080E4FF480680B27012908BF0A2710F8014BE5
:200B6000640004F5C06400BFE5070CBFC3F88090C3F80090DEF80050C3F8808000BF00BF09
:200B800000BF00BF00BF00BFC3F80080013DF3D16408013FE8D10139DCD14FF48050C3F802
:200BA0008000985920F48070985100204FF61849CFF6FF794FF480646FF0FF0B0226E246F4
:200BC00080464946C3F8804000BF00BF00BF00BF00BF00BF1C6053F80B506D0602D501312D
:200BE000F0D32CE0DEF80010A6EB4101C3F8804000BF00BF00BF00BF00BF00BF1C600131CA
:200C0000F4D3082153F80B70DEF80050C3F8804000BF00BF00BF00BF00BF00BF1C60013D49
:200C2000F4D107F040056D0045EA58080139E9D102F8018B0130BAF1010AC2D16046DEF847
:200C40000010A1EB81014FF4806200BFC3F8802000BF00BF00BF00BF00BF00BF1A60013111
:200C6000F4D3BDE8F08F40F20807C2F200074FF000084FEACC0C43F67805C1F20805C900F6
:200C80002D68C7E90180C7E90321C7E905C5BFF35F8F0120386000BF38680028FCD1F86932
:200CA000BDE8F08F2DE9F84F43F6C407C1F208070020387046F20024C4F20F041020C4F814
:200CC00080000420C4F894004FF40040C4F880004FF40050C4F880004FF4805AC4F880A099
:200CE0004FF040084FF60066CFF6FF76C4F88480A05920F00200A051A05920F00800A051CA
:200D0000A05920F00100A051A05920F40070A051A05920F48070A051A05920F48060A0519E
:200D2000A05920F40060A05140F22400C1F604204FF4B071FFF796FE13F018FB00284BD0DD
:200D40004FF480794FF0020B002500BF012038704FF480602060A05940F48060A051C4F801
:200D6000048013F003FBB8B3C4F88480A05920F48060A0510020387035B1022D2CD00820E4
:200D8000C4F8800002E000BF082020600135A05940F00800A05104206061C4F80090A0594C
:200DA00040F48070A051C4F800A0C4F814B0C4F88090642015F0ACFBC4F894B0642015F0BD
:200DC000A7FBC4F80090BE2015F0A2FBC4F880A013F0CCFA0028B9D10420C4F89400A059E1
:200DE00020F00800A0510020BDE8F88F41F22050C4F20500016841F0030101600168C90708
:200E0000FCD044F20400C4F208000021016043F68D00C1F2080001704EF28010CEF200000A
:200E20004FF480510160704741F22850C4F20500016841F0030101600168C907FCD045F2E5
:200E40000400C4F208000021016043F68900C1F2080001704EF28010CEF200004FF400513C
:200E6000016070472DE9F84F40F68077C1F20807387801303870F86B08B10068804743F601
:200E8000BC00C1F208000078012840F0FF8143F2E870C1F208000068012830D143F648002F
:200EA000C1F2080040F6B73102688A429CBF0131016043F6A400C1F20800012101702BF0EF
:200EC00093FA43F64000C1F2080000220168386A411A42F62873C1F2080341F2893A41F20F
:200EE000883600BF9D186C8934B1514504DBED68451BB54280F25A832432B42AF2D102205D
:200F000013F073FA43F27071C1F2080143F2E062C1F2080208601168014443F23079C1F2A4
:200F200008091160D9F80030034443F26875C1F20805C9F800302B681844286043F27F50A9
:200F4000C1F20800037801330370DBB2082B08D100231360037043F2E860C1F20800C90809
:200F6000016043F6BE00C1F20800007848B143F2D470C1F2080043F2E861C1F20801006817
:200F8000086043F68C30C1F208000168802905D143F2E860C1F2080000680BE0016841B16B
:200FA00043F2E861C1F20801096800684843C00900E0002043F2E461C1F208010A68821A86
:200FC00048BF5242642A24D3086043F67031C1F2080145F6C522C0F67C2209684909A1FB1E
:200FE00002124FF0FF316423584343F62F63C3F2AF33A0FB03039809B0EBD21F88BF01EBE9
:20100000FFFFFFFFFFFFFFFFFFFFFFFFFFFFFFFFFFFFFFFFFFFFFFFFFFFFFFFFFFFFFFFFF0
:20102000FFFFFFFFFFFFFFFFFFFFFFFFFFFFFFFFFFFFFFFFFFFFFFFFFFFFFFFFFFFFFFFFD0
:20104000FFFFFFFFFFFFFFFFFFFFFFFFFFFFFFFFFFFFFFFFFFFFFFFFFFFFFFFFFFFFFFFFB0
:20106000FFFFFFFFFFFFFFFFFFFFFFFFFFFFFFFFFFFFFFFFFFFFFFFFFFFFFFFFFFFFFFFF90
:206000000001FFFFFFFFFFFFFFFFFFFFFFFFFFFFFFFFFFFFFFFFFFFFFFFFFFFFFFFFFFFF9D
:20602000FFFFFFFFFFFFFFFFFFFFFFFFFFFFFFFFFFFFFFFFFFFFFFFFFFFFFFFFFFFFFFFF80
:20604000FFFFFFFFFFFFFFFFFFFFFFFFFFFFFFFFFFFFFFFFFFFFFFFFFFFFFFFFFFFFFFFF60
:20606000FFFFFFFFFFFFFFFFFFFFFFFFFFFFFFFFFFFFFFFFFFFFFFFFFFFFFFFFFFFFFFFF40
:20608000FFFFFFFFFFFFFFFFFFFFFFFFFFFFFFFFFFFFFFFFFFFFFFFFFFFFFFFFFFFFFFFF20
:20800000D8400810FDC2031A5349031A09BC011A5549031A5749031A5949031A0000000084
:208020000000000000000000000000005B49031A5D49031A0000000031BC011A658E001AA7
:208040005F49031A000000006149031A00000000000000006349031A6549031A6749031A33
:2080600013C3011A6949031A6B49031A6D49031A094F031A1BD7011A6F49031A7149031A6E
:208080007349031A7549031A7749031A7949031A000000007B49031A7D49031A7F49031AC7
:2080A00017C9011AA3C9011A8149031A8349031A8549031A8749031A8949031A8B49031AB6
:2080C0008D49031A8F49031A9149031A9349031A9549031A9749031A9949031A9B49031AD0
:2080E0009D49031A9F49031AA149031AA349031A0000000000000000A549031AA749031A50
:2081000000000000E3C8011A00000000A949031AAB49031AFFFFFFFFFFFFFFFFFFFFFFFF85
:20812000000000000000000000000000000000004A2D4C696E6B2076313220636F6D706909
:208140006C65642041756720323220323032342031333A32373A353500436F707972696799
:20816000687420323032322D32303232205345474745523A207777772E7365676765722ED5
:20818000636F6D0000000000000000000000000000000000000000000000000000000000A0
:2081A0001AFD5C81DA840DF069A66AD5A97B2D223D792299C9A96F85ED2E5CA798F81C917D
:2081C00051E7AEB64C007C3EFAC75E193FBCF4316E22CEACF3EA2F43005B17B16C38599D8F
:2081E000DECF0733F883BCA0E40C14E04329C729683EB11AD3784F463143DE08CEFF435A6C
:2082000056BC7EED01D88A675ACF06FE900619B77C259ADBCDBBE96BF7407292C7CBB71FEF
:20822000A63144D5065F2C70BFB7075F6E3FCAD4AA843DD40E2065C15BB48C48CA178CFB48
:2082400059A0ED2B03F4E3B6D86F7EB33408D4F6CAD33DC63AD8E9A5B2C0E1F1D259CD2A59
:20826000D4178A5F416A1A118A090C60B49FCFF70DE5CC8E8843A395E3AFB258CFFD709580
:208280006BBAFDD8C5FF17BB643D53939BC4EB8F84E56B35D01C3B9747C8F630A4FBCA3C4D
:2082A0000138FDD5704700BF30BFFDE700000000DB002DE9FF4F81B03A4C3B4D3B4E4FF420
:2082C00080670198013001904FF0000A10F8018D02980130029010F8019D0498082888BF67
:2082E0000820009004980099DDF800B0401A0490012080F310885FEAC87037604FF48070A7
:208300004CBF306028604FF4805028602068FFF7C7FF2F604FEA58082068FFF7C1FF37605E
:208320005FEAC9704FF480704CBF286030602068FFF7B6FF2F604FEA59092068FFF7B0FFDB
:208340004FF48050306037602068FFF7A9FF2F602068FFF7A5FF16480068400000F0800096
:2083600040EA5A0ABBF1010BC5D100064FF480704CBF286030604FF480502860002080F397
:20838000108800980399C0F1080001312AFA00F0039101F8010D0498002892D105B0BDE8F6
:2083A000F08F00003C39081000620F4080620F4000610F4038B541F20050C4F205000321D0
:2083C000016000BF41688907FCD50022C4F208021068C0074EF21000CEF200001ED14FF410
:2083E0000031C0F87411C0F874124EF26031C0F21601516040F2FF3151610B211160AA210A
:20840000552300BF91609360D468FF2CFAD91168090742BF116841F008011160EFF31083E4
:20842000012181F310884FF40031C0F874124EF2314CCEF2000C10248CF80040C0F8F4101F
:20844000AA2191605521916083F31088016821F0030101604EF60850CEF2000048F2000175
:20846000C1F60021016046F2CB50C1F60020017808064CBF002001F0030043F63041C1F296
:2084800008014FF0000C086040B1012401280CD1002145F69073C0F201030AE04BF6207331
:2084A000C0F202030021002403E04FF480714AF6C87343F63840C1F208005A1E026043F6AF
:2084C0003440C1F2080041F26F72026045F20C20C4F200001F2202601820C4F2050040F612
:2084E000000EC0F2001EC0F854E0C0F800C0C0F830E040F60005C0F6001505F140728265DD
:20850000C26A42F00102C26243F63C42C1F2080240F6000C13604FF47A72534343F62C4241
:20852000C1F20802C0F20E6C1360C0F82CC000BF826AD207FCD0C26AC26245654FF47A72C2
:208540000092009A12B1009A013AF9E7002CC26A22F4407442F0800218BF44EA0102C26275
:20856000816AC907FCD040F60401C0F200614163426B02F0F852B2F1C06FF9D1826842F0E1
:208580000102826014220092009AB2F5004F12D84FF48044009A0132009284EA5402C4F3D3
:2085A0004D0462F38E34009AB2F5004FF2D90CF5FF22144303E044F20004C0F21664C46012
:2085C00042F20002C0F230020261026942F0620202611831816000BF4168C907FCD005F196
:2085E00008010163C0F838E0C0F83CE005F184010164406D43F63860C1F20800036038BDF9
:208600002DE9F04F8BB08A468146EFF310800090012181F310883120CDE90320B9F1D05F00
:2086200038BF09F1D0590025C4F208054FEA52282868C00703D0AA20A8605520A86040F2DA
:208640000010C1F240000AA9026804A89047AA2655274FF0070BCDE9019A00BF2868C00773
:208660001CBFAE60AF600020002100BF5AF8002001320FD1002901DD013906E02968C907F5
:208680001CBFAE60AF604FF480710430B0F5007FECD144E0322004904FEA196000241A2877
:2086A00088BF0124C9F34A30082888BF0BEBD000059009F2FF10C0F34A30082888BF0BEBA2
:2086C000D000CDE906042868C0071CBFAE60AF6040F20010C1F240000AA9026804A89047E6
:2086E0000A9818BB4FF400700790CDE9059A3320049043F63C40C1F2080009940068089072
:208700002868C0071CBFAE60AF6040F20010C1F240000AA9026804A890470A9830B9B8F101
:2087200001080AF5007A09F5007997D1009880F3108801AA07CA33F0E5FD90B14AF2201403
:20874000C0F207040120012131F040FC204613F068FF0120002131F039FC204613F061FF8B
:20876000F0E70BB0BDE8F08F03281BD801460020DFE801F01A021B2346F20020C4F20F008F
:208780004FF40041C0F880104FF60061CFF6FF71425822F0010242506FF0FF01405800F00A
:2087A000010070474FF0FF30704746F20020C4F20F000121C0F8801005E046F20020C4F262
:2087C0000F00012101604FF60061CFF6FF71425842F0010242504FF400410160002070470F
:2087E00003281BD801460020DFE801F01A021B2446F20020C4F20F004FF40051C0F88010E8
:208800004FF60061CFF6FF71425822F4007242506FF0FF014058C0F3402070474FF0FF309A
:20882000704746F20020C4F20F004FF40071C0F8801006E046F20020C4F20F004FF40071B1
:2088400001604FF60061CFF6FF71425842F4007242504FF4005101600020704703281BD81E
:2088600001460020DFE801F01A021B2446F20020C4F20F004FF48051C0F880104FF600615F
:20888000CFF6FF71425822F4807242506FF0FF014058C0F3002070474FF0FF30704746F291
:2088A0000020C4F20F004FF48071C0F8801006E046F20020C4F20F004FF4807101604FF67A
:2088C0000061CFF6FF71425842F4807242504FF4805101600020704703281AD801460020DE
:2088E000DFE801F019021A2346F20020C4F20F004021C0F884104FF60061CFF6FF71425829
:2089000022F4806242506FF0FF014058C0F3802070474FF0FF30704746F20020C4F20F008A
:208920004FF48061C0F8801006E046F20020C4F20F004FF4806101604FF60061CFF6FF7168
:20894000425842F480624250402141600020704703281AD801460020DFE801F019021A2267
:2089600046F20020C4F20F001021C0F880104FF60061CFF6FF71425822F0020242506FF0E5
:20898000FF014058C0F3400070474FF0FF30704746F20020C4F20F000221C0F8801005E003
:2089A00046F20020C4F20F00022101604FF60061CFF6FF71425842F0020242501021016047
:2089C0000020704703281AD801460020DFE801F019021A2246F20020C4F20F000421C0F833
:2089E00094104FF60061CFF6FF71425822F0080242506FF0FF014058C0F3C00070474FF050
:208A0000FF30704746F20020C4F20F000821C0F8801005E046F20020C4F20F000821016056
:208A20004FF60061CFF6FF71425842F008024250042141610020704740F20801C2F2000165
:208A4000C86043F63C10C1F2080001220068C1E90520BFF35F8F0420086000BF08680028D1
:208A6000FCD1704738B58C4643F20414C4F205040146206D4FF0807363EA0000206000BF15
:208A8000206DC001FCD46420C4F2050040F60003C0F6001303604FF69453CFF6FF7341F27E
:208AA0000070C4F20500C258D2070AD14FF6905ECFF6FF7E012240F80E2000BFC258D2070D
:208AC000FCD04268D20704D1012202604268D207FCD04269D20704D1012202614269D2073B
:208AE000FCD04FF080552846624613F061FB43F20440C4F204006FF080710560206D21EAA1
:208B000000002060206DC001FCD538BD2DE9F04F43F68817C1F208079C463F78012F40F0D9
:208B2000A28046F20023C4F20F034FF480794FF60066CFF6FF76C3F800909F5947F480775A
:208B40009F514FF480571F6043F69C0EC1F2080E4FF480680B27012908BF0A2710F8014B0D
:208B6000640004F5C06400BFE5070CBFC3F88090C3F80090DEF80050C3F8808000BF00BF89
:208B800000BF00BF00BF00BFC3F80080013DF3D16408013FE8D10139DCD14FF48050C3F882
:208BA0008000985920F48070985100204FF61849CFF6FF794FF480646FF0FF0B0226E24674
:208BC00080464946C3F8804000BF00BF00BF00BF00BF00BF1C6053F80B506D0602D50131AD
:208BE000F0D32CE0DEF80010A6EB4101C3F8804000BF00BF00BF00BF00BF00BF1C6001314A
:208C0000F4D3082153F80B70DEF80050C3F8804000BF00BF00BF00BF00BF00BF1C60013DC9
:208C2000F4D107F040056D0045EA58080139E9D102F8018B0130BAF1010AC2D16046DEF8C7
:208C40000010A1EB81014FF4806200BFC3F8802000BF00BF00BF00BF00BF00BF1A60013191
:208C6000F4D3BDE8F08F40F20807C2F200074FF000084FEACC0C43F63C15C1F20805C900A2
:208C80002D68C7E90180C7E90321C7E905C5BFF35F8F0120386000BF38680028FCD1F869B2
:208CA000BDE8F08F2DE9F84F43F68817C1F208070020387046F20024C4F20F041020C4F8C0
:208CC00080000420C4F894004FF40040C4F880004FF40050C4F880004FF4805AC4F880A019
:208CE0004FF040084FF60066CFF6FF76C4F88480A05920F00200A051A05920F00800A0514A
:208D0000A05920F00100A051A05920F40070A051A05920F48070A051A05920F48060A0511E
:208D2000A05920F40060A05140F63660C1F604204FF4B071FFF796FE13F0D6FC00284BD028
:208D40004FF480794FF0020B002500BF012038704FF480602060A05940F48060A051C4F881
:208D6000048013F0C1FCB8B3C4F88480A05920F48060A0510020387035B1022D2CD00820A5
:208D8000C4F8800002E000BF082020600135A05940F00800A05104206061C4F80090A059CC
:208DA00040F48070A051C4F800A0C4F814B0C4F88090642015F0B0FDC4F894B0642015F037
:208DC000ABFDC4F80090BE2015F0A6FDC4F880A013F08AFC0028B9D10420C4F89400A05995
:208DE00020F00800A0510020BDE8F88F41F22050C4F20500016841F0030101600168C90788
:208E0000FCD044F20400C4F208000021016043F65110C1F2080001704EF28010CEF20000B6
:208E20004FF480510160704741F22850C4F20500016841F0030101600168C907FCD045F265
:208E40000400C4F208000021016043F64D10C1F2080001704EF28010CEF200004FF40051E8
:208E6000016070472DE9F84F41F28007C1F20807387801303870F86B08B10068804743F6F4
:208E80008010C1F208000078012840F0FF8143F6AC00C1F208000068012830D143F60C10AF
:208EA000C1F2080040F6B73102688A429CBF0131016043F66810C1F20800012101702BF09B
:208EC000D1FD43F60410C1F2080000220168386A411A42F66473C1F2080341F2893A41F23E
:208EE000883600BF9D186C8934B1514504DBED68451BB54280F25A832432B42AF2D10220DD
:208F000013F031FC43F63401C1F2080143F2A872C1F2080208601168014443F2F479C1F270
:208F200008091160D9F80030034443F62C05C1F20805C9F800302B681844286043F2EF5061
:208F4000C1F20800037801330370DBB2082B08D100231360037043F2B070C1F20800C908B1
:208F6000016043F67D10C1F20800007848B143F69800C1F2080043F2B071C1F20801006898
:208F8000086043F62060C1F208000168802905D143F2B070C1F2080000680BE0016841B14F
:208FA00043F2B071C1F20801096800684843C00900E0002043F2AC71C1F208010A68821A56
:208FC00048BF5242642A24D3086043F62C41C1F2080145F6C522C0F67C2209684909A1FBD2
:208FE00002124FF0FF316423584343F62F63C3F2AF33A0FB03039809B0EBD21F88BF01EB69
:20900000D21040F20021C4F20001C0438A8810440880002013F062F9044641F6CE106043F3
:20902000810AB0F5482F43F60C00C1F2080038BF002143F62808C1F208080160D8F8000014
:20904000084443F6240BC1F2080BC8F80000DBF800000844CBF8000043F67310C1F208007D
:209060000078012840F0A88043F63C05C1F20805286801302860012013F030F9201A49F2B2
:20908000A861C0F20C0101FB00F054BF8011002044F64031C0F24C018842A8BF084643F6F6
:2090A0000001C1F20801086043F62001C1F208010A6802440A6043F61C01C1F208010A68CF
:2090C00002440A6043F66001C1F208010A689042C8BF08602968642907DB43F65C01C1F20E
:2090E00008010A689042C8BF086043F66802C1F208024CF2C063C0F22D0315680021984219
:209100000B46C8BF6B1C43F66C04C1F208041360266844F24025C0F20F05A8420D46C8BF62
:20912000751C256043F66406C1F2080641F68024C0F20604D6F800A0A042C8BF0AF101014A
:2091400031604CF2C16AC0F22D0A5045A8BF022B15DA44F24122C0F20F029042A8BF092D49
:2091600011DC41F68122C0F20602904243F62C05C1F20805A8BF28291EDB032008E0581C42
:209180001060012000E0022043F62C05C1F2080543F63801C1F20801086043F66810C1F218
:2091A0000800007840B929F00DFA01204FF4FA710A46134630F070FE43F61800C1F2080004
:2091C0000168013901602DD10A210160D9F800000021C9F80010D8F8002043F62003C1F23F
:2091E0000803C8F80010D3F800A019604CF6CD41CCF6CC41A0FB010343F63000C1F20800CE
:20920000DB080360A2FB010243F60800C1F20800D2080260AAFB010143F2FC70C1F208002D
:20922000C908016043F61400C1F208000168013901602BD164210160286800212960DBF801
:20924000002043F61C03C1F20803CBF80010D3F800A0196048F21F51C5F2EB11A0FB010325
:2092600043F61000C1F208005B090360A2FB010243F60400C1F2080052090260AAFB010127
:2092800043F2F870C1F208004909016043F62410C1F208000168013101600A2940F0D380E9
:2092A0000021016043F60C10C1F2080040F20008C2F2000801680131C8F80410016043F61D
:2092C0008A10C1F20800007801280CD143F62440C1F20800007830B9386A4DF2BF41C0F26F
:2092E000010188420DDCEFF31080012181F310880821C4F20801AA220A6055220A6080F3A7
:20930000108843F61C16C1F208063568012D2FDB43F6E80AC1F2080A0CD1DAF8000062288B
:2093200000F10100CAF8000004DC0020002130F04DFE06E000240020012130F047FECAF87A
:2093400000406FF00040854208BF0125681C306040F2B2218D4218DB642132F073F9002864
:209360004FF000000CBF0021012130F02FFE0CE0002D0ADA0020002130F028FE30680138FE
:20938000306010F5FA7F00F0118143F28050C1F2080043F2B072C1F208020168126840F254
:2093A0004C439A420BD345F6FF32C0F22652914209DC11B94268013242600A3104E011B1EC
:2093C0004168013141600021016031F093FDB0FA80F04109012030F0F9FD43F62810C1F21F
:2093E00008000168013101600A292CD10021016043F61010C1F20800016831B101680131BD
:2094000001600068332880F0AD8043F62640C1F208000078012804D104F04EFF002800F062
:20942000A98043F62C10C1F208000168013101600A2908D10021016043F60810C1F208003D
:2094400001680131016043F6C410C1F20800061D386AC0F3420900F0010A0020012543F60B
:209460003068C1F2080800BF318899B14C1E0FD116F8011C002914BF04210221745A16F83A
:20948000011C81F0010106F8011C002130F058FD34800DE016F8031C51B1D8F80010BAF130
:2094A000000F18BF11F0070102D0494630F048FD0A36E8074FF001004FF00005D4D1F86B3C
:2094C00018B1816A4FF491708847386B60B30120787187F83400F86B18B1816C4FF49170F5
:2094E00088473878012805D1786818B1F86B28B1806802E0F86B08B1406880474FF08000F5
:2095000080F3118800BF00BF3878012803D1786808B112F017FC3878013838704FF0000096
:2095200080F31188BDE8F88F386A07F124030ECB01300132386243F10003C7E90A23401AED
:209540005CBF01207871B8680028C4D090F848100029C0D0013980F84810080604BF012075
:209560003871B8E744F22130C1F23420C8F8000012F08CFE41F270700021C8E9001032247E
:209580000825C4F20805AA264FF0550A4FF47A7013F047F8EFF31080012181F310882E60D0
:2095A000C5F800A080F31088013CEFD112F06EFEF8B515460E460446C068884207D9606898
:2095C00040F8265005BB204613F0DAFC1CE0DDB1771CB84215D2204639462BF0BBFD002800
:2095E00048BFF8BDE168B9420AD2606800EB8100711A0131002200BF40F8042B0139FBD150
:20960000E760606840F826500020F8BD2DE9F843002948D00546C068002844D00F462846B4
:2096200013F004FD38441F30410928462BF092FD002848BFBDE8F8837E0911D06968EA681F
:2096400001EB8600920012F00FFE6868B10012F0D5FDE8688319EB6017F01F0701D122E06A
:20966000EB6803B3D5F804C04FF00009A7F12002C7F1200E614618460C6824FA0EF6002AA3
:2096800004FA07F85CBF4FF0000804FA02F648EA090841F8048B0138B146EDD11EB14CF869
:2096A0002360581CE8600020BDE8F8832DE9F04F89B014460E468346039203A8043014217D
:2096C00012F09CFDDBF80C90B9F1000F6AD04FEA490A03A851462BF03DFD002866D4CDE952
:2096E0000164CDF818A0049E4FEAC901304612F085FDA9F1010EDBF804100020324600BF02
:2097000000F1010CCC4511D2D1F8008000270425704600BF53594C59E4FB6873575104355D
:2097200001381F46F6D1501904E000BFC000043030440023043103600832AEF1010ECC459C
:209740006046DDD103A80121FFF760FF00283FD4DBF804100498002200230027DDE901643E
:2097600050F8338051F82350E5FB657840F8337000EBC30701337D6818EB0508C7F8048079
:2097800042F100074B45EBD3CDF818A0BAF1000F08D0AAF1010100BF50F8212012B90691EB
:2097A0000139F9D203A958462BF012FD054603A814F027F8002D07D458463146224609B0D9
:2097C000BDE8F04F13F0F6BC284609B0BDE8F08F0546DDE90164EAE72DE9F04790B09A46F1
:2097E0001646894604460A930AA80430142112F005FD0020049004A80430142112F0FEFC73
:20980000E76837B1206920B1F068E0B1306938B919E0F06808B1306958B927B1206910B16E
:209820003046214601E02046314613F05BFC002807D420463146524613F0BCFC002843D4C1
:20984000E768002F51D0D9F80C00002844D000206946CDE904010421CDE90610CDE9080017
:209860000AA8314614F049F800282DD4484613F0DDFB451E24D40DF1280800BF40463146A3
:209880005246FFF713FF00281ED4D9F80C00B0EB551F05D96809D9F8041051F8200000E0A5
:2098A000002005F01F01C840C00707D0404621463246534613F014FE002805D4013DDDD5C9
:2098C0000AA9204613F0D3FF07460AA813F099FF04A813F096FF09E04AF27061C1F60121ED
:2098E000204613F0C4FF074600E00027384610B0BDE8F0872DE9F04F99B005460792D0E953
:209900000203801843F10002C5E90202089105F1240008A907AA02902BF0F0FB002800F0FD
:2099200096800DF1240A47F69918C5F682280195D5E904E9D5E90643D5F820C0002100BFBD
:2099400050F8212012BA4AF8212001311029F7D100206746CDE903341D4622464946CDE932
:20996000059E734699469646AB460F282CD900F10D0202F00F0200F1080303F00F035AF84D
:2099800022205AF823305A40831C03F00F035AF823305A4000F00F035AF823506A401328B7
:2099A0004FEAF2754AF8235007EBF96303EBF2760FD9272814D88EEA0B024A404EF6A13364
:2099C000C6F6D96321E000BF5AF8202007EBF9639E182BEA010201EA0E031A44424415E04C
:2099E0003B280BD801EA0E0241EA0E0303EA0B031A434BF6DC43C8F61B7306E08EEA0B027B
:209A00004A404CF2D613CCF662231A44B31801304FEAB10250285F4675464946A2D10BEB38
:209A20000C00DDE9031771443A44DDE905752B44019D4F44C5E90437C5E906212862029845
:209A400008A907AA2BF05AFB00287FF471AF19B0BDE8F08F00B5027882B100F1010C4FF0ED
:209A6000000E00BF1CF80E200EF1010E002AF9D10A783AB9BEF1000F24D50EE00A780AB37C
:209A80004FF0000E002200BF01EB020C01329CF80130002BF8D1964501DA012000BD012AF3
:209AA00010DB7044A0F1010C002300BFC81810441CF803E010F8010C8645EED1D018013B99
:209AC0000128F3D1002000BDF8B514460D46064690F83C0020B97068716B002200F01AF8A1
:209AE00006F10C0207CA8F1AA742A8BF2746104429463A4612F05CFBD6E90401394471617B
:209B0000814202D1304613F033FEE41B08BFF8BD3D44E5E72DE9F84F93460546002028670D
:209B2000012085F8800005F14408002A43F2AC1AC1F2080A60D042F2DE31C1F60421404606
:209B400013F080FE4046594613F07CFE40F26361C1F60421404613F075FEA86950B14FF6BD
:209B6000D711C1F60321404613F06CFEA96940462BF07AFB686950B142F2FE31C1F60421F6
:209B8000404613F05FFE696940462BF06DFB687F08B9287F50B1DAF83C10002904BF4FF665
:209BA000E111C1F60321404613F04CFE95F89B0030B140F27861C1F60421404613F042FE4C
:209BC000E96F11B1404613F03DFE95F89A0040F29161C1F60421002804BF4CF24631C1F629
:209BE0000321404613F02EFE404613F0C1FD95F89A002867BDE8F88F0E46087838B1701C1A
:209C0000002700BFC15D01370029FBD100E00027781E42F2D63BC1F6042B00BF00283FF530
:209C20008AAF315C01382E29F8D100F10109DAF8184000BF44B1231D304639464A4600F077
:209C400021F8B8B92468F5E700244AF2A86AC1F6012A42F2D63BC1F6042B00BF0AEB0403D8
:209C6000304639464A4600F00DF828B90834602CF4D102E083465EE7834643F2AC1AC1F295
:209C8000080A58E7F8B51F461B681D783DB15D1C002400BF2E5D0134002EFBD100E0002441
:209CA000D64331448C4205D11044411C184612F01DFA08B10020F8BD7868F8BD2DE9F843D6
:209CC00088460546012600BF012A03DCB8FBF6F00A2804D3013A06EB86004600F4E795F879
:209CE0003C0020B96868696B0022FFF713FF42F27654C1F604244CF6CD49CCF6CC4900BFB6
:209D0000B8FBF6F72846E15D13F0D9FE07FB1688A6FB0901C808092E0646F1D8BDE8F88396
:209D20002DE9F04F85B00E46044600680121417394F83C00002840F0CD809A46904643F265
:209D4000AC17C1F2080760683A6900212AB1037BB3F1640518BF154600E00025DDF83C90B4
:209D6000012284F83C2001672046314613F06AFD4FF64521C1F60321204613F063FD25B114
:209D800040F29161C1F604211EE040F2B771C1F60421204613F056FD98F8000050B108F149
:209DA000010040F2122100BF013110F8012B002AFAD101E040F2122120460022FFF77EFFE2
:209DC00040F2C871C1F60421204613F03BFD40F2911081454CD14CF28C31C1F603212046A9
:209DE00013F030FD38684CF29F31C1F60321002804BF4FF6BD21C1F60321204613F022FD39
:209E000040F2E571C1F60421204613F01BFDDAF80400416819B94FF6C321C1F603212046A2
:209E200013F010FD4FF6D521C1F60321204613F009FD3868B8B1DDF838B04FF6D721C1F6D3
:209E40000321204613F0FEFC03CF01238268D1F800A020465946D0474FF6D521C1F6032100
:209E6000204613F0EFFC4CF24631C1F6032103E042F26241C1F60421204613F0E3FC2046BA
:209E800013F076FC6DB1019460680121016700200490CDE90268ADF8109001A8A84703286C
:209EA00018D1E06A30B94CF24631C1F60321204613F0C8FC2046414613F0C4FC0A264FF6A4
:209EC0008725C1F6032500BF2046294613F0BAFC013EF9D1204613F04BFC05B0BDE8F08F18
:209EE00010B5D0E902C24FF0000EF44512D00368002100BF9C5C202C01D0092C09D144689D
:209F00000132A242A8BF724601318C45F2D1E64600E08E46ACEB0E01C0E90212704610BD7F
:209F200030B583B0019043F2AC10C1F208008DF80810856A35B101AC6968204688472D6812
:209F4000002DF9D103B030BD2DE9F04FADF5037D0290032A03DA0DF5037DBDE8F08F9846D3
:209F60008A4603AF7C1C44300090002550462BF019FA6FF02F0151FA80F10A290ED300F08B
:209F8000DF0141391A2909D36FF02C0151FA80F1022903D3C1B25F2906D100BF785501356B
:209FA000B5F5FF7FE2D1D6E7002078553D29D2D1681C01902E4600BF50462BF0F3F9C1B2BB
:209FC000B8F1000F16D025291ED150462BF0EAF9834650462BF0E6F981465FFA8BF02BF003
:209FE0002BF983465FFA89F02BF026F940EA0B1003E000BF31B3262924D0A0550136B6F583
:20A00000FF7FD9D1A7E700BFA1F130020A2AF4D300F0DF02413A1A2AEFD32B2901D1202054
:20A02000EBE76FF0200252FA80F21F2A08D8012303FA02F243F2C933C8F200031A42DCD1DA
:20A040005F29DAD00020A055019807EB0009029839462A464B4613F0E1FE00250028BFF627
:20A0600085AF0298806A8368002B3FF47FAF009839464A46984779E72DE9F04383B043F21A
:20A08000AC12C1F20802074692F8640010B1012087F8800097F8810008B1002639E0894652
:20A0A00007F1440819F8010F38B1881C002400BF015D01340029FBD100E00024B86AC568F0
:20A0C000296881B1002600BF4846224632F01AF918B905EBC6004268FAB905EBC6000136DC
:20A0E00081680029F0D14FF4CA700021CDE9001040F60E01C1F6042140F62702C1F60422CC
:20A1000040460023FFF70CFE4FF0FF36404613F02FFB304603B0BDE8F083B86E10B1F96DE1
:20A12000404601E0404600219047EFE72DE9F84F0446007F01281CBF0120BDE8F88F934614
:20A140000D46486A48B1284613F046FD95F83D00002853D00020BDE8F88FDDF82880286ADD
:20A16000404577DD04F1340A94F8990080064CD450462BF017F9E36DD4E919717A1E914245
:20A1800065D05FFA80F903EB010CA9F130060A2E0FD309F0DF06413E1A2E0AD3A9F1210690
:20A1A0000D2E11D8012202FA06F643F2C93216420AD08CF80090481CE16D0022B8F1010864
:20A1C0000A54A066D4D13EE0B9F15F0FF1D0CE1CBE423BDAC0F3031325278CF8007042F243
:20A1E0007657C1F6042700F00F00FB5C8CF8013017F800900CF1020C0231DAE72046594602
:20A20000FFF73AFFC017BDE8F88FA869D4E90D12236C1944A2EB0309C14501DD424608E046
:20A220004A4611F0C5FFA8EB0902A869DAF80010484411F0BDFF504641462BF09DF8A86911
:20A24000002100F808100A9868627CE70A4600209854A2664FF0FF30BDE8F88F38B541F2E0
:20A260008005C1F208050246287801302870506931B151620B6813600A6013B35C6918E0C7
:20A28000294651F80C3F53B15C69A0420CD200BF19461B681BB15C69A042F9D306E05162B9
:20A2A000002010600A600CE005F10C01516213600A605A62844214BF002092F8490082F863
:20A2C0004800107C70B94FF0800080F3118800BF00BF104614F0B6F8687818B94FF0000040
:20A2E00080F31188BDE8384014F0F7B800B50346808AD3F804C0D3F810E00EFB00CE00BF9A
:20A300001EF8012B01F8012B0138F9D19868D3E9031201328A4228BF002288429868A0F19F
:20A320000100986041F28000C1F208001A61407809D118B94FF0000080F311881846BDE88A
:20A34000004014F0F5B800B100BD4FF0000080F3118800BDF8B50D4641F28006C1F208061C
:20A360000446F06B38B1076BC16B20468847014649202A46B8473078013030704FF0800025
:20A3800080F3118800BF00BFA06850B9204640212BF0E6F84FF0800080F3118800BF00BF19
:20A3A000F2E760682169405C2870A068D4E9031201328A4228BF00228842A068A0F10100F8
:20A3C000A0602261707808D118B94FF0000080F31188204614F0ACF804E018B94FF000001B
:20A3E00080F3118814F079F8F06B20B1816C4920BDE8F8400847F8BD41F28002C1F2080207
:20A400000146107801301070002050704FF0000080F3118843F68610C1F20800017000BFD7
:20A4200001780029FCD17047C0EBC00042F2C851C1F2080101EBC00043F21421C1F20801B0
:20A44000C27901EB0210002181724FF0800080F3118800BF00BF41F28000C1F2080041783F
:20A46000013141700121914046F2B412C4F20002116000BF13680B42FCD1417801394170E7
:20A48000407800B170474FF0000080F3118870474FF0800080F3118800BF00BF41F280009E
:20A4A000C1F2080041780131417046F24011C4F2000102220A6000BF0A689207FCD4417824
:20A4C00001394170407818B94FF0000080F311880020704738B546F24015C4F2000502218E
:20A4E000686C296029688907FCD400F08070696C08436864686E40F0080068660A20A8662E
:20A500004FF00210686243F25070C1F208004FF440710468204611F071FE0820012100BF31
:20A5200021504030B0F5427FFAD148F20000C2F2400020602064AC61286820F47F0028601F
:20A5400043F22C70C1F2080040F25711C0F2010100688031002804BF40F25711C0F20101CF
:20A56000A96038BD2DE9F04F89B046F24015C4F200056868A96801EA000A40F2D710C0F266
:20A58000010000EA0A0068605FEA0A6009D543F22C70C1F20800006818B1696CC90718BF34
:20A5A00080475FEACA7000F05083EE6FCDF808A0002E00F0938142F2C85BC1F2080B4FF036
:20A5C00000090396012000FA09F0304200F0DC80D846E86743F21420C1F2080000EB091B67
:20A5E0005F4617F80A0F002800F0CD80DBF804000022416843F67F13C1F20803C0691A704B
:20A60000C1F30E41461A48462BF0EEFB9BF80B100490D1B1C0EBC00008EBC004E26812B152
:20A620002069314690472069616930442061881B6061049821462BF0F7FC0921002808BF6D
:20A640000121606B00F070FD76E0DBF80C30059390B3C0EBC00008EBC005EA681AB11846D2
:20A6600031469047059BAA465AF8100FE8B32A46344652F8141FB14298BF1468194684B12F
:20A6800019460192224611F093FDDAF8000020440199CAF800000868001B08600598011993
:20A6A000361B04980C4629462BF0BEFC21460924002808BF01241AE042F63003C1F208034C
:20A6C000587BC8B3002400BF03EB8401D1F844213AB105983146904742F63003C1F20803A9
:20A6E000587B01348442EFD326E001241946DDF808A0CEB105F11C00324615F015F9697EC0
:20A70000C90702D0298888420ED22E4616F8180F50B142F63000C1F20800D0F85C01816A5F
:20A720000498884700203070686B214600F0FCFC46F24015C4F20005B9F1000F1CD038782F
:20A7400000B343F67F10C1F208000078D0B90498C0EBC00208EBC2010869002800F0B18049
:20A7600038F832304F699F4240F2AF80C97E002908BF3B460246AAE043F68111C1F208013C
:20A7800000200870039EC3464FF4803000FA09F0304200F08F80E86709EB490043F2D4315A
:20A7A000C1F2080101EB8000817A002900F08280406800EB411050F81C0C00067AD4B9F109
:20A7C000000F484618BF40F080002BF00DFB044698B1C4EBC4000BEBC000014651F80C2FAB
:20A7E000022A0ADB4FF0FF320A60C17D406B002914BF0421062100F097FCC4EBC4000BEB51
:20A80000C008474617F81A0F00284FF0000047F80E0C0FD0204600F0C1FC3878022849D8FE
:20A8200098F81800002845D0B8F80A10204615F07FFB3FE042F63007C1F20807D7F85C0108
:20A84000816B2046884754B1B8F80A10204615F06FFBD8F83400402100F066FC2AE097F9E2
:20A8600009000028394619DA00F07F04D1F85C014C72C16920468847002C42F63000C1F238
:20A88000080018BF0124007A00F0FB0040EA840015F002F942F63001C1F2080191F8D3011F
:20A8A00040B18DF81800D1F85C0106A9026C0420904700BF09F10109B9F1060F7FF482AEA7
:20A8C0000CE00023039E059A02E002463B46039E58464946059215F0B6F854E7E86E0028AD
:20A8E00000F0B3814FF00110E8670120E863E86EC10700F0A881E866E86EC007FCD143F285
:20A900005070C1F208000168286840F400502860886ACA6A2B689B04F6D5CDE90602296845
:20A9200021F4005142F63007C1F208072960D7F83C91B9F1000F0FD006AC00BFD9F804106D
:20A9400020468847002800F07E81D9F80090B9F1000FF3D19DF8180010F06001D7F85C8113
:20A960001CD0202951D0402940F06A817878002800F0668107F148064FF0000906AC00BF0F
:20A9800056F8201B29B120468847002800F05B81787809F101098145F2D351E19DF81910BC
:20A9A0000B2969D8DFE811F00C0079004C017C004C0181009E004C01F100070118013D0103
:20A9C0009DF81A10002940F03B819DF81B10002940F036819DF81E10022940F031819DF86E
:20A9E0001F10002940F02C8100F00F00022800F01F83012800F03C83002846F24015C4F224
:20AA0000000540F01D81F87A41E3C0B200F01F0002289DF81C0026D115F070FB002800F1F1
:20AA20000F817A786AB10121012A98BF0A4601FA00F307F134010E88334203D12031013AFF
:20AA4000F9D10021BA7862B10123012A98BF1A46834007F1F80007883B4213D12430013A8E
:20AA6000F9D181B9ECE07978884280F0E98007EB401000F1340106E0302900F0E48031291D
:20AA80002DD0DDE001460969002900F0D98006A88847002840F0D480D5E006A8002101E043
:20AAA00006A801212BF028FBCDE0387C9DF81A40002800F06F81D8F81C1020468847002CD3
:20AAC000204618BF0120397A01F0FB0141EA800014F0E2FF7C72387C012840F0B4802BF09E
:20AAE00093FBB0E09DF81B00411E0E2900F29C820020DFE811F00F009901550199029902C5
:20AB00006E018E019902990299029902990299029902A00115F03DFB40F68074C1F2080433
:20AB20004FF489712180B988A180B979A17142F2C851C1F2080101280978C8BF0921E171DB
:20AB4000B7F8D011B1F5047F0A4688BF4FF404720228A8BF0A466280D7F87C0101882181B2
:20AB600040886081D7F87401804740F20121E1812073000A6073D7F87C010121C068617490
:20AB8000002818BF0320207421E242F2C850C1F20800012140F68072C1F20802C0E907211D
:20ABA0008176002181758182387AC0F340001070D8F8301026E29DF81A40022C40D22BF0FD
:20ABC00023FB002C18BF0124387A00F0FD0040EA440014F061FF36E09DF81A0080BB9DF829
:20ABE0001E0001282CD19DF81C007978884227D2397A01F00601062922D107EB401042F269
:20AC0000C851C1F2080101220DF12303C1E907328A7600228A758A8290F83A008DF823009E
:20AC2000C6E7387A00F00600062809D19DF81CA07878824504D89DF81B00002800F0098181
:20AC4000D8F824008047DDF808A05FEACA3019D5A86BC00716D043F68110C1F208000178CD
:20AC600071B9012404704020079043F21420C1F2080006AAC1680691012114F0D5FC2C67FC
:20AC80000120A8635FEA4A605ED543F27471C1F2080100200968C43143F21424C1F20804DA
:20ACA00043F2D439C1F20809002200BF8B5823F080138B5004EB8203987602EB42034B4406
:20ACC00004329875142AF1D14FF0FF37AF630026EE636F60E86EE866E86FE867286F48B18A
:20ACE000686CC005FAD4FFF7F5FB286840F001002860F3E76F670120A07243F68110C1F25E
:20AD0000080089F80A60067042F63000C1F208004672017A017802290CD398BF022101393D
:20AD200042F2C852C1F208024032002302F8383B0139FBD1017AC27A02F00102C27201F02F
:20AD40001000083014F0A8FE5FEACA5048BF15F01AFB5FEA4A701AD5686C6C6C696C00F01A
:20AD6000010901F0400010EB090008D042F63000C1F20800007A00F0FE0014F08DFEB9F1F8
:20AD8000000F02D014F0800001D015F0FCFA09B0BDE8F08F2BF038FA44F08000787252E781
:20ADA0009DF81A90B9F1040F00F2D6804FF6FD24C1F60324DFE809F003DDE1E5EB0040F684
:20ADC0008070C1F2080040F20431C0F209410160FDE015F09EF8002800F0268115F0D9F9F6
:20ADE000012800F3218140F68070C1F2080040F20A61C0F20021016001210181B9888180FD
:20AE0000B979817142F2C851C1F208010978C171DDE015F07EF8002800F0068115F0B9F9C4
:20AE2000022880F20181012000F0CCFC40F68070C1F2080008E0D7F8B801002800F0F4803E
:20AE40008047002800F0F0808178C27841EA0221C2E007EB4A142BF0D7F99DF81A000394FF
:20AE6000002805903ED084F83A0007F1F409002442F2C850C1F2080040300490A04699F8B6
:20AE80000000824526D199F806000599814221D1387802281ED3B9F804B0049D01262BFAED
:20AEA00006F0C00711D030464FF0FF312AF014FF2C70D7F85C010021026A30469047D7F871
:20AEC0005C01C16B09B1304688473835013638788642E4D309F124095FEAC8704FF0010827
:20AEE000CDD02BE04FF0000884F83A803878022824D3B4F8349042F2C850C1F2080000F1F4
:20AF00004004012629FA06F0C00712D030464FF0FF312AF0E1FE84F80080D7F85C010021DD
:20AF2000026A30469047D7F85C01C16B09B1304688473834013638788642E3D3039846F25D
:20AF40004015C36C002BC4F200053FF47CAE026D05995046984776E6A9F10500397B88422F
:20AF600053D207EB8000143046F24015C4F200050AE0D7F87C01043006E0D7F87C010830DA
:20AF800002E0D7F87C010C300468002C4CD0204611F0E8F840F68071C1F2080103224A708A
:20AFA000022202EB40020A7088B102230022FF2B03D901340138FAD109E02678CE5402D189
:20AFC0004FF48073F5E75E1802337270F1E740F68070C1F20800017842F2C852C1F2080295
:20AFE0000123937600239382BDF81E30994238BF0B46C2E907032CBF002001209075D7F811
:20B000005C01016B002088471DE6D7F8706146F24015C4F200053EB1716848468847002840
:20B0200050D13668002EF7D1D7F85C01406A09E6387A80079DF81C0007D4002846F240151C
:20B04000C4F200057FF4FCAD002015F057F8002846F24015C4F200053FF5F2ADC0EBC000F7
:20B0600042F2C851C1F2080101EBC000007A0EE0387A800746F24015C4F200057FF5E0AD31
:20B0800078789DF81C108142BFF4DAAD002040F68071C1F208010022087042F2C850C1F266
:20B0A00008004A70C161022101620121817682758282D8F830100020884746F24015C4F2D0
:20B0C0000005C0E5044662E72DE9F04104461AB316468846A068002708B3D4E90012E368A7
:20B0E0001844904288BF1046C51AB54228BF3546194440462A4611F05BF8D4E90110E2688E
:20B10000401B2A44511A18BF1146C4E90201A8442F44761BE0D101E0A068002708B900208B
:20B12000E0603846BDE8F08138B540B10C460546D5E90121204690472D68002DF8D138BD23
:20B140002DE9F041984616460C460546069F002F1CD400BF28462146324643462AF056FE0A
:20B16000011D08D1284639462AF018FF0028F1D00020BDE8F0810028FBD1284639462AF0A0
:20B18000E7FE301A38BF0020BDE8F0812846214632464346BDE8F0412AF038BE2DE9F0474A
:20B1A00082B08246C0EBC00042F2C851C1F2080101EBC004254615F81A0F002800F08180B7
:20B1C000BAF1000F02D0E16800297AD1264656F81C1F00294FF0000106F8051C06D00228A9
:20B1E00004D3206A10B9204614F018FC42F63000C1F20800D0F85C01D0F85090B9F1000FFE
:20B2000023D0A08A0190297801AB50463246C84707000198A08234D4781CA246E0605AF83E
:20B22000208FB946474508D9204614F0F7FBA9EB0809DAF80080C145F6D8A8EB0900CAF86E
:20B24000000030684844306024E0216A2788B94238BF0F46791CE1603168436B50463A4682
:20B260009847206AC01B20623068384430602FB120884FF6FF710144394205D00020A08250
:20B2800008E00120E0601CE0B7FBF0F0A18A0844A082012720462AF0E5FE206A88B9287848
:20B2A000022803D3204614F0B9FB0AE03FB1A08A28B114F8160F10B10020207001E00020F0
:20B2C000287002B0BDE8F0870022C0E9011242F63002C1F20802D2F8A01139B10B4600BF8E
:20B2E000834208BF70471B68002BF9D1C2F8A001016070470022C0E9012142F63002C1F216
:20B300000802D2F8681139B10B4600BF834208BF70471B68002BF9D1C2F8680101607047F0
:20B320002DE9F04F85B00446007800F06000402834D0002840F0B2816078062840F0AE8115
:20B34000E078032840F0AA81A0780125EE2840F0A68194F806E0E17941F68C62C1F6032297
:20B3600040F6807CC1F2080C6346B2E89108A3E891081088188042F2C850C1F208004EEA65
:20B3800001218576857500258582122928BF1221C0E907C153208CF81000B6E060785328B4
:20B3A00040F07C812079617940EA012080B2052800F0B580042840F0718194F80680E47961
:20B3C00040F68075C1F208054FF480772846394610F014FF04950025CDE9025743F66917C2
:20B3E000C1F208071020397801EB410100EBC10B02A859462AF056FEDDE90201884205D2A4
:20B4000004990D54DDE9020101300290884205D2049A01231354029801300290884206D2D9
:20B42000049904220A54DDE9020101300290884205D2049A0023135402980130029088426F
:20B44000CDF804B004D2049A3B7813540130029007220023884203D2049D2B540130029054
:20B46000013AF7D148EA042A3A78C2B3002543F21804C1F2080401260DF1080BA84600BF28
:20B48000884207D208EB4802049B14F832201A5401300290884203D20499421C0E5402920E
:20B4A00008EB480004EBC0095846D9F8081014F005FDD9F80C10584614F000FD0622DDE992
:20B4C000020100BF884203D2049B1D5401300290013AF7D108F101083A789045D0D3019870
:20B4E00001210025504538BF824642F2C850C1F208008176858240F68071C1F20801C0E920
:20B50000071A294638BF0121817542F63000C1F20800D0F85C01016B00208847BFE043F611
:20B520006910C1F2080001250178002900F0B780A278012988BF0D4643F21800C1F2080002
:20B540000230002310F8027C974204D0183001339D42F7D1A2E08B4280F0A080D0F8026037
:20B56000002E00F09B8040F68071C1F20801049100254FF48071CDE902510088009002A8F6
:20B5800000212AF08FFDDDE90201884205D204990D54DDE9020101300290884205D2049AB1
:20B5A00001231354029801300290884206D2049905220A54DDE9020101300290884205D2B2
:20B5C000049A00231354029801300290884204D2049A009B135401300290884204D20499A6
:20B5E00000220A5401300290009900295BD04FF0000A019096E8200AF7680DF108084046A6
:20B6000000212AF04FFD404629462AF04BFD40464946022200F066F8042D0AD0032D16D0A4
:20B62000012D019D28D102A85946032200F05AF822E002AD284604212AF034FD584615F063
:20B64000C0F8014628462AF02DFD019D14E002A839462AF027FD019D77B1DDE9020100BFF2
:20B66000884205D2049A9BF800301354013002900BF1010B013FF3D102980499421B4A555F
:20B680004B19170EDF70170C9F70120A5A700AF1010A1036009A9245ABD105E00125284608
:20B6A00005B0BDE8F08F04990870020ECA70020C8A70020A4A70A179E37942F2C852C1F20D
:20B6C000080240F68077C1F20807D7610127977697750025958241EA0321814238BF084665
:20B6E000106212E7F8B516460D46044629B1284610F038FD08B1471C00E00027032E07D091
:20B70000022E09D1780081B220462AF0B7FC03E0790020462AF0C6FC6FB17E1E15F8011BBE
:20B7200020462AF0ABFC013EF8D120460021BDE8F8402AF0A3BCF8BD2DE9F04182B0884601
:20B7400000EB400042F6A851C1F2080101EBC00541F28007C1F2080701AC00BFF86B38B1EC
:20B76000066BC16B28468847014642202246B0473878013038704FF0800080F3118800BFD4
:20B7800000BF00BFA86858B92846402129F0E8FE4FF0800080F3118800BF00BFF2E700BF5B
:20B7A00028462146FEF7A2FD12F097FEF86B10B1816C422088470198404504BF02B0BDE80F
:20B7C000F081CBE72DE9F04F83B0834640F68076C1F2080600207080092535700420B071E0
:20B7E000012070710720BBF1000F08BF022042F63007C1F208077070B87A7978317140F076
:20B800008000F0714FF48070CDE9010607F5A17414F0BFFC0128C8BF07F24314207830724D
:20B8200000957878A0B30025EA4607F1F40900BFD7F8640118B1426828465146904707EBB2
:20B84000451000F13402504629465B4600F024F8B878C0B14FF000084C4600BF2078854222
:20B860000BD114F096FC94F90110884205DB221D504629465B4600F00FF808F101082434D8
:20B88000B8788045EAD3013578788542D0D3009D758003B0BDE8F08F2DE9FA4F83B0154610
:20B8A000074610880021B1EB500F0AD04208002002F0010318445308B1EB520F1A46F7D171
:20B8C0000146D7E90002904206D2BA6809231354D7E9000201303860904206D2BA68042382
:20B8E0001354D7E9000201303860904206D2BA68039B1354D7E9000201303860904206D250
:20B90000BA68AB781354D7E9000201303860904205D2BA681154D7E9000201303860904263
:20B9200006D2B968EA780A54D7E9000201303860904206D2B9682A790A54D7E90002013004
:20B940003860904206D2B9686A790A54D7E9000201303860904205D2B968EA790A5438688D
:20B9600001303860AB681BB1A97803983A46984714F0CFFA009014F00CFC42F63008C1F278
:20B980000808019098F800000228C0F0A08042F2C850C1F2080000F138040198C0F10100FD
:20B9A00002904FF001094FF0000A00BF288820FA09F0C00700F08380D7E90001884206D2C4
:20B9C000B96807220A54D7E9000101303860884206D2B96805220A54D7E900010130386063
:20B9E000884206D2B968E2790A54D7E9000101303860884209D2A179627A02F03C02114322
:20BA0000BA6811543868013038606088049929B1A179029A14F0D9FA08E000BFDDE90012CB
:20BA2000914202DDA17914F0D0FA2080B0F5806F28BF4FF4806081B238462AF01FFBA6881B
:20BA400014F0A7FBA179012906D0032910D1A0B1002E08BF082602E008B9F01DC608002007
:20BA60000130BAEB560F4FEA5606F9D10EE000BF0228ACBF0020012008E0F01DBAEBD00F30
:20BA800014BFC0080420FF2828BFFF20D7E90012914204D2BA685054386801303860D8F840
:20BAA000BC2112B1204639469047D5F80CB0BBF1000F04D0E279A97803983B46D84709F161
:20BAC0000109383498F800008145FFF46FAF05B0BDE8F08F00B50B0BC1F3032CC1F3421EEE
:20BAE000C90658BF50F8233050F82C20BEF1060F07D8DFE80EF004090B0E11141700D1187E
:20BB000012E002FB03F10FE0D11A0DE002EA03010AE042EA030107E082EA030104E002FA3A
:20BB200003F101E022FA03F140F82C10B1FA81F149094164002000BD0A0BC36BD0F848C0A8
:20BB400003EB8202C263C1F3032200EB82006FF0030202EA912149420CEB030252F8043BF6
:20BB600040F8043B0431F9D1002070472DE9F04782B01C4691468A460746406A00F01F08E2
:20BB800001AE00BF1AF8015B242D00F24880DFE805F04C131313131313134E50161616163B
:20BBA000161616531C1C1C1C1C1C1C562323592A2A5C31315F3838003846294629E03846E2
:20BBC000102115F086FDA91E22E03846112115F080FDA5F10A011BE03846132115F079FDE8
:20BBE000A5F10D0114E03846172115F072FDA5F110010DE03846122115F06BFDA5F1130127
:20BC000006E038461B2115F064FDA5F1160100BF3846324614F05CFE002828D4019849F860
:20BC2000040B013C7FF4AEAF1BE0B86902E0386A00E0F8690190F2E7384611210AE0384685
:20BC4000132107E03846172104E03846122101E038461B2115F03DFD384631462AF05CFC3D
:20BC6000DAE73846414615F034FD002001E04FF0FF3002B0BDE8F0872DE9F0471C46924604
:20BC800089460746406A00F01F0800BF19F8016B5AF8045B242E00F24B80DFE806F04D13AE
:20BCA0001313131313134F5116161616161616531C1C1C1C1C1C1C562323592A2A5C3131BA
:20BCC0005F3838003846314629E03846102115F000FDB11E22E03846112115F0FAFCA6F1D3
:20BCE0000A011BE03846132115F0F3FCA6F10D0114E03846172115F0ECFCA6F110010DE0C7
:20BD00003846122115F0E5FCA6F1130106E038461B2115F0DEFCA6F1160100BF38462A4607
:20BD200014F010FD002844BF4FF0FF30BDE8F087013C7FF4ABAF1AE0BD61F9E73D62F7E7BE
:20BD4000FD61F5E7384611210AE03846132107E03846172104E03846122101E038461B2190
:20BD600015F0B7FC384629462AF0C4FBDAE73846414615F0AEFC0020BDE8F08770B586B039
:20BD80000D4604460026CDE9006607210522002316F0CBFA38B9CDE9006620460F210022C2
:20BDA000072316F0C2FA226840F61566CEF600662046314614F010FD05A90DF1130220461D
:20BDC0002AF064FB607B48B122692046002114F0B9FC22682046314614F0FEFC216A2046F5
:20BDE0002AF036FBD4E90701C1F3401141EA0002E2612046002114F0A5FC22684FF6107142
:20BE0000CEF22F11204614F0E7FCA2692046002114F098FCE06A20F42051002D18BF01F5E2
:20BE20000061E16220462AF055FBA07B60B1B4F846206169D4F8AC002AF004FB236804F175
:20BE4000AC0207CA2AF0ECFA236804F1D00207CA2AF0E6FA00280BD4642603AD2046294630
:20BE600015F08BFC9DF80C00800704D4013EF5D14FF0FF3000E0002006B070BD2DE9F04397
:20BE800093B015468846064608464FF4987110F0B5F93146707B11F80C2F42EA00208A78AE
:20BEA000C97842EA0121474640EA014047F8040F30687860707938720020129007F59671E1
:20BEC000CDE90B710E90A5F59870CDE9101020EAE07001EB50010D914008C0000F900BAD86
:20BEE000012602AC0DF104092846012122464B4615F07BFCF8850298B8850198388607F1BA
:20BF0000540128462EF0F8F828460121224615F06AFDB8860298788607F1600128462EF031
:20BF2000EBF803AC2846214622221FF065FCF88607F16C0128462EF0DFF8284600214A4681
:20BF400015F0B1FD38870198788707F1780128462EF0D2F82846214621221FF04DFC203050
:20BF6000B88707F1840128462EF0C6F82846012115F049FF2846214620221FF03DFCF88700
:20BF800007F1900128462EF0B7F82846012116F070F82846214620221FF02EFCA7F84000B0
:20BFA00007F19C0128462EF0A7F82846052115F02AFF2846214622221FF01EFCA7F84200DC
:20BFC00007F1A80128462EF097F82846052116F050F82846214622221FF00EFCA7F84400AE
:20BFE00007F1B40128462EF087F82846082105222EF02EF82846032109F02EFD07F1C00118
:20C0000028462EF079F82846042105222EF020F82846012109F020FD07F1CC0128462EF03C
:20C020006BF8284600211F2206231FF009FB07F1D80128462EF060F82846042115F0E3FE63
:20C0400040F69A71CEF60761284616F052F807F1E40128462EF050F82846012109F0FCFC83
:20C060002846214621221FF0C7FB2030A7F8460007F1F00128462EF03FF82846012115F061
:20C08000F8FF2846214620221FF0B6FB0730A7F848002846042115F0B6FE07F1FC01284605
:20C0A0002EF02AF8284631460022002315F09DFB0290711E012903D039B9A8F8520004E093
:20C0C000B8F85220801AA8F85400481C0E2801D0461CE7E70BAD47F6FE71CEF6A00101AAA1
:20C0E000284615F0E0FC0198A8F8560008F58C76284631462EF000F808F592712846324682
:20C1000026F019FC012600BF28463146002215F06AFC0290711E012904D041B9A8F84E0095
:20C1200005E000BFB8F84E20801AA8F85000481C0E2801D0461CE7E708F586710BA82DF054
:20C14000DBFF10AA07CAC8F80000A1EB420013B0BDE8F0832DE9F04F87B00E2A02D307462B
:20C16000980704D00026304607B0BDE8F08FCDE90513002004904FF0010B02921046B0F579
:20C18000006F28BF4FF4006000260E21002223F04DFA81463846132115F09BFA3846002123
:20C1A000059A14F0CFFAB7F85430B7F85210D7F818010E22009200EBD10001F00702069DCC
:20C1C00029460BF035FD3A6843F63463C1F20803D7E946011C68D7F820316468A04700280D
:20C1E000C1D1B0462C46CDF80C90B9F1010955D088F0010808EB480007EB800A3834DAF895
:20C200001801B7F85430B7F852100E22009200EBD10001F0070221460BF00AFD43F6346013
:20C22000C1F2080000688068804700289AD13B68B7F85600C10800F00700595C21FA00F071
:20C24000C0071AD1002600BF07F1880207CA2AF0E7F8002886D43B68B7F84000C10800F02E
:20C260000700595C0BFA00F00840622E02D801360028E9D000283FF475AF43F63460C1F244
:20C280000800D7F820610268DAE9460155681A463346A84700260028A7D064E743F6346070
:20C2A000C1F2080000688068804700287FF45AAF3B68B7F85600C10800F00700595C21FAD0
:20C2C00000F0C00714D0DDE90306C0EBC000069901EBC0010691059901EBC00106EB400624
:20C2E0000298801B0D28CDE904613FF648AF3AE7642407F1880207CA2AF092F800283FF591
:20C3000031AF3B68B7F84000C10800F00700595C21FA00F0C007D6D10026013CE9D122E797
:20C320002DE9F0471D46904689460746B0F850A0B0F84E40002600BF386804F12001C90821
:20C34000405C04F00701C840C00704BF0020BDE8F087484621462FF02FF908F8260008EB22
:20C360008601020ECA70020C8A70000A4870544401360E2EE0D145B1D5E902013830A8603F
:20C38000884202D32968284688470E20BDE8F0872DE9F8431E46904689460546132115F008
:20C3A00098F9284600214A4614F0CCF9089CAA8FE86F41F20101CEF2D041012C04BF41F2A7
:20C3C000B201CEF2D001022C04BF41F20401CEF290412AF037F8686EEA8E41F61561CEF657
:20C3E00000612AF02FF8012000FA04F7C1462B6805F17C0207CA2AF013F800286CD42B6886
:20C40000E88FC10800F00700595C21FA00F0C00722D005F1640207CA2AF002F800285BD4D4
:20C420002B68298F01F12000C00801F00702185CD040C00728D018462FF0BEF8012F3AD02D
:20C44000022F3AD0042F40D13070010A7170020CB41C1821032334E0642400BF05F18802B9
:20C4600007CA29F0DDFF002836D42B68B5F84000C10800F00700595C21FA00F0C007C8D164
:20C48000013CEBD128E000BF642400BF05F1700207CA29F0C5FF00281ED42B68698F01F1E8
:20C4A0002000C00801F00702185CD040C007C2D1013CEBD110E0314606E0082101230246E1
:20C4C00034462270C840F11808703E44B9F101097FF48DAF4FF00009284615F036F94FF0B9
:20C4E000FF31002808BFA8EB09010846BDE8F883012AB8BF70472DE9F04F43F28473C1F285
:20C50000080343F64817C1F20807D3F800E043F6E009C1F208093B68D9F800904FEA690877
:20C520000EEBD30505EB0804082A9246A8BF4FF0080A03F00707C7F10809CA45CB46B8BF0B
:20C54000D3466FB1CEB2BE4095F800C046EA0C062E70C6B206FA07F72678374302E000BFC8
:20C56000297007462770CA4507DDCFB227FA0BF76F70C7B227FA0BF76770A2EB0A02534425
:20C58000090A000A002ACBDC43F64810C1F208000360BDE8F04F70472DE9F04741F280075C
:20C5A000C1F208070446386A00F1640843F2BC69C1F2080943F68E1AC1F2080A20464946B7
:20C5C00015F0F9FF0646BAF81C50204629F0F6FF002818BFBDE8F087711960682AF006F8FB
:20C5E00000F01901092904BF0020BDE8F087C00644BF0320BDE8F087386AA8EB000000289B
:20C60000DCDC0220BDE8F087F8B5044632B143F2EC70C1F208000068E06041E00D4643F2AD
:20C62000DC61C1F20801204615F0C5FF06464FF0FF30A840C0430021CEF6800101EB40009B
:20C6400027F03AFC43F68E17C1F208070146388E3218206829F0ACFF43F2EC61C1F208010C
:20C66000204615F0A8FFB98D4618022D0AD36F1E43F2EC65C1F208052046294615F09BFFB1
:20C68000013FF9D143F2E461C1F20801204615F092FF266143F2EC70C1F20800E1680160E1
:20C6A000204616F06CF900B1F8BD43F63460C1F2080000688068BDE8F84000472DE9F843F6
:20C6C0001C461546894643F68E11C1F20801804691F8200018B38CB342F2E677C1F604274E
:20C6E00043F2EC66C1F208064046494629F08EFFC1B2C0F30722795CBA5C120442EA016159
:20C70000C0F30742000EBA5C385C41EA02210844716845F8040B8944013CE5D10EE06CB1DB
:20C7200043F2EC67C1F208074046494629F06EFF796845F8040B8944013CF5D1BDE8F883F7
:20C740002DE9F04FADF2546D0DF13700012126F001FA9DF8370029F06BFF0EA8082126F078
:20C76000F9F943F29440C1F208004FF480710022C16210AB03F5007903F5807680E84802BE
:20C78000C26003F5A06903F5806603F5407300F1140C8CE84A024262DDE90E700190042877
:20C7A00006D843F2C460C1F2080029F0EFFE10BB43F29444C1F2080443F2D461C1F20801C4
:20C7C000204615F0F8FE43F68E10C1F20800394690F8200018B1384627F06EFB014643F6F8
:20C7E0008E12C1F208022068128A29F0E1FE204629F0E4FE28B1064600240DF2446B0199CE
:20C8000079E0F80701D1019931E00020CDF840060DF5C860012126F09DF90198451E43F6EB
:20C820008E10C1F2080090F8200028B1DDF8400627F042FBCDF8400643F29461C1F20801BE
:20C84000204615F0B8FE43F68E11C1F20801498A42182068DDF8401629F0AAFE2046FFF726
:20C860009BFE10B10646012442E001372946022964D317F0020061D00D460020CDF840060A
:20C880000DF5C860022126F065F943F68E10C1F2080090F8210028B1BDF8400600BA000C02
:20C8A000CDF8400643F68E10C1F20800023D90F8200028B1DDF8400627F0FEFACDF84006E6
:20C8C00043F2B461C1F20801204615F074FE43F68E11C1F20801898A42182068DDF84016C1
:20C8E00029F066FE2046FFF757FE28B3064602240DF2446B294649B10DF5C865284689463A
:20C90000012126F027F9B9F10101F7D10DF24460834502D0584626F042F8F0B226F001F96E
:20C92000300405D038462DF059FC20462DF056FC0DF2546DBDE8F08F0237294604290FD38E
:20C94000112910D30E4609F0B9F8054638212EF079FE281A009026F00FF83146834606E06E
:20C960000DF2446B81E1102000900DF2446B0020099043F2846AC1F2080A42F2C858C1F291
:20C98000080843F2AC69C1F208090026CDF814B0029121F003050098854228BF05465846EF
:20C9A00029462DF037FC25F00300CDE9030500239AF80100C0EBC00008EBC000016900BFE5
:20C9C000F1B14269002AA5EB020222F00302A2EB030217D0382AF3D310463821BB461F467F
:20C9E000C24690462EF02EFE4246D0463B465F46DDF814B043F2846AC1F2080A121A01E0BD
:20CA00000398C21A002E40F02481CDE9073723F0030083440692900800210022CDE90B2077
:20CA20000E28074628BF0E270A9101F0010505EB450004EBC00A0998B8420BD143F29C701F
:20CA4000C1F2080043F68E180068CAF80C00C1F2080881E0504643F29C61C1F2080115F059
:20CA6000AAFD06464FF0FF30B840C1430020CEF690000C4640EA410027F01EFA43F68E181A
:20CA8000C1F208080146B8F818003218DAF8000029F08EFD5046494615F08DFDB8F816107A
:20CAA000084443F2A071C1F2080108600020002D08BF38460990022F09D3A7F1010800BF28
:20CAC0005046494615F077FDB8F10108F8D14FEA4408504643F2A461C1F2080115F06BFDBF
:20CAE00006460020CEF6900000F5801040EA080027F0E2F943F68E18C1F208080146B8F834
:20CB00001A003218DAF8000029F052FD504643F2BC61C1F2080115F04EFDB8F81C1055460C
:20CB2000084445F8100F0C980E2815D3DAF80C2043F29446C1F20806DAF80010B069073289
:20CB4000D40822460FF034FBDAF80810306A22460FF02EFB2868B06243F2A070C1F20800AD
:20CB6000DAF80060056898F822003C46B84698B15BF8040B27F0A0F9014606EBD50605F081
:20CB8000070530462A462EF029FDD9F804000544013CEDD110E000BF06EBD5065BF8041B59
:20CBA00005F0070530462A462EF018FDD9F804000544B8F10108EFD10B9810B115F0F5FD70
:20CBC00070BB43F29C71C1F20801DAF80C000860504615F0D4FE00BB0C980A990131C01B6A
:20CBE000524643F29444C1F208047FF417AF504615F0DBFD064600280898DDF814B043F243
:20CC0000846AC1F2080A42F2C858C1F20808DDE906231AD1171800261AE006460C9F03E047
:20CC200006460C9800F10E070898DDF814B043F29444C1F2080443F2846AC1F2080A42F2DD
:20CC4000C858C1F20808DDE906231044A0EB8707049D1344AB427FF4ABAE0299491B0329B9
:20CC60003FF696AE0EB1042445E688073ED50D460020CDF840060DF5C860022125F06AFF3E
:20CC800043F68E10C1F2080090F8210028B1BDF8400600BA000CCDF8400643F68E10C1F22A
:20CCA0000800023D90F8200028B1DDF8400627F003F9CDF8400643F2B461C1F20801204607
:20CCC00015F079FC43F68E11C1F20801898A42182068DDF8401629F06BFC2046FFF75CFCF2
:20CCE00010B10646022405E602372946002571B3CDF840560DF5C8600D46012125F02AFFED
:20CD000043F68E10C1F20800013D90F8200028B1DDF8400627F0D0F8CDF8400643F2946193
:20CD2000C1F20801204615F046FC43F68E11C1F20801498A42182068DDF8401629F038FCC9
:20CD40002046FFF729FC10B106460124D2E543F29446C1F2080643F2F461C1F208013046DD
:20CD600015F029FC304629F029FC06460024019804283FF6BFAD002E7FF4BCAD43F21C7034
:20CD8000C1F2080029F002FC0646B3E510B50446002000210122FFF7ABFB013CF8D110BDFB
:20CDA0002DE9F04141F2D004C1F2080480466078012810D1002603270120F143751C20FA6E
:20CDC00005F201FA07F328EA030393422CD0013F042D2E46F2D143F64810C1F20800006822
:20CDE00020B9002000210122FFF782FB2678E578032000210422FFF77BFB701B043818BF14
:20CE000013F0AAFDB5FA85F04009C00041460422FFF76EFBADB1012D02D0681E13F09CFDAF
:20CE20000120012101220AE0032000210422FFF75FFB28FA07F10120B040C0B22A46FFF7E5
:20CE400057FB012000210122BDE8F041FFF750BB70B582B041F2D005C1F2080504462E7934
:20CE60000220FFF79DFF01940523002E08BF04236878012816D15A1E012000FA02FC002183
:20CE8000C84300BF72B101312CFA01F600FA02F524EA0505013AB542F4D1501C24FA00F0DC
:20CEA000019000E0194601A813F078FF02B070BDA2B043F63040C1F2080043F2C055016837
:20CEC0000E910220002908BF01200C9012A800F12001079100F110010691011D08910830F8
:20CEE0000590C1F2080542F66470C1F208000C300D9042F60828C1F2080841F2800BC1F2A1
:20CF0000080B42F2107A00BF284611F05BFC4FF0010900240D9F00BF08EB0405286900282E
:20CF20006ED095F8400000286AD095F84100002866D13868DBF820105044884260DDEE6AC1
:20CF4000706840B3306930B3307BC0070CBFDBF8200028F05FFB7169091A00293CDCD6E9EB
:20CF600002E3DB07D6F820C044F6D352C1F26202AEFB023208BF4FEA921E71440029C8BFD4
:20CF800008447061DBF82000844506D196F82800C00715D020E000261FE03062E869016A0C
:20CFA00021B128698847012831D0A8B996F82800C00705D095F84110E86A012225F0A3FB5C
:20CFC000307BC0070CBFDBF8200028F023FBB169411A28461DF0ECFF0126284621F046F82C
:20CFE000002808BF8146002EE86918BF4FF00009016D29B128468847002808BF814600BFE3
:20D0000024374434B4F5AA7F7FF486AF0AE096F82800C007E0D195F84110E86A002225F044
:20D0200072FBD9E7B9F1000F18BF4FF0010901F073F88246002843F64000C1F2080018BF93
:20D040004FF0010A006838B143F23C70C1F20800006808B12EF0AEF843F28070C1F20800D4
:20D0600000270068002800F0F780D0F8FC04002800F0F28042F63000C1F20800007A00F0B3
:20D080000300022840F0E88043F65C10C1F208000078012802BF43F65C10C1F20800077032
:20D0A00042F63000C1F20800007A00F0030002280AD143F67210C1F208000078002848D0AD
:20D0C000012011F029FC2DE043F67210C1F20800077043F67110C1F20800077043F6651075
:20D0E000C1F208000078B8B142F68841C1F2080101F14104002500BF54F8311C2770C9695A
:20D1000031B1E8B2884743F66510C1F208000078483401358542EFD343F65C10C1F2080048
:20D120000121017043F28070C1F20800006890F80515002950D042F68844C1F2080494F8DA
:20D14000411041B326F012FF26F060FF84F841703BE043F6D810C1F208001421407800914C
:20D1600043F21C41C1F208014022002312F00FFD1F2800F08880002840F0018143F6D81094
:20D18000C1F2080014214078009100210022002312F0FDFCC6E7D0F8F004DBF82010081A67
:20D1A000B0F5FA6F58DB12F0F7FD4FF47A7011F0B3FB26F0DBFE26F029FF42F68840C1F27C
:20D1C000080080F8417012F0B8FF43F28070C1F20800006880F80575D0F8F824DBF8201044
:20D1E00012B9C0F8F8140A468B1A0A2B34DB90F804358BB3D0F8003573BBD0F8EC34CB1A70
:20D20000B3F57A7F28DB521AD0F8E8341A44C0F8E824C0F8F814D0F8E80400281CDC22F04E
:20D2200055FB42F68840C1F20800012280F8402043F28070C1F2080043F25C41C1F208017A
:20D240000068C96A80F80525DBF82020C0F8F024C0F8F414C0F8F87409EA0A0443F2C05583
:20D26000C1F20805284611F0EBFA0E98204342F2107A3FF449AE43F25460C1F208000C9960
:20D2800010F08BFD40E643F21C40C1F2080043F2F045C1F2080529468CC88CC1CCC8CCC139
:20D2A0002E4602880A8080788870284613F089FA45F25531C4F24231884240F06B8043F202
:20D2C000F051C1F208017068486043F66510C1F20800747B00780025A0422F4640F26F8163
:20D2E00006F1080013F06DFA864696F90C000028384648BF01200A90BE45774604EBC40083
:20D3000042F68841C1F2080101EBC00018BF01270B90D0F810C0F37B099701222E2B43DCC9
:20D32000112B58DDA3F11A04102C00F2C283082002260021DFE814F06B007200C903C903A6
:20D340007200C903C903C903C9034700C903BD00C903C9031100C903CD030B98DCF804207B
:20D36000007812A97446904743F2F040C1F20800A646C08ABDF84C10000400BA90E0FFF65F
:20D380009FAE43F67210C1F20800012101702EF0EDF8C7E643F67210C1F20800012101707E
:20D3A0002EF0E4F80027BDE6A72B2ADCA3F14300172863D8012101FA00F04CF28901C0F2F9
:20D3C000800108425AD043F2F040C1F20800C08A000405BA20E0294603B3032B17D0082BBE
:20D3E00040F073830078DCF8042012A97446904743F2F040C1F20800A646C07CBDF84C10F2
:20D400003AE0BC2B1CDCA82B3DD0BB2B37E043F2F040C1F20800C57C01220221292B05DD59
:20D420002A2B0AD0BE2B08D0A82B02E0082B04D0282B0E46284636D03BE00E46284632E036
:20D44000BD2B00F02D83BE2B40F03F830078DCF8042012A97446904743F2F042C1F2080289
:20D46000A646507D917DD27D090241EA00401044BDF84C1001F59871484312E02F2B4FF0A6
:20D480000001CBD021E30078DCF8042012A97446904706F1150013F04AF9A646BDF84C10E1
:20D4A0004843022601220B9991F83110002908BF084643F2F051C1F2080100270F738F6020
:20D4C0004AB15EEA060142D143F67110C1F20800002505706FE043F2F041C1F2080191F9E5
:20D4E0000C00002800F15A818868002800F0568143F6D814C1F2080442F2C8556078C0EB95
:20D50000C001C1F2080505EBC10101220A7242F63001C1F20801D1F85C110A6A0121904771
:20D520006078C0EBC00005EBC00000BF007A002800F06181012011F0EFF96078C0EBC00078
:20D5400042F2C851C1F2080101EBC000EEE7BE4508BF022E28D0BEF1000F08BF012E23D0A8
:20D56000DDE9091505EA0102002E334618BF012382F001010B4340F0758243F2F050C1F222
:20D580000800014680F808E043F67110C1F20800042202704FEA1E60C8724FEA1E4088724D
:20D5A0004FEA1E20487205E0012043F67111C1F208010870002543F2F046C1F20806307B49
:20D5C000717BF67B0F9501EBC10142F68842C1F2080202EBC10C00F080000B90122E2AD0DE
:20D5E000032E40F0818041F64470C1F6032012A90C46CCC8CCC400882080002D00F0CB8043
:20D600009CF801008DF84A00BCF80200ADF8540043F6D810C1F208000027007800972A4675
:20D62000012364460AF0A4FAA4460F990F97451A18BF012535E12426242D43F2F040C1F227
:20D64000080038BF2E46408A000400BA864228BF0646002E00F01A8143F2F042C1F20802F7
:20D6600048F20001507CC0F204211291202113919CF830108DF84810117CC90740F0DA80AC
:20D68000002840F007810996059E30461C21202264460EF0B4FD0A94646C256828460EF0B3
:20D6A00061FD0246082828BF08223046099E29460EF07EFD656828460EF054FD0246102874
:20D6C00028BF1022069829460EF072FDA56828460EF048FD0246042828BF0422079829466A
:20D6E0000EF066FD12A9C4E0604664462DF00CFF002800F0E680636BA44673B143F2F04033
:20D70000C1F2080000F10F0160460FAA64469847A4460546FF2840F0C48001242E2E00F321
:20D720009581A6F11A00102842F2C853C1F2080300F2E481DFE810F010021100CA00CA0008
:20D740002702CA00CA00CA00CA004502CA009802CA00CA00E801CA00CE0243F2F040C1F29E
:20D760000800DCF80820C07C00F003054AB19CF80000294664469047A44642F2C853C1F206
:20D780000803DFE815F0040023030400230301208CF841008FE00025002782E043F6D81436
:20D7A000C1F2080442F2C8552078C0EBC001C1F2080505EBC10101220A7242F63001C1F228
:20D7C0000801D1F85C110A6A012190472078C0EBC00005EBC00000BF007A60B1012011F07E
:20D7E0009BF82078C0EBC00042F2C851C1F2080101EBC000F0E743F2F040C1F2080043F6AE
:20D800006511C1F20801407B097888420BD200EBC00042F68841C1F2080101EBC00020219E
:20D8200041800521417043F2F051C1F2080101200873BEE080282DD121208DF84B0080208D
:20D840008DF8490008982021202264460EF0D7FC606C0A94C56828460EF084FC0246202849
:20D8600028BF202212ACA01A243029460EF0A0FC214643F6D810C1F20800324600780097E0
:20D880000123FDF75DFC0F9DDDF828C0A81B0F90002506E02420ACF8020005208CF80100AD
:20D8A0000125E8B201280CD0002842F2C853C1F2080340F0C3800024ACF802408CF801402C
:20D8C00004E0012442F2C853C1F2080343F2F050C1F2080043F6D81504730F980028C1F2E3
:20D8E000080546D043F2F051C1F208010A460872010ED172010C9172000A50722878C0EB90
:20D90000C00103EBC10101220A7242F63001C1F20801D1F85C110A6A0121904742F2C853E0
:20D92000C1F2080384F001000B99002918BF012108431ED16878C0EBC00103EBC101012295
:20D940000A7242F63001C1F20801D1F85C110A6A0121904742F2C853C1F208036878C0EBEB
:20D96000C00003EBC000007A18B1012010F0D4FFF0E743F67110C1F20800007880071CD4C7
:20D9800043F67110C1F208000078400736D443F67110C1F208000078C00705D043F2F0514A
:20D9A000C1F208010220087343F67110C1F2080007700AF01FF9FFF7B5BB6878C0EBC0015E
:20D9C00003EBC10101220A7242F63001C1F20801D1F85C110A6A0121904700BF42F2C85322
:20D9E000C1F208036878C0EBC00003EBC000007A0028C5D0012010F08FFFEFE72878C0EB69
:20DA0000C00103EBC10101220A7242F63001C1F20801D1F85C110A6A012190472878C0EBE3
:20DA2000C00042F2C851C1F2080101EBC000007A0028ACD0012010F06FFFEFE743F2F05178
:20DA4000C1F2080101200873FFF76CBB2F2E42F2C853C1F2080300F04B815A2E7CD0A82E81
:20DA600052D033E7B31EB3FA83F35B091A40012A7AD1864578D943F67111C1F20801042289
:20DA80000A7043F2F053C1F20803AEEB000119720A0EDA720A0C9A72090A597205468AE593
:20DAA000F07D317E41EA0020864598BF70460226FFE4122B09D143F2F040C1F208000226BD
:20DAC000C07C864528BF7046F3E4002500210022A4E40B98DCF80420007812A9744690477C
:20DAE00043F2F040C1F20800A646C08ABDF84C10000400BA484301220126D4E4002E3FF413
:20DB0000DAAE082E7FF4E2AE0B9800283FF4D3AE43F2F040C1F20800DCF81010C57B0491DC
:20DB20004A68CDF828C09CF80000099012A99047A82D00F05781282D00F06381082D40F09C
:20DB4000C28143F2F040C1F208000246407C917CD57C41EA002660E160460FA9644626F050
:20DB60002BF9A44605469CE6BEEB000318BF012382F00102134340F0158143F67110C1F225
:20DB8000080007701AE1DCF8041069B143F2F040C1F208006446C07C00F001008847A44659
:20DBA00042F2C853C1F208039CF8300005283FF482AE2420ACF8020005208CF8010001244B
:20DBC00084E69CF83100002800F0FB800F9D002D3FF45EAEDCF810109CF800004A6810A978
:20DBE0006446904710208DF84B008DF84A708DF849708DF848708DF859708DF858708DF8CA
:20DC0000517002208DF8500010988DF84F00BDF844108DF85B108DF857008DF85310020A07
:20DC20008DF84E20030C8DF84D30000E8DF84C00090A8DF85A108DF856208DF855308DF875
:20DC4000540043F6D810C1F208008DF8521000780097142D28BF142512A92A46012309F0F5
:20DC600087FFA446451BE3E49CF83100002800F0A8800F9D002D3FF40BAEDCF810109CF8BB
:20DC800000004A6810A9644690478DF84D708DF84C70BDF844008DF84F00000A8DF84E006B
:20DCA000109801388DF84B00010A8DF84A10010C000E8DF8480043F6D810C1F208008DF880
:20DCC000491000780097082D28BF082512A92A460123A7E40B9800287FF4EDAD9CF8380015
:20DCE000002800F01D812720ACF802000720D5E543F2F045C1F20805687C80077FF5C8AD22
:20DD0000DCF81040CDF828C09CF8006005F1110012F00DFD0146E88A000403BA002B00F096
:20DD20001881A768039330460D4610AAB84703460294E768109A09963046049529461C46CC
:20DD4000B8470027002840F0C78043F6D810C1F2080001214078009112AE314640220023FB
:20DD600011F015FF402840F02981109D2846314640222EF0C7FA002840F0208105F140004A
:20DD80001090013CE1D1DDE90243099DA768049E2846314610AAB8470346E768109A284644
:20DDA0003146CCE70023864528BF01231A4310D143F67111C1F20801012008707546FFF741
:20DDC000FABB3A20ACF80200022067E58CF8417071E5721E18BF0122114340F0848005205E
:20DDE000FFF7E3BB43F2F045C1F2080505F1110012F09DFC064605F1150012F098FC05468B
:20DE00000BE043F2F045C1F2080505F1110012F08EFC0646E88A000405BADDF828C00F9875
:20DE200000283FF435AD002D53D0BDF84C10B0FBF1F0A84238BF0546002D00F08C801298B9
:20DE4000864280F028815CF80C7FCDF808C02FB100950998012101223346B84700270396E2
:20DE60003E442C460498EB1B85680998314610AAA84700287ED00546BDF84C00002879D02B
:20DE800004983146C668109A09982B46B047002870D143F6D810C1F2080010990078BDF873
:20DEA0004C2040F6B833009305FB02F63246002309F05EFEB0425DD12F442546BC42039EBD
:20DEC000CED8002557E00F98DDF828C000283FF4DFAC00250F95E4E4DDF828C01120ACF8D3
:20DEE00002000320DAE4BEFA8EF14909294381F0010181F00102002E334618BF012313436B
:20DF00002BD143F2F050C1F20800014680F808E043F67112C1F2080202201070FFF73ABB28
:20DF2000DCF8106043F2F040C1F208001130644612F0FDFB0546099672680A942678304622
:20DF400012A99047BDF84C000F99814238D2002532E000253FE00F97A2E4B31E18BF012346
:20DF60001A433BD143F67110C1F2080003210170FFF720BB0125029806682EB1009409981B
:20DF8000039B01210022B047E01BBDF84C1048430F90F5B10A9C112060800320607043F6E9
:20DFA000D810C1F208000027007800970125002100220123FDF7C4F8A44672E401250AE0FB
:20DFC000B1FBF0F251191298814217D92120A44661E400250027DDF828C062E4721EB2FAF1
:20DFE00082F252091140012958D1864556D943F67112C1F208020221117042E58542A446BF
:20E0000049D26046049250F80C7F01903FB100923046002101222B46B847049AA446CDE95B
:20E0200002650027099CBA4256D9D31B25693046039E314610AAA847054643F6D810C1F2B0
:20E04000080010994078BDF84C20012300936A43099240F6B83311F09AFD099988423ED103
:20E06000E8190990B9196769109A029E30462B46B847DDE9093C00281F46049AD3D06046B5
:20E08000344610F8011F19B903210170ACF8021001251F462DE02120FFF7FDBBBEEB00028F
:20E0A00018BF012281F001010A433FF466AD00258645284628BF0120084343F2F046C1F291
:20E0C00008067FF47CAA43F67111C1F20801012008707546FFF773BA3446002509E0029C85
:20E0E000DDF828C00320ACF802008CF801000125049A0198066846B1009220460021002218
:20E10000039BB047049ADDF828C0D01BBDF84C1048430F90FFF740BB70B588B043F6C4009E
:20E12000C1F2080043F6C802C1F20802016842F63003C1F2080310681A7A02F003020125A9
:20E14000022A40F0B680002900F0B380411C00F0B08043F6CC01C1F2080141F28002C1F23A
:20E1600008020B68166AF31A8342C0F2A280126A121A0A6043F65811C1F2080109780129E1
:20E1800040F0978043F6D001C1F208010C68616E89B100284FF0000060660CD1236E43F225
:20E1A0009870C1F20800D4F868220168204621F017F90120E065E06DD8B120462DF094F80B
:20E1C000E16C43F2D426C1F20806A1B1226DA06D2C2300FB03600123007E27F017FE002871
:20E1E00021DB0025E564D4E91401401860651CD135E001255DE0D4E9060188423EBF20694D
:20E20000226A1044421A0BD0C4E913122369256A2B44984228BF401BE0610029D7D102E07B
:20E220000020C4E91300606DC0B1A06D2C2100FB0160007E12F0AFF90546D4E90401226A49
:20E24000636D5B1B19441044814228BF891A616120462DF00BF86565002500E00125D4E980
:20E260000A01C9430A1844BF606B0244202AA8BF2022F2B1A06D694610F017FE012818DBCE
:20E2800002466D462046294609F040FCD4E90A01C9430A1844BF606B0244202AA8BF20227C
:20E2A00032B1A06D294610F000FE02460128E9DA0025284608B070BD00200A2142F66472FC
:20E2C000C1F20802535A002B18BF01302431BE29F8D1704730B5A3B013AD284640210DF021
:20E2E0008DFF02AC204644210DF088FF4FF0FF3001F002FB43F6F001C1F20801086840B1F2
:20E3000000220A6043F63461C1F2080108600069804701A8042124F01DFC9DF80510402941
:20E3200003D89DF8060040280BD908461EF08EFF9DF806001EF03EFF4FF0FF302BF04EFF76
:20E3400050E011B113A82BF031FF9DF8040003281AD8DFE800F0021C333740F20800C2F2E2
:20E3600000009DF8061043F63C12C1F20802C4601268C0E90512BFF35F8F0221016000BF6D
:20E3800001680029FCD121E09DF80510CDE740F20800C2F200009DF8051043F63C12C1F2ED
:20E3A0000802C5601268C0E90512BFF35F8F0121016000BF01680029FCD107E002A8FAF731
:20E3C0003BFB03E09DF84C000EF03AF99DF80600002122182154D17091705170011D204620
:20E3E00024F01BFB23B030BD2DE9F04186B00DF10B00012124F0AEFB9DF80B000B2800F209
:20E400003381DFE810F00C000E0031013101310131013101310131013F008B00A00001207E
:20E42000D3E043F67810C1F2080044F2D801C1F208010078073121F00704002818BF2046B1
:20E440002BF0BCFE43F67410C1F208000021C2F201010078002818BF081B2BF0AFFE43F201
:20E46000D054C1F20804204610F0ACF9012014F0C1F82BF0A3FE002014F0BCF8204610F0D6
:20E48000DFF9F1E005A8042124F064FB059FBFB343F25C70C1F208000468002C00F098801C
:20E4A000D4F8A00028B90020A4F8A4000120C4F8A00004F1800800BF94E843002269F34376
:20E4C0005D1848BF15441044801BA842B8BF05468DB1AF4238BF3D46304629462BF066FEBF
:20E4E0007019216822690A44904208BF0846BFF34F8FA0607F1B40460FF01AFD002FDBD1A9
:20E5000043F25C70C1F208000068002860D0D0F8A000B0FA80F0400940005AE043F25C7039
:20E52000C1F20800046854B10120C4F89C0004F180000FF0FDFC04F18C0026F0BDFF002056
:20E5400024F0EFFA90E043F25C75C1F208052868D0BB4FF69101C1F6032141F6A8002BF0C1
:20E56000F3FD002800F0838004462860A8210DF045FE04F1800026F081FF28688C3026F048
:20E580007DFF4FF4807041F2A8612144606241F2A8722244C4E90011A160C4E90402C4E997
:20E5A00006224FF4B05004F1A801CDE9001004F1280040F2B341C1F6042149F20143C1F637
:20E5C00001231B220FF0D5FF00202BF007FE4BE00220039003A8022124F081FA43F25C7485
:20E5E000C1F2080400200399022903D1216809B1B1F8A400039003A8022124F070FA2068AA
:20E6000030B1D0E90612511A44BF406A014400E00021049104A8042124F061FA049F0FB3B0
:20E620002668D6E90504716A0844051BBD4228BF3D462046294624F052FA2C447069716A7B
:20E6400001448C4208BF04467D1B04D02046294624F045FA2C44BFF34F8FB46106F1800076
:20E660000FF066FC2BF0C0FD06B0BDE8F0814FF0FF30AAE72DE9F04FA1B06846042124F009
:20E6800069FA0025009800286ED043F68411C1F208010DF104080F784FF0010942F21C0A36
:20E6A000C1F6000A43F6254BC1F2080B00260024C10751D00E2C08D00D2C0CD143F6000096
:20E6C000C1F208000121006809E043F60810C1F20800006802E020460DF03AFF0021421C9B
:20E6E00011D01C2C34D809FA04F212EA0A0F2FD0F1B99BF80010012908D143F62011C1F26B
:20E70000080109680EE04FF0FF3021E046F28001C1F600218BF8009043F62012C1F2080256
:20E720000968116000294FEA410158BFA0EB610077B9002805DB4FF47A71002220F076FF43
:20E7400006E040424FF47A71002220F06FFF404248F82600013600980134B5EB500F4FEA5F
:20E7600050000090A4D100E00026B10001A824F054F921B0BDE8F08F10B5A2B001A80421A9
:20E7800024F0E8F900200199E1B143F2805CC1F2080C0DF1080E0022002300BFCC0708D09D
:20E7A000032B94BF5CF823404FF0FF344EF8224001320133B0EB510F4FEA5101EED100203B
:20E7C00001901046810002A824F027F922B010BD2DE9F04184B00DF10F00012124F0BAF9E3
:20E7E00002A8042124F0B6F901A8042124F0B2F900284AD4DDE90140204346D007F05EF9E6
:20E80000844202D907F05AF904464FF62931C1F6032120462BF098FCD0B307462146AA2231
:20E820000DF0EDFC43F28468C1F20808019D00BFA542264638BF2E469DF80F0064280FD0E4
:20E84000652825D198F8000011F0A5FE0028F9D102983860384631462BF0B6FC06E000BF76
:20E86000384631462BF0A2FC00280BD4AD1BDFD19DF80F00652808BF2BF0B6FC02980138D3
:20E880000290D3D1384624F08AF804B0BDE8F08112F06AFF2DE9F04F87B00DF11A00022132
:20E8A00024F058F905A8022124F054F904A8022124F050F903A8022124F04CF902A80221A2
:20E8C00024F048F9BDF81A0000EB400009304CF22951C1F603212BF037FC0446BDF81A6056
:20E8E00031462BF063FC019404EB060ABDF81A1050462BF05BFC059C039FBDF808B0BDF847
:20E900001A90BDF810504FF0800080F3118800BF00BF2BF0ADFA062025F0DDF846F2942031
:20E92000C4F20F000AEB06080221016045444FEAC90900BF200412D043F63460C1F20800AA
:20E94000019900684246466850464B46B0472878697840EA01203840013C5845EAD141F255
:20E960008000C1F20800407818B94FF0000080F31188BDF81A10404624F04FF8019824F01B
:20E980000EF807B0BDE8F08FF0B585B00024CDE903444CF60027C3F69A37CDE901476FF04B
:20E9A0000706002500F018F800280DD4B842BCBF02900746A042C4BF039004460544013606
:20E9C000F0D3E808049001E00120019001A8102124F023F805B0F0BDDFF800F0413C081096
:20E9E0002DE9F043C3B042A8042124F0B3F841A8042124F0AFF843F2F071C1F20801419899
:20EA00000F68791C02292ED3429C40EA040111F0030128D101AD00BFFF28814688BF4FF4CE
:20EA20008079A0EB09004190A8464E46204625F067FA80EA070108F8041B0A0E08F8012C44
:20EA40000A0C08F8022C090A08F8031C0434043E80F0A537EAD12846494623F0DEFF4198F9
:20EA60000028D9D101E01EF0A5FB43B0BDE8F0832DE9F041C2B0884604460125012988BFC2
:20EA80000D4600260DF1070738463146012223F011FEA05D9DF807100140814237D10136CB
:20EAA000B542F1D104F1200025F02AFA78B3204625F026FA58B345F60066C1F60026316867
:20EAC0004A1C18BF884222D14FF0FF300CB3B8F5007F1ED102AD284621464FF480720DF03E
:20EAE00067FB304629464FF4807225F06FFF04F5807128464FF480720DF05AFB06F580704D
:20EB000029464FF4807225F061FF002001E04FF0FF3042B0BDE8F08170B542F66471C1F280
:20EB2000080101F11C05002435F8121C814204D024350134052CF7D170BD002625F8126C2E
:20EB400055F8040C18B123F02AFF45F8046C286818B123F024FF00202860204624F0A2FE55
:20EB6000FFF7AAFB002818BF70BD0DF05CFE43F68B10C1F208000024047043F68D10C1F2C7
:20EB8000080043F24C75C1F208050470286810B123F005FF2C6043F64800C1F208000168AA
:20EBA00021F01001016070BD30B583B043F26075C1F20805012128680068826801A890473F
:20EBC0009DF8044000208DF80400286801210068C26801A89047EF2C10DC601E052800F24B
:20EBE0007A80DFE800F003030330030300208DF8040028680068C26801A86AE0FC2C1CDD46
:20EC0000FD2C34D0FE2C43D0FF2C64D102208DF80400286801210068C26801A8904728682B
:20EC20000068006A80470190ADF80A00286802210068C2680DF10A004CE0F02C36D0F12C43
:20EC400049D1082014E0286842F2CE54C1F60424017B012904BF42F2CA54C1F60424217886
:20EC6000D9B30121625C0131002AFBD136E004208DF80400286801210068C26801A8904779
:20EC800000200190286804210068C26801A821E001208DF80400286801210068C26801A83B
:20ECA000904728680068406A80470AE001208DF80A00286801210068C2680DF10A00904757
:20ECC000072001908DF80A0028680068C2680DF10A000121904703B030BD0121019100680E
:20ECE0000121C26801A89047286800680199C2682046EFE72DE9F04F87B043F26076C1F206
:20ED00000806012130680068826806A890473068022100689DF81890826806A890473068ED
:20ED200001210068BDF81870826806A890479DF818A0CAF381000490484614F071FA054636
:20ED4000002814BF6C6D00240AF001080197A7F1010B30680AF002064068029000270397E7
:20ED6000B94600BFE6B943F26070C1F20800042100680068826806A8904774B3069AB8F1A2
:20ED8000000F14BF636923692846049998470746CB4509F1010A25D0002FD146E2D521E0FA
:20EDA00054B1B8F1000F14BFE368A3682846049905AA9847814601E04FF0FF39DDE90217D6
:20EDC000059841F8270001980137013801903FD0B9F1000FBA46C2D50EE0039800F1010AB7
:20EDE0004FF0FF37236805AA2846032198478146002FB8BFB946039F062043F26075C1F202
:20EE000008058DF81800286801210068C26806A89047ADF818A0286802210068C26806A82F
:20EE200090470120B9F1000F48BF04208DF81800286801210068C26806A890472FB1286820
:20EE40000068B900C2680298904707B0BDE8F08FBA46D1E72DE9F04F8DB043F26077C1F212
:20EE6000080701213868006882680DF1230090479DF8235014208DF8230038680121006869
:20EE8000C2680DF12300904700208DF82300386801210068C2680DF123009047002D3CD003
:20EEA0000DF1100B0DF1230938680121006882680DF1330090479DF8336016F03F0A08BFB5
:20EEC0004FF0400A0AF10700C408700604D4584621460DF093F904E058462146FF220DF0F8
:20EEE0008EF938682146006882684846904743F63460C1F20800594600686A46D0F8048042
:20EF000048465346C047300605D5386821460068C26868469047013DC6D10DB0BDE8F08FDF
:20EF20002DE9F04F85B04FF66931C1F60321DC202BF00AF943F25479C1F208090446C9F8A2
:20EF40000000DC210DF05AF945F60060C1F600200D210068049104F10C010022302300BF91
:20EF60008B540132049EB242FADB31190022CA72172504AC0A21224620F058FBD9F80010A9
:20EF80009DF8102030324A55013D0B2DF2D143F6E852C1F2080201F10C00D06010F01CFCFC
:20EFA00043F2E050C1F208000F21FF220DF027F942F63007C1F208074AF2C070C1F601204E
:20EFC000C7F8640143F66E10C1F20800002404704FF0010887F8068040F2EF20B8800094A9
:20EFE000012003210122002326F0D4FE0546D9F800004021009100F119030020032101221C
:20F0000026F0C8FE43F67616C1F208060290307843F66A1AC1F2080AB0B986F8008043F236
:20F02000A800C1F2080088210DF0E8F843F27870C1F20800314604608AF8004043F20C60D1
:20F04000C1F20800FCF756F9787B052809D8411C797307EB800045F2FD71C1F60321C0F8BF
:20F06000441197F8018008F10100787007EB48140195E8B20121224601FA00F022F8340FF9
:20F0800045F69901C1F603219160002696800321D1709AF800E00EEB0E1A43F2A801C1F20A
:20F0A000080101EB8A0B5B46D7F83CC143F83CCF4FF22F25C1F601255D60C7F83C3102991D
:20F0C0000B0610D0CBB2C3EBC3054FF0010C0CFA03F3184342F2C853C1F2080303EBC503E6
:20F0E00083F819C01080CBF81860FA78387B531E2CBF1A460B23FB708BF81320072809D8B1
:20F1000007EB80024FF6EF23C1F603235361421C3A73461D43F2A802C1F20802019802F8F6
:20F120002A0084F83B6041F2663043F6E85AC1F2080AC1F20800CAF800004FF24730C1F699
:20F140000120606443F66A12C1F208020EF1010010708BF812800025CBE90D554FF6833090
:20F16000C1F60320CBF804002620ABF802008BF80110D9F800000DF10F04C0F800E000BF36
:20F1800005F150012046012223F06BFA9DF80F0028B1FF2803D00135202DF1D12FE04FF617
:20F1A000DF70C7F6FF70054229D0DAF80840207838B1601C002600BF815D01360029FBD18E
:20F1C00000E000267019023042F24271C1F604212AF0BAFF98B18146214632460CF0E8FF06
:20F1E00009EB060420465F2100F8011B50212A4623F037FA601900214170CAF80890C7F88E
:20F200007CA110F09AFF05B0BDE8F08F2DE9F04143F25475C1F208050C462F688046B8688B
:20F22000402802D118F095F92F68B868C0F14006A64288BF264638449930414632460CF074
:20F24000B7FFB8683044B860A41BB04408BFBDE8F081E5E72DE9F04F89B014460D46049021
:20F2600096B206F02BFC864238BF3046B0F5805F88BF00F47F404CF29C51C1F603210390DD
:20F280002AF062FF089000B34FF6FF7024EA000815F003002C461CD02546C0F10404A6426C
:20F2A00038BF3446089F384621462AF07FFF04982246C1694346D1F808C000972946E04744
:20F2C000311BA0426ED12C4404E04FF0FF35314671E03146002968D0CDF81C80029643F22C
:20F2E0008468C1F2080842F2C859C1F20809DDF810A000BF039D0691A94238BF0D460898F6
:20F3000029462AF087FF4FF0000B05942146002498F80120C2EBC20209EBC2073A6900BF2F
:20F3200062B17B69002BA5EB0303A3EB0B0607D0402EF5D326F03F0602E000BFA5EB0B06CC
:20F3400014B14FF0FF341AE0DAF81C20089B97685B44009350463246079B0C46B847214632
:20F36000841B18BF4FF0FF34891922BFDAF83C000130CAF83C0042F2C859C1F20809B344D5
:20F38000AB45C5D1002C0699A1EB050118BF4FF0FF35002D0BD454B9059C2C440029A9D173
:20F3A000029D0CE04FF0FF3505E0354609E0002D58BF4FF0FF3511B108461DF047FF08984C
:20F3C00010B1089823F0EBFA284609B0BDE8F04F2AF004BF2DE9F04F8FB08B4607464FF6F5
:20F3E000FF7022EA0000CDE9032096B2112E0ED306F1040A06F062FB0446824538BF544657
:20F40000204623F0B9FA0546A4F1040800E00025002D08BF4FF0100840F2FF10B8F5806FA7
:20F42000C14688BF29EA0009002D08BF0DF11405029600BF4FF400700D9047F2CD30C1F6C3
:20F4400003200A9000200E90CDE90B50F869464544680AA8CDE90050B24688BFCA46384603
:20F4600059465246049BA0470446012814DB1BEB040B22BFF86B0130F8630E98211A361B56
:20F4800014D011B128442AF09FFE2AF0ADFE5445D0D00298841B02E00E98361A02D030464C
:20F4A0001DF088FE20462AF099FE0EE0039B2B5528190022C27082701A0A42700E98284427
:20F4C00004312AF081FE2AF08FFE05A8854202D0284623F064FA0FB0BDE8F08F2DE9F04366
:20F4E000D3B0054600260DF1070843AF02AC00BF4046012123F02EFB9DF80700FF2804D031
:20F50000B8550136402EF3D14026E9692869D1F80C90394622463346C8479DF80710FF2984
:20F5200005D0B100204623F078FA0026E0E744F82600042000EB8601204623F06EFA53B091
:20F54000BDE8F0832DE9F04385B00646002404941425CDE902450DF10700012123F0FAFAA9
:20F560009DF8070090B30DF106050DF108090DF1070703AC0DF110082846012123F0EAFA3C
:20F580009DF80600032807D0022809D001280DD19DF80710404606E09DF80710484602E090
:20F5A0009DF8071020462AF001FE03E09DF807001DF04CFE3846012123F0CCFA9DF8070035
:20F5C0000028D9D1049CDDE9022500E00022F16930694F6A29462346B8472AF0FFFD05B07C
:20F5E000BDE8F0832DE9F04786B0044600250120CDE90405CDE902050DF10700012123F02A
:20F60000A9FA9DF8070000283CD00DF106050DF107060DF114080DF110090DF1080A03AF70
:20F620002846012123F096FA9DF806000438072812D8DFE800F004090D11111111179DF8E6
:20F640000710404611E000BF9DF8071048460CE09DF80710504608E09DF807001DF0F6FD71
:20F6600005E000BF9DF8071038462AF09FFD3046012123F06FFA9DF807000028D0D1059DEB
:20F68000039800E00020E063E16920698A6A2946904741F28000C1F20800017801310170F5
:20F6A00001200FF039F9E16920694A690299904704980FF031F9E1692069C969884704461D
:20F6C0000EF00BFF20462AF089FD06B0BDE8F0872DE9F04F93B001AC204644210CF08EFDB3
:20F6E0000DF10300012123F035FA0DF10200012123F030FA9DF8020000286CD004F104084A
:20F7000004F1050B04F108090DF101070DF102044CF2AF5AC1F6032A3846012123F01AFAE2
:20F720009DF801000738032818D8DFE800F0021D21279DF8021000201290B9B312A823F019
:20F7400009FA9DF848109DF849309DF84A209DF84B00000612041B022BE000BF9DF8020032
:20F760001DF074FD2AE000BF9DF80210404602E09DF8021058462AF019FD1FE09DF80250D8
:20F78000082D28BF0825484629462AF00FFD9DF80200461B12D0304651462AF0D5FC069095
:20F7A000A8B131462AF002FD079607E0002200230021194311430843019000BF20460121A3
:20F7C00023F0C8F99DF802000028A5D103E09DF80200401BC4E79DF8030001A924F0A9F8A9
:20F7E0009DF803000024052800EB001042F60821C1F2080138BF01EB8004206928B960696E
:20F8000018B123F0CCF80020606113B0BDE8F08F2DE9F04184B0074603A8022123F09AF944
:20F8200004209DF80C109DF80D2000EB82004843CE1D00EBD60023F09FF804469DF80C00F8
:20F840008100002C3DD09DF80D2004EB8005504305EB8008F60820462AF0A8FC9DF80C00EA
:20F860009DF80D104843810028462AF09FFC404631460CF0C3FCF96938698F6D9DF80C103F
:20F880009DF80D20CDE9001221462A464346B847002824D42EB1404610F8011BF9B9013EE5
:20F8A000FAD101202AF08AFC9DF80C001F304509404629460CF0A2FC4046294623F00FF9DF
:20F8C00011E008461DF0C2FC9DF80C009DF80D10484380001DF0BAFC6FF0010001E04FF07D
:20F8E000FF302AF06BFC2AF07FFC14B1204623F056F804B0BDE8F08100B50022411C24BF56
:20F900000521104600EB001C42F60823C1F2080303EB8C03403300BF53F830ECBEF1000F6F
:20F9200018BF1A70443301308842A8BF00BDF3E72DE9F04F83B00091074601201325C0F285
:20F94000800500BF3978A1F10902172A05D800FA02F22A4201D00137F4E7019700200029D8
:20F9600000F08D804AF67048C1F60128012600BFA1F161001A2805D35F2903D0A1F1410091
:20F9800019287AD8012400BF385DA0F130010A2908D3A0F161011A2904D35F2802D04138AC
:20F9A0001A2801D20134EFE74FF0000A4FF00109C34600BFDBF80400A04206D1DBF800006A
:20F9C000394622462CF09EFC78B1BAF1070F4FF0000938BF4FF001090AF1010A0BF10C0BFF
:20F9E000BAF1080FE6D108F1600B3819019000BF01780939172905D806FA01F1294201D083
:20FA00000130F5E7019010F8011B3D2935D1019001A802A91FF04AFE5FEAC97005D0DBF852
:20FA2000082012B10298009990470198471C00BF0178A1F10902172A06D806FA02F22A4281
:20FA400002D001370130F3E70190A1B1A1F10900172807D806FA00F0284203D017F8011B9D
:20FA6000F4E700BF17F8010C3B2806D10197397800297FF47DAF002001E04FF0FF3003B063
:20FA8000BDE8F08F2DE9F04F8DB004460CA8042123F060F806F012F8B0F500704FEA900143
:20FAA00044F62512C2F29242A1FB021748BF01270C98874288BF074657B143F62940C1F20B
:20FAC0000800007858B100200290B946019016E04FF0010904A8019006A802900FE0C7EBFE
:20FAE000C70080004CF2DF51C1F603212AF02CFB07EB8702029000EB82000190B946D4F85F
:20FB00001CB0BBF1000F75D00299B1FA81F04FEA5018002973D0DBF86450002D6FD00097CB
:20FB2000E96A584688470C9843F28467C1F2080741F28008C1F208084C4600BFA04238BFD7
:20FB4000044604EB8400810002982AF02FFB00BF387810F020FD0028FAD1CCB34FF0000A42
:20FB6000DDE90196039400BF347CB07CE0B1D8F8207000BF707C00280CBFAB68EB68584663
:20FB800021460BAA9847002817D4D6E901120B9B1940914211D0D8F82000F168C01B8842E4
:20FBA000E8DB4FF0FF3008E0707C002832680CBF2B696B695846214698470B99C9E9000110
:20FBC0000AF1010A09F108091436039CA245CBD1E10001982AF0F8FA0C98001B0C9043F292
:20FBE0008467C1F20807A9D12AF0FEFA4FF00008009F17E00298B0FA80F04FEA50180C98F6
:20FC000000EB800080001DF021FB00200590C043049004AC2046082122F0FFFE0C98013859
:20FC20000C90F7D12FB1B8F1000F02D1029822F0B6FE0DB0BDE8F08F2DE9F04F85B00446E0
:20FC40004069002840F0AD8004F14000E06304A8009000274FF00109204600210122012384
:20FC600018F023FB04986FF35F500490E16B04F13800CF708F704F700F70049A12F007067B
:20FC8000CDE9020660D00DF10C0A4FF0100B8846002500BF042E03D002F00603022B3DD11B
:20FCA00081F80090A06B40000090204600210022022318F056FBCDF800A02046002101222A
:20FCC000002318F0F2FA039901F00700CA08C1F34E3101314FF0FF33013349000029FBDC54
:20FCE00008EB8501C3F11E034B706FF39F22531C4FF0FF3201325B00002BFBDCC2F11E0296
:20FD00008A700BFA00F04FF0FF32034601325B00002BFBDCC2F11E02CA70049AD108049192
:20FD2000D4F83C806B1C012D08EB830108F82370CF708F704F70049A02F00706039604D86D
:20FD4000002E1D46A6D100E00023029D4FF0FF312B6000BF013140000028FBDCC1F11E00FF
:20FD600084F83500082084F8340048F27340C1F6022047F64D01C1F6032147F62902C1F6AF
:20FD8000032248F2CF73C1F60223264604F1800846F8308FC4E90042C4E90231C4E904067A
:20FDA000A56105B0BDE8F08F2DE9F04F83B09A4616468B460746D321D32001908DF80B106A
:20FDC0003846202127F008FD4FF0D309D32000BF9BF800403568092C14D8DFE804F0050723
:20FDE000131313131313090B7D6504E0BD6502E0FD6500E03D6604360BF1010BBAF1010AD6
:20FE0000E6D1BEE0A4F152011F2947D8B9F1D30F15D038464FF2D301CEF2213113F0C6FF60
:20FE200038464FF26F01CFF27F5113F0BFFFD321D32001908DF80B1035689BF80040D6F8EB
:20FE40000490386A294618F0E4FA384640F61568CEF61068414613F0A9FF386A494618F03F
:20FE6000D8FA08F58051384613F0A0FF04F10E00C0F3430100F02000084440F61031CEF631
:20FE800041410143384613F091FFAAF1010A08360BF1020B4FF0D309D320AFE7492CAAD803
:20FEA00042F24A61C1F6042101EB44010A2C11F8014B38BF0DF10B0191F80080804516D016
:20FEC0004FF20000CEF26F1000F1D97048EA0001384613F06BFF38464FF26F01CFF27F518A
:20FEE00013F064FF8DF80B80CDF80480C146386A294618F08EFA3F2C06D840F61560CEF6E3
:20FF0000106040EA043137E0FF2C0CD1384640F61561CEF6106113F049FF38464FF2000189
:20FF2000CEF26F1129E004F0E000802813D1384640F61561CEF6106113F038FF04F01F006C
:20FF4000C10341EAC0103FFA80F040F61021CEF60061014310E004F0F000C0280FD138464F
:20FF600040F61561CEF6106113F020FF40F61021CEF6E06164F31341384613F017FF40464A
:20FF800039E70198D3280DD038464FF2D301CEF2213113F00BFF38464FF26F01CFF27F515E
:20FFA00013F004FF002003B0BDE8F08F2DE9F04F83B09A4691460F4606460C990F2000EAA6
:20FFC000216001F00F0401286ED83046FFF734FE09FA04F23046394616F04EFC304620219A
:20FFE00027F0FAFB002800F1A180306A394618F010FA002800F19A8040F61567CEF6106770
:020000041A01DF
:200000003046394613F0D2FE002800F18F80B9F1000F00F07F80012000FA04FB4FF00008E7
:200020004AF6D845C1F6012507F58050029000270AEB0800022C08BF10F003010ED01AF81B
:200040000810BCB1427841EA0221012C0CD1306A18F0DFF9002814D568E000BF5AF808100D
:20006000306A18F0D6F910E08278C07841EA024141EA0061306A18F0CCF9002856D4012C0D
:2000800005D83046029913F091FE00284ED455F82410304613F08AFE00283DDBD844013780
:2000A000B945C5D14F4639E0D6F820800328D8F854500FD0022815D196F8A200B0B3726F8E
:2000C0004FF0000B3046002313F026FE6E6BCDE9004B19E0B26F3046002313F01DFE6E6B92
:2000E00001200FE0082821D30816182202EA513200F00700104402063046002313F00CFE0C
:200100006E6B0320CDE90040404639464A465346B0470EE0002701E0033007D14FF24F0136
:20012000CFF27F51304613F041FE01E04FF0FF37384603B0BDE8F08F2DE9F04784B0814683
:200140004EF60060C0F6156040F20043CDF213530B43D9F820A0D9F8EC70DAF85450002F85
:2001600008BF40EA017314466F69504601211A46B8476B68504602210022984741F280068B
:20018000C1F2080603AF306A00F11E086B68504602213A4698470398810009D4400604D439
:2001A000306AA8EB00000128F0DA4FF0FF3717E06B68002750460021002298476B6801AA83
:2001C0005046032198476B6802AA50460221984702982060D9F8EC00002818BF0198606040
:2001E000384604B0BDE8F0872DE9F04182B041F28005C1F2080504462F6A006A0221466D9D
:200200000022736898470DF1040800BF206A73680221424698470198C10106D4286AC01BA8
:200220001D28F3DD4FF0FF3017E04021C0F200110840884210D1206F00F19001204627F09F
:20024000E5FC206A7369002104229847204619F0E4FD6FF0010000E0002002B0BDE8F081B9
:200260002DE9F04182B041F28005C1F2080504462F6A006A0221466D0022736898470DF190
:20028000040800BF206A73680221424698479DF80700400606D5286AC01B1E28F2DB4FF028
:2002A000FF3000E0002002B0BDE8F0812DE9F8430546076A006FD5F88C107C6DB5F8942018
:2002C00000F12403384619F026FEE3686A46384603219847009840F0040200926369384635
:2002E000032198472846012114F096FB00281AD4286F00F18001284627F088FC41F28009F2
:20030000C1F20809D9F82080286A27F09FFC01280CD00646D9F82000A0EB0800642802DC25
:20032000002EF1DA06E04FF0FF3603E0284627F09FFC0646B5F89420286A2B6FD5F88C1025
:20034000243319F0E8FDE3686A46384603219847009841070BD520F004020092636938462A
:2003600003219847E3686A46384603219847002E4FF0FF30A8BF0120BDE8F8832DE9F04F65
:2003800085B004464069D0BB04F14000E06304F1380BD4F8EC10CDF804B099B30021C1701B
:2003A0008170417001702020019D4FF0FF312A60013140000028FBDC082084F8340047F6CD
:2003C0006170C1F6032047F65D72C1F6032247F62D73C1F6032347F66577C1F60327C1F124
:2003E0001E0184F83510A34604F19C014BF8301FC4E90043C4E90272C4E9040BA56105B088
:20040000BDE8F08F204619F008FD4EF6306AC0F6107A0AF5001102AA204627F071FD029FDE
:20042000002517F0070151D00AF1100B4FF01008002600BF0429D4F83C9003D007F006017F
:20044000022938D1720020465946002327F0C0FCCDE902552046514602AA27F051FD0120BF
:2004600009F82600029901F00700C1F3C902C1F34E3101314FF0FF33013349000029FBDCF0
:2004800009EB8601C3F11E034B70531C4FF0FF3201325B00002BFBDCC2F11E028A7008FA13
:2004A00000F04FF0FF32034601325B00002BFBDCC2F11E02CA70721C012E3FF675AFC7F326
:2004C000C201FF0800291646B4D16DE700226BE72DE9F04F93B01E46154608910746006AD9
:2004E000396F406D01908031384627F08FFB3846002119F078FB012EC0F2248207F1C400E8
:20050000049007F1BC0907F1CC0002904EF65144C0F610344FF0000B0795CDE9059600BF6B
:20052000089805EB8B0310F80BA0AAF15A084FFA88F0002824D44FEA980AD7F89000D7F803
:20054000EC100993C1B3504500F03281B94610AF0026C9F6666646EA4A1148463A4627F038
:20056000CFFC0546DDE91023059C204623F0B9FC002D6DD00020C4E90000C4E9020075E062
:200580000AF12600C0B2072836D81AF0010440F02C81AAF1DA004008D7F8EC101D4600298B
:2005A00000F010814AF60C51C1F6012151F8200040F4001110E100BF504500F0F9803E6A40
:2005C000A14608F02004756D6AF3430449EA04426B693046012198473846FFF705FE00282F
:2005E00000F0888005990020C1E90000C1E90200DDE906654C46D9E0BAF1E20F07D1D7F830
:20060000EC00002800F0018100201860F7E00AF0FE00442834D11AF0010415D1D7F8EC00CC
:20062000002844F22001CDF23C5104BF4FF2EE31C8F2300138460EAA1D4627F061FC2B4663
:20064000DDE90E01C7E93301029850F82400D0E04FEA4A1006F59001014348463A4627F0A3
:200660004FFCDDE91023049823F03BFCC9F890A0DDE906654EF65144C0F610344F4697E04F
:200680000AF0F800482840F0D0805FEACA7040F0D9804FF0AA30CDE91000D7F8EC000028AA
:2006A00000F04881B86D97F8F01000F00102AAF148004008884280F00381984652EA0001D6
:2006C00000F02F8142F2DE61C1F6042140F20072085CC10241EA8011C0F20702114000F0A8
:2006E000030041EA401044F20001CDF23851014338461BE103954D46B9462704484600213B
:2007000010AC2246FFF718FD1098010E89F8BF10010C89F8BE10010A89F8BD1089F8BC00B1
:20072000484601212246FFF707FD1098010E89F8C310010C89F8C210010A89F8C11089F85E
:20074000C00005F5803047EA000203984F4643693046012198474846FFF746FD4846002133
:200760002246FFF7E9FC1098010E89F8C710010C89F8C610010A89F8C51089F8C40048468F
:2007800001212246FFF7D8FC1098010E89F8CB10010C89F8CA10010A89F8C91089F8C800DC
:2007A000DDE906654EF65144C0F61034C7F890A008F0030007EB8000BC3023F0A1FB09999C
:2007C00008601CE042F2E661C1F60421085C4EF6F061C0F610210143384610AA27F090FB60
:2007E000DDE91001C7E933012B4607EB8400D0F8CC001860079D4EF65144C0F610340BF1D8
:20080000010BB345FFF68CAE9CE038464EF6F061C0F610210EAAA0462C461D4627F070FB3A
:200820000E98286025464446E9E70993D7F8EC0058B1504600210BAA19F041FC024600204B
:200840000A9009E0D7F8D000DFE6504600210BAA0AAB27F0CFFA0246501C099B09D062B964
:20086000BAF1020F40D0BAF1000F42D1D7E918013CE04FF0AA300F9039E00199386A4B6929
:20088000012198473846FFF7AFFC0A9848B30020CDE90C00384601210DF130084246FFF765
:2008A0004BFC0C9C384600214246FFF745FC0F944EF65144C0F61034079D0C980E901EE091
:2008C000C2B337D1384640F2E031C9F2001110AAA0462C461D4627F013FB2B46254644460E
:2008E00028E03846002107E0D7E91A010F910E9006E04FEA5A0138460EAAFFF71DFC099BEE
:20090000DDE90E1019600B9900293FF478AFD7F8EC100A9A114318BF014659600BF1010BB1
:200920006DE7384640F2E031C9F2001110AA27F0E7FA4346DDE91001CDE90E011860C7F8C8
:20094000D0105CE7002013B0BDE8F08F2DE9F04182B09C461746046A0546666D884673697F
:2009600020460321624698477369204600213A4698474EF61060C0F6156040F20041CDF293
:20098000335148EA0102D5F8EC10002908BF40EA087201927369204601219847736820462A
:2009A00002210022984741F28007C1F2080701AD386A00F11E0800BF7368204602212A469D
:2009C00098470198410009D5400604D4386AA8EB00000028F0DC4FF0FF3000E0002002B019
:2009E000BDE8F0812DE9F04F89B01E4617468B4682461299D0F820800F2000EA216001F05B
:200A00000F05D8F85490012800F29780022D00F2CC80DAF82800C46B504619F0FEF950461A
:200A2000002119F0E0F8504600215A4623460394FFF78CFF0446012D00F0BA80022D40F0DB
:200A4000BF80DAF8EC004AF61C51C1F60121D9F8143051F82020404601219847504600F068
:200A60002BF9044300F108810595CDF808B0D9F8043000254046022100229847D9F80430A1
:200A80000DF1200B404602215A469847089840F480120892D9F8143040460221984700BFA9
:200AA000504600F009F9044316D4D9F80C30404603215A46984765B1B007089807D0307063
:200AC000010EF170010CB170000A707000E0306004360135AF42E3D1D9F80430404602215B
:200AE00000229847D9F8043008AA404602219847089820F480120892D9F814304046022118
:200B00009847002C00F1B880504600F0D5F8044300F1B2800497D9F80C3008AA40460321E0
:200B20009847B007089800F0C5803070010EF170010CB170000A70707FE0139B03280DD00D
:200B400002281BD19AF8DE0078B3DAF88820504627F026F8D9F830A0002007E0DAF88C2079
:200B6000504627F01DF8D9F830A00120CDE90050404659463A463346D0478AE0082814D335
:200B80000816182202EA513200F007001044BAF89820002A00F08080904206D2DAF82C20F7
:200BA00052F83000C4B2FF2C79D14FF0FF376FE00595CDF808B04AF62C50C1F6012006E07B
:200BC0000595CDF808B04AF62450C1F60120DAF8EC10049750F821B04AF63455C1F601254A
:200BE000D9F81430404601215A4698475046FFF7FBFA04433FD4DAF8EC00D9F8143055F8BE
:200C00002020404601219847504600F055F8044331D4D9F80C304046032108AA9847304630
:200C2000089900F8011B059921B10898000A7070023600E00646013FD2D1002506AA504653
:200C40000021FFF779FADAF8EC100029DDE905100CBFCDE90605079DDDE9033707FA01F115
:200C6000029A521843EBE17169405040084318BF4FF0FF3400E0049F5046012118F0B3FF2C
:200C80004FF0FF31002818BF0F46002CB8BF0F46384609B0BDE8F08F0206032401E020F01E
:200CA000FF025046002326F07BFFD9F830A0CDE900545DE73060C0E72DE9F04182B041F218
:200CC0008005C1F2080504462F6A006A0221466D0022736898470DF1040800BF206A7368A2
:200CE0000221424698479DF80700800606D4286AC01B1E28F2DB4FF0FF3000E0002002B0CE
:200D0000BDE8F0812DE9F04F83B0D0F820B09046DBF85440DDF83090019301290ED0002906
:200D20001F467CD1D0F8E410C9B10021C0F8E410D0F8801048F8041B5F1E11E0D0F8E81019
:200D400090F8DD20D2B300291F4668D10121C0F8E810D8F80010C0F884105F1E5FE01F46A3
:200D6000002F5BD0016F803126F050FF6368584602210022984741F28006C1F208060DF18E
:200D8000080A356A636858460221524698479DF80B0080060CD5636858460321002298470A
:200DA00063685846022142469847013F08F10408306AA7B3401B4845E4DB30E01F4671BBBF
:200DC000016F803126F022FF6368584602210022984741F28006C1F2080602ADD6F820A077
:200DE000019F00BF6368584602212A4698479DF80B0040060BD458F8042B636958460021EA
:200E0000984763685846022100229847013F306A2FB1A0EB0A004845E4DB00E0002701982B
:200E2000C01B03B0BDE8F08F2DE9F0419046066A0D46776D002400BF58F824207B6930466B
:200E4000002198470134A542F6D12846BDE8F0812DE9F0419046066A0D46776D002400BF84
:200E600058F824207B693046002198470134A542F6D12846BDE8F0812DE9F04F8DB09246B3
:200E8000EB2A02DCAAF1EC06FBE00F4604460846EC210BF0B3F97C623D46A06845F8A40FFD
:200EA000267B607BA17BE27B4FF4704303EA002040EA014040EA026045F8540CA169019407
:200EC000002051B1D4F814B09BF801909BF800201406022905D1804624E0804681460024F3
:200EE00020E003399BF802801CD000960BF10300029123F005F8014600F001060298042879
:200F000009D00BF10800029122F0FAFF0299F8640BF10C00F86287F8A060002E40F0B580EB
:200F2000009E01E087F8A0003006002687F8A290C7E91D404FF45160002E0CBF10204FF499
:200F40005066A7F87E00A7F87C605FEA08600DD5012087F8A1004FF4600000EA085008F092
:200F6000200140EAC13080F4801038674AF6A460C1F60120B8624FF0000807F1EC00089099
:200F80000490CDE902A5AAF1EC01CDE9091821EAE17100EB5100CDE905084808C0000790FE
:200FA0000DF10C0A0BAEC1468DF83080CDF82C805046314623221AF01FFC05465046082136
:200FC00004F04AFDB9F1000F06D0B9F1010F08BFA5EB040B01E000BF2C4609F10109B9F167
:200FE000100FE1D1C7E92B4B07F1BC0503AE3046294629F081F807F1C80130462A4621F061
:201000009AFC002530461AF0E6F92DB1012D08BFA0EB040B01E000BF04460135102DF1D12A
:20102000C7E92D4B07F1D40103AD284629F064F80F2400BF28461AF0CEF9013CFAD107F1F7
:20104000E00103A829F058F808AA07CAC7F8A800B1EB4206029814D4811B384629F088F898
:2010600003AD284614210BF0C9F800200590019800680490D7F8A4000690284614F06AFF33
:20108000386230460DB0BDE8F08F40F6FF7021EA00004BE72DE9F04F85B090468346D0F88C
:2010A000A800DBF8C4200390073200EBD2000490102943F63467C1F2080731D30BF1BC0425
:2010C0004FF0010902910D4689F0010909EB490ADBE92B0354F82A1010220092C21C01EB11
:2010E000E20002F00702414606F0A2FD38688068804754F82A0003A904EB8A0351F8292078
:20110000D3E901133E680733DB083668B047103D08F140080F2DD7D8029820F00F0400E091
:201120000024386880688047204605B0BDE8F08F2DE9F84F8346006A9046006D0D46D0F80F
:2011400000A010292DD30124009500BF43F63466C1F208063168DBF8D4000F68DBE93612E6
:201160000732D3085246B847306880688047DBE92D0904FB0900C71CA4F1100650463946D8
:201180002AF01AFA4F4448F8040B0136F6D3103D00240F2DDAD8009820F00F044FF00009DD
:2011A00002E000244FF001090F2D22D143F63466C1F208063168DBF8E0000F68DBE939124B
:2011C0000732D3085246B847306880688047DBE92D0509FB0500C61CA9F10F07504631467F
:2011E0002AF0EAF92E4448F8040B0137F6D344F00F042046BDE8F88F30B59C4603685403CE
:201200002AD490F89D400CB1016E22E0846E644512D1D0F85CE0BEF1000F10D0446804EB82
:20122000CE04043C54F8045C8D4211D9083CBEF1010EF7D111460CE04FF4401109E090F825
:201240009F1000294FF4700108BF4FF4401100E0216802F000520A4303991A61826E6245FF
:201260000CBF446E40F2FF34C3E9054C4FF000029A774FF0010C83F81DC0196090F89C10EC
:2012800019770BD190F87A10FF2908BF30BD0121D960D0E91B10C3E9011030BDC3E901223C
:2012A000DA6030BD2DE9F843054600680022476D88467B680321984741F28004C1F2080403
:2012C0006E46206A00F1C80928687B68032132469847002844BF4FF0FF30BDE8F8830099CE
:2012E000080304D4206A4845EEDD002000E00120C8F80010BDE8F8832DE9F84F9946924604
:20130000884690F8A01031B1414652464B4614F007FC044641E00768B0F876307D6D4EF6D8
:20132000F051CEF200014FF0005226F043FF002831D441F28006C1F20806EB4618F8012BAE
:201340006B693846012198476B683846002100229847306A00F1C8046B68384600215A465E
:2013600098479DF80200C00704D1306AA042F3DD11E000BF6B6800243846022100229847C6
:201380006B683846022152469847B9F101090AF1040AD3D101E04FF0FF342046BDE8F88F1C
:2013A0002DE9F84F1D469046894690F8A01031B1494642462B4614F00FFCBDE8F88F07687C
:2013C000B0F876307E6D4EF6F051CEF200014FF0005226F0EFFE00282ED441F28004C1F266
:2013E0000804EB4658F8042B7369384602219847736919F8010B00F58032384601219847B6
:2014000073683846002100229847206A00F1C80A7368384600215A4698479DF80200C007AD
:2014200004D1206A5045F3DD06E000BF0020013D08BFBDE8F88FD5E74FF0FF30BDE8F88F9C
:201440002DE9F84F002B68D18946074608466FF31300B0F1604F60D097F87B0000285CD00E
:2014600090463C68B7F87430666D4EF20001CEF2010138464FF0005226F09CFE736800250A
:20148000204603210022984733686A4620460321984700983865C0043AD5DDF828A03846EA
:2014A00014F0AAFA97F8311000984FF0010B0BFA01F5C10705D1736940F00102204603219F
:2014C000984787F858A087F859B000207865684200EA090A09EB0801013901EA000BC7E9AD
:2014E00012AB73694EF66872CEF20002204601219847AB4473692046032152469847AA4452
:20150000D345F7D133682046032100229847002525624FF0FF30C4E909000020BDE8F88FA9
:20152000C16D0139C16518BF704743F2707CC1F2080C0023614600BF1A460B681BB103F18B
:2015400058018342F8D1002A18BF02F1580C816DCCF8001021F023BAF8B514460546066DD7
:2015600071B301F00307286A012807D0336806F1180207CA1CF0D9FA0120286207EB47007A
:2015800006EB80053368642705F16C0207CA1CF0CCFA3368F088C10800F00702595CD1400D
:2015A000C90705D0013F04BF4FF0FF30F8BDEBE724B1C11C184629F0FFFF20600020F8BD12
:2015C000336806F19C0207CA1CF0AFFA3068718929F0F2FF206000202862F8BDF8B51446D3
:2015E000054601F00307006A2E6D022807D0336806F1240207CA1CF098FA0220286207EBDA
:20160000470006EB80053368642700BF05F16C0207CA1CF08AFA3368F088C10800F007028E
:20162000595CD140C90705D0013F04BF4FF0FF30F8BDEBE724B1C11C184629F0BDFF2060E2
:201640000020F8BDF8B514460D460646006A376D022807D03B6807F1240207CA1CF065FA03
:201660000220306205F0030000EB400007EB8005B98855F83C0FCA1C214627F0BFF93B6884
:20168000642400BF95E807001CF04FFA68B93B68B888C10800F00700595C21FA00F0C007DF
:2016A00004BF0020F8BD013CECD14FF0FF30F8BD2DE9F04F8FB00F460B90D0F81480DDE9CF
:2016C00018040228CDF81C800DD1102A80F0AC8000240B98121BC07C800658BF07EB840765
:2016E00003EB840300E00024002A00F08881069408930120189EB0400A90DDF82CB01546AC
:20170000DBF81090584639463246199B1CF06DF928EA0701F1404C1CA54238BF2C465FEA4F
:201720008901029548BF2C46002800F16681584603210DAAFFF752FF002800F15E81DBF884
:201740000000099700283FD01899D0F80CA00A9A04FA01F80020C24524BF0120C246CDE909
:2017600000202AFA01F258463946DDF820B05B4614F044FE002800F14081B946189EDDE934
:201780000A7500BF2868514627F05EF9B8EB0A0829D028682969C0680022804598BF01221D
:2017A000CDE90072890058BFD144D3444045C24638BF82462AFA06F2284649465B4614F02B
:2017C0001DFE0028DED518E10A98009001200190584639462246089B14F010FE00285D4631
:2017E000189E00F10A81284627F00EF90028C0F20A81002CAB46099FDDF81C80029D00F100
:20180000FE8004FA06F0DBF810905FEA890158BF07442D1B0699089A214402440892069149
:201820000C467FF46FAFEAE00B98029200694FF0010B3E461546CDE908379A4628EA060341
:2018400080002A4658BF0BEB9302B5EB930F98BF2A46102AC0F09A800B980A92D0F850B0E2
:2018600005963146022223461CF0BFF8002800F1AC8006900495DBF800200BF1AC030BCB1E
:201880000733544602EBD30A43F63467C1F20807CDE90D2AD7F80090DB08D9F80090C84775
:2018A00038688068804701250394DDF82880A946B8F1210F24D343F63466C1F208063168B3
:2018C000DBF8AC000F68DBE92C120732D3085246B84785F001050DA8224650F825A00B981D
:2018E00051464B4600F092F83168064688688047A8EB060804EB86044FF00009002ED7D172
:2019000085F001000DA90B9F51F82010384622464B4600F07BF88146384603210CAAFFF789
:201920001BFE0C9844F82900069800280A9808BF0130A0EB080010EB090A0DD0384627F012
:2019400063F8002844DBBAF1000F099F0B98DDF81C80199C08D540E0384627F01BF8384697
:20196000099FDDF81C80199C00698100DDE9045658BF06EB8A060A9A039BB2EB0A02A5EB7C
:201980000A0503EB8A0A4FF0010B18D00220CDE90004DDF82C904846314693465346FFF7A9
:2019A00087FE00280FD4D9F81000810058BF06EB8B06A5EB0B050AEB8B0A4FF0010B002DFA
:2019C0007FF43CAF0CE0824607E04FF0FF3A04E06FF0020A099FDDF81C801AF103000CD044
:2019E0000B9827F011F8002807D4029A089B002A14467FF56EAE144601E04FF0FF342046BB
:201A00000FB0BDE8F08F6FF00204F8E72DE9F84F91460546006D8A46B0F8AAB0B0F8A86031
:201A200000276FF00F0400BFF00806F007011AF80000C840C0070BD1002BA3F1010806DCF1
:201A4000F11C504629F0B8FD49F8040B013743465E440134E8D32868B90026F0F5FF3846A1
:201A6000BDE8F88F2DE9F04F87B0002A00F0BE809B4690468A46054600696C69109A01217A
:201A80009140CDE90215C2F10301CDE900414FF0000900BF24EA0A01D1404F1CB84538BF6A
:201AA0004746800048BF474628465146022A11DB1646119B1DF025FA002800F19A80032ED0
:201AC00016D1286879005A4614F0E4FDC143C90F084179E0119B1DF014FA002804D4072025
:201AE000002105F00FFE48B14FF0FF306CE000BF286839465A4614F0CDFD65E0022F5C46BC
:201B000056462CD37D1E5C46564600BF072004A905F0F8FD98BB0398807F38B106F0030005
:201B2000029908442021A1EBC00002E001983040C000109A0499C1402046049100F8011B2F
:201B400022B10498000A6070023400E004460398C07C8006029858BF0644013DD6D103207C
:201B600004A905F0CFFDE0B9039DA87FE8B106F00300029908442021A1EBC00018E043F660
:201B80003460C1F2080043F6D1610068C1F20801466843F6CB60C1F208000DF11602302331
:201BA000B0474FF0FF30039D0DE001983040C000109A049921FA00F00490207012B1049895
:201BC000000A60703846009C002812D48144B84210D1109A286907FA02F1830058BF8A44CC
:201BE000B8EB07088B447FF455AF03E04FF0000900E08146484607B0BDE8F08F2DE9F04F5D
:201C000093B0002A00F077819A4617460D461C9CD0F810904FF00111002C08BF4FF001310A
:201C20000391012202FA04F3B4F120010D9358BF0023012C904608BF4FF00118002C08BF45
:201C40004FF00138032C214608BF02218A40CDE90181203958BF0022CDE90B23E11EB1FA6A
:201C600081F14909CDE90510002300BF0993867FD0F814801D9B294622461DF042F90A9580
:201C800028EA0501E14001F1010B5F4538BFBB465FEA8901089748BFBB46012C38D8BEB349
:201CA000002800F13D81CDF81CA00AF10105D8460A9FDDF81890DDF80CA000BF15F8014CED
:201CC0001C9848B1287844EA002407F0030027F00301081A811C01E087F00301052005F01B
:201CE00099FC064604FB0AF1072005F093FC304340D499F8130080060D9858BF07440C9802
:201D00000544B8F10108D9D14FF0000843E000BF002800F105810598029F0BFA00F52C46AC
:201D2000022F08BF1AF0030040D004950AF10105DDF81890DDF8048015F8010C57B129785B
:201D400040EA0120012F05D0697840EA0140A97840EA016000FB08F1072005F05BFC0028AC
:201D6000C0F283800B980544013CE5D1002400268DE000BF43F63460C1F2080043F6D16166
:201D80000068C1F20801476843F6CB60C1F208000EAA3023B84721F06BFF0320002105F093
:201DA000B1FCABEB0800DDF81CA08CE0012DBCD91DF012F906460028CDF81CA069D4049535
:201DC0004FF0FF30109040F2FF10ADF844005546DDF818904FF0010843F6346AC1F2080ACF
:201DE0008DF83D8055F8040B80EA104181EA112181EA111181EA910181EA51013B2262F3F4
:201E00005F018DF83C100E90DAF8000010A947680EA80DF146022E23B8479DF84B0000F09D
:201E20000E00022804D01DF0D7F8002834D40026013C012CD4D8286880EA104181EA112166
:201E400081EA111181EA910181EA510101F001018DF83C100E90DAF8000010A947680EA8E9
:201E60000DF146022123B84717E0064643F63460C1F2080043F6D1610068C1F208014768D0
:201E800043F6CB60C1F208000EAA3023B847049D09E0DDF8189001E00646049D002E3FD403
:201EA0000024DDF81CA021F0E3FE002E05D40320002105F027FC002821DB059925FA01F046
:201EC00024FA01F1401A099B002816D40344584528D11C9C0BFA04F24846D9F810900A9DAC
:201EE000089F5FEA890158BF1544B7EB0B0792447FF4BCAE16E0002314E0034612E043F610
:201F00003460C1F2080043F6D1610068C1F20801476843F6CB60C1F208000EAA3023B8470B
:201F20004FF0FF33184613B0BDE8F08F2DE9F04F83B01C4690460E46074602AD05F10309D9
:201F4000A81C019007F1180B3078252825D81BF800A0F87A0A2115F0A9F8002822D48DF886
:201F600008A03078232801D020280AD102208DF809004046042210F8011B8DF80A10494624
:201F800005E001208DF8090003224046019900780870F87A294600F0D7FB08F10408013699
:201FA000013CD1D1002003B0BDE8F08F70B5044600F00CFAE07A002115F078F8002844BFCB
:201FC0004FF0FF3070BD41F28005C1F208052E6A204614F091FE38B9286A801BB0F5967F85
:201FE000A4BF002070BDF3E7012070BD2DE9F843602A69DB16460C460546084660210AF028
:20200000FDF8D5E90512C4E91612287A20726B7A6372AB7AA372EB7A23732B7B63736B7B9C
:20202000A373AB7BE373EB7B2374072A25DB0A7822764A7862768978A17604F11B010322DE
:20204000002300BFCA54013301321D2BFAD1202184F83810D4E91612F0274B7984F83A701B
:2020600084F83930CB7884F83B30812384F83C300B7984F83D30072A01DAB42300E08B7991
:20208000E37208B909202072A6F16009082A10DBCB7963740DD00B7AA3740A2A09DB4B7AE1
:2020A000E3740C2A05DB8B7ACF7A43EA0723636025D10022904238BF1046012101FA00F601
:2020C00006EBD600814503DA4FF0FF30BDE8F88304F160004FEAD608E6648719C4E91007EE
:2020E00031460AF08BF8384641460AF087F828682060A9EB0600A0EB0800BDE8F8830D2ADA
:202100000A7B22751CBF497B6175D3E72DE9F04F85B09A460F4604460E9802FA00F60020B3
:20212000B0EB116F5BD18DF80E00607A18B10DF10E0100F031F90296002E4ED0607A28B164
:20214000B7F5803F06D3FD0B0CE000BFBFB2002508E000BF9DF80E0000F00F05B7F5004FA9
:2021600038BF0025B8B2217A227D1AB16368984228BF1146012202FA01F14A1E02EA000983
:20218000A1EB0908B04528BFB046494200EA010B606D60B1A06C834504D194F85000E9B251
:2021A00081420AD0204600F011F9606D28B984F8505001206065C4F848B0206C484451460F
:2021C000424609F0F5FF606C4946424621F0A3FEB6EB0806C2444744AED1029ED1E0B0EB4A
:2021E000576F09D10C200090204639463246534600F060FA0646C4E0380E02284ED8204657
:2022000000F0E4F8002E7BD0B346029607F07F00C0F18008D845A8BFD84638060AD40A2051
:202220000090204639464246534600F043FA81462CE000BF07F17E404FF0FF3101EB102602
:20224000050A0ED0A07A60B120460DF10F0126F025FCF1B29DF80F00884202D020461CF066
:202260004AFF0A200090204639464246534600F021FA81464DB1A07A38B19DF80F10F0B22C
:20228000814202D020461CF036FF029EC14576D1BBEB080BC2444744B8D131E00020B0EB76
:2022A000976F74D1E06D002869D0607BBFB260B3012864D10DF11108354600BFFF2DA946FC
:2022C000A8BF4FF0FF09E07A0F2114F0EFFE002855D48DF813908DF81270380A8DF811007D
:2022E000E07A4146032200F02FFAE07A51464A4600F02AFAB5EB0905CA444F44DED140E00C
:20230000B8F1000FB8BF46463BE0A07BB8B3E07BA8B3207C98B3A07A04A900F03DF8217B3C
:202320009DF81000884202D0A07A00F0F1F93546E07B5FFA87F8414600F0EAF9A07BC7F38B
:20234000072100F0E5F9C8F580784545B8BFA846C14600BF1AF8011B207C00F0D9F9B9F1E7
:202360000109F7D1B5EB08054744E1D1207B9DF81010814205D0A07A00F0CAF901E04FF0CC
:20238000FF36002E03DB0E9846FA00F001E04FF0FF3005B0BDE8F08F10B50C460AF050F9A4
:2023A00040F20800C2F2000043F63C11C460C1F2080101220968C0E90521BFF35F8F0221A3
:2023C000016000BF01680029FCD110BD2DE9F04F8DB00446406D002800F06981207D04F194
:2023E000080818B16168A26C8A4204D298F800004FF0010A01E04FF0000A012101FA00F971
:202400002046494614F060FFA07A58B10DF12701204626F043FB9DF8270018B12046002155
:202420001CF069FE607C70B10DF12A01FFF7B4FF9DF82A10880706D4607C41F0020100F022
:2024400067F9002600E00126A07C40B3E17C31B30DF12901FFF7A0FFE07C0AA9FFF79CFF42
:202460009DF829009DF9281082070AD5002908D400F0FD018DF82910A07C00F049F99DF8D4
:20248000281048B200280ED4E07C41F08001C9B200F03EF969200AF0C4F8012504E00120E6
:2024A000049000250DE000259DF82910880706D4A07C41F0020100F02BF9002000E0012095
:2024C0000490A06C94F8501049B198F80020A0F50040D040C903D14051FA80F808E0BAF1AE
:2024E000000F1ABF98F8001020FA01F8C0F30718E07A082114F0DAFD089068B9E07A5FFAA5
:2025000088F114F0D3FD089030B900200890E07A08A9012200F018F9607A78B10DF12B01D9
:20252000FFF73AFF94F850009DF82B2040EA0010C1B28A4202D0607A00F0EAF8206C059098
:20254000B4F84800069040F20807C2F2000741F28008C1F208080DF1300AB9F1FE0FCB4677
:20256000A8BF4FF0FE0BE07A072114F09FFD00286BD48DF82EB006988DF82D00000A8DF8E1
:202580002C00E07A07962E460BAD2946032200F0DBF8E07A29463546079E012214F01AFE6D
:2025A0009DF82C000D2850D10395CDE90194E07A0AF046F8D946059E012443F63C10C1F270
:2025C0000800FE600068C7E90540BFF35F8F3C6038680028FCD10136D8F8200000F5FA75DC
:2025E0005046F6F729FA0C98810705D5D8F820008542F5DA26E000BFC00710D00DF12F0010
:20260000F86043F63C10C1F208000068C7E90540BFF35F8F0220386038680028FCD1B9F12C
:202620000109CAD1DDF804900698B9EB0B0958440690059858440590079EDDE902457FF411
:202640008CAF02E0079EDDE90245607A50B194F850209DF82B1042EA0212D2B2914218BF96
:2026600000F056F80020606584F85000A064606CE26C002128F0ECFF26B9607C9DF82A109F
:2026800000F046F8049820B9A07C9DF8291000F03FF825B1E07C9DF8281000F039F8A07A4C
:2026A00028B19DF8271011B120461CF024FD0DB0BDE8F08F2DE9F84F9B4690460546CFB25F
:2026C000DDF828A00DF10209164600BFFF2E3446A8BFFF24E87A514614F0E8FC002812D419
:2026E0008DF803408DF80270E87A4946022200F02BF8E87A5946224600F026F8361BA34444
:202700002744E3D101E04FF0FF384046BDE8F88F80B58DF8031009F093FF40F20800C2F24B
:2027200000000DF10301C16043F63C11C1F2080101220968C0E90521BFF35F8F026000BF10
:2027400001680029FCD108BD2DE9F84F93460E46C0B209F075FF40F20807C2F200070124CB
:2027600043F63C19C1F2080941F28005C1F20805EA46FE60D9F80000C7E90540BFF35F8F9B
:202780003C6000BF38680028FCD10136286A00F5FA7800BF5046F6F74FF99DF80000800773
:2027A00004D5286A8045F5DA06E000BFBBF1010B08BFBDE8F88FDCE7BDE8F88F2DE9F84F7E
:2027C0009B4690460546CFB2DDF828A00DF10209164600BFFF2E3446A8BFFF24E87A51468B
:2027E00014F064FC002812D48DF803408DF80270E87A49460222FFF7A7FFE87A594622468E
:2028000014F0E8FC361BA3442744E3D101E04FF0FF384046BDE8F88F2DE9F84F9B461646D6
:202820008A460546D0F88C1100F5DC7026F0FCFA4FF62074C3F601442846214615F0F4F82E
:20284000284626F03BFB4FF0000904F1E0000090002400BF1AF8010B04280BD8013803289D
:2028600000F2C680DFE800F0026B6E7130686860BEE000BF1F2825D8D5F8501205EBC10735
:202880004B1C87F85892D6F80080C5F850324FEA004C4CEA184202F17052C7F854221FFAC3
:2028A00088F7002F46D005EBC302023182F85892C5F850124CEA4050384340F05050C2F81E
:2028C000540237E0382808D8242860D02C2856D0302867D1306868618AE03A2838D8D5F8BB
:2028E000501205EBC102009F82F85892336847EA1347C2F854729BB24A1C53B105EBC202AF
:202900000027C3F242473B4382F85892C2F854328A1C511C3A2805EBC20080F85892C5F8EA
:20292000501240F21101C0F2400118BF0231C0F8541200BF2846002100F020FF52E03068AF
:20294000A86055E03068E86052E0306828614FE0A0F1410130294BD829684FF6FF72C1F28F
:202960000112914244D140F65211C1F604210844336810F8410CC10800F007022FE0306842
:20298000A969814234D001212977A86130E040F63911C1F604210844012410F8200C00F092
:2029A00007021AE040F63911C1F604210144352811F8200C00F007020FD129684FF6FF73C0
:2029C000C1F20213994207D04FF6FF73C1F20113994208BF013200E001323368C108284645
:2029E0001CF0F3FD002844BF4FF0FF30BDE8F88F0436BBF1010B7FF42DAF14B128461CF096
:202A0000ACFC0020BDE8F88F2DE9F8430446D0F88C1100F5DC7026F007FA20461CF09DFC5F
:202A2000204615F08FF904F5B070202109F0E6FB0027C4F84872204626F040FAD4F85022DE
:202A400004EBC200B946C3F6024980F85872A9F1D001C0F85412501C6369D9053D46C3F2A9
:202A6000214548F20001C4F2820118D404F5157849EA134648F8306043F4807308EBC000D1
:202A8000636108EBC20607713775377701F56050B06105F504109BB218433061101D227F19
:202AA000F2B104EBC003002283F85822A76949EA1746C3F85462431CBFB24FB104EBC30314
:202AC00005F5041683F858223743C3F85472831C04EBC300227780F85822C0F85412581C84
:202AE00004EBC001002781F858721822C3F20342C1F8542281F8607241F62702C0F260029A
:202B0000C1F85C2281F868720022C8F62242C1F8642281F8707241F22403C0F24303C1F842
:202B20006C3281F8787202F10052C1F874220530C4F850022046002100F020FE002800F10F
:202B4000B180D4F8500204EBC00105F1FC6381F85872626843EA1243C1F8543291B2421CB2
:202B600041B104EBC202002382F858322943C2F85412821C04EBC200002180F85812A368A0
:202B800049EA1347C0F85472501C9BB25BB104EBC007901C87F85812C4F8500205F50412FC
:202BA0001A43C7F8542204EBC003002283F85812E768C3F6034242EA1741C3F85412411C7B
:202BC000BBB253B104EBC101002781F8587205F584073B43C1F85432811C04EBC1030020B7
:202BE00083F85802276902F5803242EA1742C3F854224A1CBBB24BB104EBC20205F5C607C8
:202C000082F858023B43C2F854328A1C04EBC201013281F858020F20C1F85402C4F8502258
:202C20002046002100F0AAFD00283BD4204626F045F9D4F8500204EBC001002281F85822A2
:202C40001F22C4F20022C1F854220130C4F850022046002100F092FD002823D441F280060F
:202C6000C1F2080604F50078306A00F5FA7740F20025CFF6207500BFD4F88C11404626F0AD
:202C8000D3F8D4F88C01D4F83C1228F095FC000704D5204626F0EEF8A84207D0306A381A5E
:202CA0000128E9DA4FF0FF30BDE8F883204600F003F80020BDE8F8832DE9F041044626F062
:202CC0007BF808B1BDE8F081D4F88C1104F50078404626F0A9F8D4F80C02D4F840224DF254
:202CE0000001C8F2040126F0BFF8D4F88C1104F5037026F099F820684FF6FF71C1F20011CA
:202D0000884250D1D4F88C1104F5D67026F08CF8D4F88C1104F5E27026F086F8D4F8DC0195
:202D2000D4F82C2200211CF0EEFBD4F88C1104F5EE76304626F078F8D4F88C11D4F82C221E
:202D4000D50812F00703C3F108004FF0FF3707FA00F74D5D25FA03F323EA070305D001EBCA
:202D6000D2077F7807FA00F00343980717D4D4F8DC01FE211CF0C7FBD4F88C11304626F037
:202D800053F8D4F8DC01D4F82C2200211CF0BBFBD4F88C11304626F047F8D4F88C1104F5AC
:202DA000DC7026F041F841F28007C1F20807D4F88C61386A00F5FA754046314626F034F8FE
:202DC000D4F88C61D4F83C12304628F0F5FB000708D4386A281A0128BCBF4FF0FF30BDE824
:202DE000F081E9E7204626F085F80120BDE8F081B2F53D7FBCBF4FF0FF3070472DE9F04118
:202E00008AB015460F46064608464FF43D7109F0F5F93146707A11F8082F42EA00208A7867
:202E2000C97842EA012140EA0140C7F89001306838600026C7F84462099607F53D7007F549
:202E4000C871CDE90210A5F53D71CDE9070121EAE17100EB5100CDE904064808C00006906C
:202E600002AD28460A21052227F0F2F880208DF8030004208DF80200C0208DF801008DF824
:202E8000006069462846202218F0B6FCC7F83C02059810F0070004D0C0F1080102A802F0EE
:202EA000DBFD07F5007102AD284627F025F98DF80460009628460A21052227F0C9F86946B5
:202EC0002846202218F098FCC7F84002059810F0070004D0C0F1080102A802F0BDFD07F521
:202EE000037102AD284627F007F900208DF80400009069462846212218F07EFCC7F830021E
:202F0000059810F0070004D0C0F1080102A802F0A3FD07F5F47102AD284627F0EDF808249D
:202F20006E4600BF28463146212218F065FC80462846032102F090FD082C04BF0598C7E972
:202F40008980013CEED1059810F0070004D0C0F1080102A802F080FD07F5067102AD284691
:202F600027F0CAF869462846082218F045FCC7F82C02059810F0070004D0C0F1080102A81F
:202F800002F06AFD07F5EE7102AD284627F0B4F828460421052227F05BF8059810F00700D5
:202FA00004D0C0F1080102A802F056FD07F5D67102AD284627F0A0F828460521052227F0B3
:202FC00047F8059810F0070004D0C0F1080102A802F042FD07F5DC7102AD284627F08CF8A4
:202FE00028460721052227F033F8059810F0070004D0C0F1080102A802F02EFD07F5E2718A
:2030000002AD284627F078F828460921052227F01FF869462846202218F0EEFBC7F83402DA
:20302000059810F0070004D0C0F1080102A802F013FD07F5CA7102AD284627F05DF8284684
:203040000E21052227F004F8059810F0070004D0C0F1080102A802F0FFFC07F5E87102AD3A
:20306000284627F049F828460321052226F0F0FF059810F0070004D0C0F1080102A802F0FE
:20308000EBFC07F5FA7102AD284627F035F828460821052226F0DCFF69462846202218F06B
:2030A000ABFBC7F83802059810F0070004D0C0F1080102A802F0D0FC07F5D07102A827F0D9
:2030C0001BF807AA07CAC7F88C01A1EB42000AB0BDE8F0812DE9F04F8BB0984614468A46D9
:2030E0008346D0F88C1100F5DC7025F09DFE0020CFF6207000F5500000EA0A0010F1814F32
:20310000149D0BD00020CBF68070824509D204FA05F05044013810F1814F02D358461CF0A0
:203120001CF95FEA88704FF0010006900CD10690202C09D31AF0030006D1022D04D1584642
:2031400000F060F9002006900020ADF828000BF5E87004900BF120070BF5157003902646F0
:20316000059700BF06FA05F0CDE907A0584607A900F0A2FA08989DF8291020FA05F929B168
:2031800009FA05F1404609F039F809E09DF82800A8B10998391809FA05F2404609F008F81C
:2031A0004846002800F1C080361A484540F0C08009FA05F082448044002ED3D1B7E0DDE92A
:2031C000060740B10095584639464A46434614F089FC059FE5E70194DBF800000290584695
:2031E00025F06CFEDBF85002039C0021C3F6014141EA174144F8301004EBC001C3F22147A4
:2032000000250D710D738F600D754FF62072C3F602420A610D770423C3F242438B6181F891
:20322000245002EB1942E0320A6281F82C504A46C3F263428A6281F834504FF6FF72C1F223
:203240000212029B934240F60002CAF2000208BF4FF000420023C3F6044343EA12430B6397
:2032600081F83C50C3F2634202F504128A6381F844500F220A640930CBF85002584600213C
:2032800000F07CFA584625F019FEDBF8500204EBC0010822C0F2800244F830200D710D7341
:2032A0008D600230CBF850025846002100F066FADBF88C11049825F0B7FDDBF8E801DBF867
:2032C000301201F00702C910012303FA02F2435C23EA020242544C464546059F58460021FE
:2032E0002A4614F04BFB00281ED40435013CF5D141F28000C1F208000025006A00F57A74DE
:20330000CFF62075584625F0B5FDA84208D041F28000C1F20800006A201A0128F2DA03E042
:203320004846019C149D3CE74FF0FF3001E00026A01B0BB0BDE8F08F2DE9F04F87B09B4612
:2033400017460E468246D0F88C1100F5DC7025F06BFD109D07FA05F430466FF3130010F13E
:20336000814F09D00020CBF68070864207D23019013810F1814F02D350461BF0EEFF5046E6
:203380003146224614F0AEFA0020ADF818000AF120080DF10C09029707FA05F0CDE90360E7
:2033A0005046494600F088F904989DF8191020FA05F449B99DF8180098B10598404404FAF3
:2033C00005F2594608F0F4FE2046002811D43F1AA04212D104FA05F006448344002FDBD1FD
:2033E0000AE003990095504622465B4614F00CFCEBE74FF0FF3002E000270298C01B07B092
:20340000BDE8F08F2DE9F047BEB00446D0F84402002840F016814FF6FF70C1F2001000F51A
:20342000003122688A4240F6000AC8F2000A0AF1005508BF4FF000450227824240F0898040
:20344000009704F1600342F21006CBF6887620463146012214F046FB009706F1100904F193
:20346000640320464946012214F03CFB009706F1200A04F1680320465146012214F032FB29
:20348000009706F1300104F16C032046012214F029FB4FF400603B90E06ECDE93C00009713
:2034A0000DF1EC08204631460122434614F0ACFB009708F1040320464946012214F0A4FB94
:2034C000009708F1080320465146012214F09CFB009704F1200320462946102214F002FBDF
:2034E00000974BF26C03C1F6012320462946102214F08AFB24208DF80B000DF10B012046DA
:203500004246012313F07AFFDDF8EC900DF16C084046802108F072FE0DF10C0A5046202146
:2035200008F06CFE226E8AB3616E79B3A06E68B34FF000531D934FF00047CDE91B728F1A84
:2035400000F08280CDE9207382F000421F9202257BE0009704F1200320462946102214F08F
:20356000C1FA00974BF26C03C1F6012320462946102214F049FB002084F87C004FF000507C
:203580004021C4E91CA1A067012055E04FF000401B904FF000501D90E06E1C900026012557
:2035A00008EB05174FEA051A38464146524608F005FE07F1080000212A4600BF016050F813
:2035C000083C03F1005340F8083C1030013AF5D15FEA497002D44FF0000A1CE00BAF1BA908
:2035E0003846524608F0EAFD07F108004FF020412A4600BF016050F8083C83F0004340F82C
:20360000083C1030013AF5D104F170000BA9524608F0D4FDAA4604F1700707EB0A10320110
:2036200003A908F0CBFDB24407EB0A106A011BA908F0C4FD0AEB45000121C4F84412C4F80A
:2036400050013EB0BDE8F0870125421A15D02B0181F0004748F8037008EB051301261E734E
:203660004FF00057C3E901274FF00453CDE9042301F1FE410391013500E00026E16E091AFA
:203680008ED0320100F1FE434AF802302A0180F0004048F802000AEB06104FF00452C0E98D
:2036A000011208EB0510012202734FF00052C0E901120135013673E770B500228A818A6007
:2036C000D0F84422002A58D00B68D0F85021012A2CDB00F17C0CA3F1010E00BF5CF80C4C05
:2036E0009C4205D94D687544A54207D30BE000BF5CF8085C6619013EB34207D9013A0CF1B2
:20370000100CEBD112E0E21A4A600FE0E21A2A449CF800604E735CF804CC6344D1F804C0D3
:20372000944538BF6246C1E9003236BB00684FF6FF72C1F20212904240F60000CAF200009B
:2037400008BF4FF0004083420ED300F13F0293420AD8181A01220A738860C0F140004A6837
:20376000824238BF104607E0834206D24A681A44013A824201D3C01A486070BD2DE9F84FC5
:203780000C468346D0F84C02DBF850924FF0000A002600BF082815D1002558464FF6FD7189
:2037A000C1F20001002214F0E9F80746AEB10BEBC60090F8500280B1800706D458460021BB
:2037C000224605E0002700250FE021685846002214F0D4F8074304340125584600210022BF
:2037E00014F0CCF8CBF84CA207430BEBC6085846D8F85412002214F0C1F807439EB195B9A8
:2038000098F8500228B1800705D458460021224604E0002507E021685846002214F0AEF883
:20382000074304340125002F0BD4DBF84C020430CBF84C020136B145ACD12DB10027CBF8FA
:2038400050723846BDE8F88F0BEBC60595F850120029F3D008280FD158464FF6FD71C1F24C
:203860000001002214F08AF895F85002800710D45846002122460FE058460021002214F05A
:203880007DF895F85002800711D458460021224610E021685846002214F070F800255846D9
:2038A0000021002214F06AF8CBF84C52C6E721685846002214F062F8DBF84C020430CBF892
:2038C0004C02BBE7F8B51C4615460E46074600BF16F8011B38462A4625F0C6FB002848BF11
:2038E000F8BD0435013CF3D10020F8BDF8B51C4615460E46074600BF16F8011B38462A4622
:2039000025F0F0FB002848BFF8BD0435013CF3D10020F8BD2DE9F04F87B0002A68D01C4664
:203920001746894680461DF092F84BF2BC11C1F6012140460322002300F076F8054640461E
:2039400003214A4603231DF0E2F8054304AA404604211DF044F955EA000661D4109800F0A9
:2039600003054BF2C810C1F60120DDF8109050F8251040460422002300F056F800284ED409
:20398000CDF80490012000FA05F90026FF2FCDE90274BA4688BF4FF4807A0134D34600BFA4
:2039A00014F8012C25B1207842EA0022012D01D1002007E06078A17842EA004040EA016221
:2039C00041F3C01040F00303404604211DF09FF800280FD44C44BBF1010BE1D1DDE902741D
:2039E000B7EB0A0756440AFA05F00444CED102E0002615E0064640460221019A01231DF0DC
:203A000086F805464BF2D811C1F6012140460222012300F009F8284348BF064600E0064635
:203A2000304607B0BDE8F08F2DE9F8431C46174688468146551E0026A81BB0FA80F04009D1
:203A4000002C214618BF012111EA000318BF0223102E38BF43F0010358F8262048463146D9
:203A60001DF055F8002848BFBDE8F8830136B742E2D10020BDE8F8832DE9F04741F2800575
:203A8000C1F2080504462E6AD0F8ECA043F63467C1F208073968206ED1F80080D4E9191339
:203AA000D4F8C0200733DB08C047386880688047D4F8C080B4F850104046022200F022F81B
:203AC000E8B120F0010002281CBF6FF00100BDE8F0873968E06ED1F80090D4E91C1207324F
:203AE000D3084246C847386880688047286A801B5045A4BF6FF00200BDE8F087CAE7002092
:203B0000BDE8F08700B54FEAE10C01F0070310F80CE02EFA03FEC3F1080393420ADA60447A
:203B2000013000BF10F8011B99404EEA010E08339342F7DB4FF0FF3090402EEA000000BD5C
:203B4000F8B50446D0F8E450A801411C204625F051FD0120C4F2000040EA85110091204615
:203B600025F048FD2068112142682046904741F28006C1F208066D46376A00BF206894F8A9
:203B8000111101290AD102692046294690472068112142682046904705E000BF8368204651
:203BA00011212A4698479DF80200800707D4306AC01BB0F5FA7FE1DD4FF0FF3500E00025C2
:203BC000D4F8E4008001411C0091204625F012FD2846F8BDF8B541F28006C1F208060446A8
:203BE000376A6D46206894F8111101290AD102692046294690472068162142682046904779
:203C000005E000BF8368204616212A4698479DF80100C0065CBF0020F8BD306AC01BB0F5C3
:203C2000FA7FC4BF4FF0FF30F8BDDBE72DE9F8431C46164605461A4600231EF08CF9012012
:203C400000FA04F995F81101DDF8208001364746012829D116F8010C012C07D064B940EA0C
:203C6000002141EA004141EA00620EE0317840EA004040EA012006E0317840EA012071781B
:203C800040EA0140B17840EA016228683C21036828469847284600F047F8002833D44E4400
:203CA000013FD7D12DE000BF16F8010C012C07D064B940EA002141EA004141EA00620EE0E2
:203CC000317840EA004040EA012006E0317840EA0120717840EA0140B17840EA0162286812
:203CE0003C2103682846984728683821426828469047284600F018F8002804D44E44013F97
:203D0000D2D1002600E046462868C16828468847284621461EF062F90021002808BFA8EB97
:203D200006010846BDE8F883F8B541F28006C1F208060446376A6D46206894F811110129E9
:203D40000AD102692046294690472068382142682046904705E000BF8368204638212A46EB
:203D600098479DF8020080065CBF0020F8BD306AC01BB0F5FA7FC4BF4FF0FF30F8BDDBE75C
:203D80002DE9F843134688460446B0F84E10D0F88400D4F8EC9000EBD10001F007021946B2
:203DA00027F01CFC236CD4F88400B4F84C20414614F042FA41F28005C1F208052F6A00BF46
:203DC00004F184030ECBD4F8C0001EF068F9B4F85010D4F8C08040461EF074F9B8B10646C5
:203DE00004F16C030ECB40461EF059F9032E0AD1286AC01B4845E3DB04F178030ECBD4F8C7
:203E0000C0001EF04CF94FF0FF30BDE8F8830020BDE8F8832DE9F8430446B0F84C20036CA3
:203E2000D0F89000D4F8EC9014F006FA41F28005C1F208052F6A00BF04F190030ECBD4F8E1
:203E4000C0001EF02CF9B4F85010D4F8C08040461EF038F9B8B1064604F16C030ECB40461A
:203E60001EF01DF9032E0AD1286AC01B4845E3DB04F178030ECBD4F8C0001EF010F94FF02F
:203E8000FF30BDE8F8830020BDE8F8832DE9F84341F28005C1F2080504462F6AD0F8EC90A3
:203EA00004F19C030ECBD4F8C0001EF0F8F8B4F85010D4F8C08040461EF004F9B8B10646AD
:203EC00004F16C030ECB40461EF0E9F8032E0AD1286AC01B4845E3DB04F178030ECBD4F857
:203EE000C0001EF0DCF84FF0FF30BDE8F8830020BDE8F8832DE9F8431D4690460C4606462A
:203F0000B0F85090042700BFD6F8A80002214A46022314F091F9336CD6F8A80009F1220220
:203F20003C2114F089F9B6F852008144013FEBD130462146022200231EF00DF84446B8F173
:203F4000040F29D3B6F85090002700BFE819E95D427841EA02218278C07841EA024141EAC4
:203F6000006109F10202D6F8A80000EBD20002F0070227F033FB0437102FB6F85200814430
:203F8000E4D106F1A8030ECBD6F8C0001EF087F83D44043C032CD5D8336CD6F8B400B6F86A
:203FA0004C203C2114F048F9D6F8B400B6F850200221022314F040F90CB300BFB6F84E2034
:203FC000D6F8B40015F8041B00EBD20015F8033C41EA032115F8023C41EA034115F8013CD7
:203FE00041EA036102F0070227F0F8FA06F1B4030ECBD6F8C0001EF052F8013CDED130465F
:2040000002211DF0EBFF002818BF4FF000084046BDE8F8832DE9F84F1C4690468A460746E8
:2040200040F20009CFF62E294FF6FF7BC0F6105B58F8045B1AF8016B0F2E0FD8280440EAA2
:20404000063000F2FB2016F0B7F849EA154000F091FC002840F196809AE000BF192E00F084
:2040600091803869584509D06FF07241884205D04FF6FF71C0F62051884202D1182E00F0B8
:204080008180182E17D8304625F0F4FC290641EA004047F2FD31084316F08EF8280A00F174
:2040A000385016F089F840F2F930C0F2033000F061FC00286CD406F0FE001A282BD146F68E
:2040C000FD00CFF6173016F077F82802123016F073F81B2E4FF60050C0F2171004BF4FF6C6
:2040E0000050C1F2171040EA156016F065F84FF22E40C0F2033000F03DFC002848D446F657
:20410000FD20C2F6716016F057F840F2F930C0F2033004309BE71C2E34D3786990B31F2EEC
:204120001BD846F6FD00CFF6173016F045F82802123016F041F8A6F11C00C1B2022941F2D5
:20414000FD71C0F2B10106D840B24BF20841C1F6012151F820100802C5E7202E12D147F2C5
:20416000FD30C0F20D0040EA056016F025F8280A00F1385016F020F840F2F930C0F2033098
:2041800065E700BF013C04BF0020BDE8F88F4FE74FF0FF30BDE8F88F2DE9F04383B0044632
:2041A00013208DF80B00002000900DF10B0101AA2046012300F076FA47F2FD38C0F21008B5
:2041C000019D48EA056015F0F7FF280A00F1385015F0F2FF40F2F939C0F20339484600F03E
:2041E000C9FB002827D447F2FD30C0F2111015F0E3FF4FF0385015F0DFFF484600F0BAFBDB
:20420000002818D42046012115F026FE41F28007C1F20807386A00F1640500BF20461DF02F
:2042200060FF01280AD00646002804D4386A281A0028F3DC03E04FF0FF360FE0012608F58B
:20424000803015F0B9FF4FF0385015F0B5FF484600F090FB0028B8BF4FF0FF36304603B02C
:20426000BDE8F083F0B583B0C6208DF807000DF10700012401AA0225012102231DF0AEFFDF
:2042800002280ED18DF809408DF8085088208DF807000DF107000321002200231DF09EFF1E
:2042A00020B14FF0FF34204603B0F0BDC6208DF8070041F28006C1F208060DF10704306A66
:2042C00000F5FA7701AD00BF204601212A4602231DF084FF0228E4D1BDF80400C00705D129
:2042E000306A381A0028EFDC002400E0012402208DF8080088208DF8070000208DF8090025
:204300000DF107000321002200231DF067FF002818BF4FF0FF34C6E72DE9F04F8BB099462F
:2043200093468A4604461DF082FF0121C8F2000108B10846B4E007941498012101FA00F729
:20434000784202900DF1270808F1010001900DF1220400265D46CDE903B7CDE905954FEA73
:204360001A6B4FEA1A454FEA1A2700BF8DF826B08DF825508DF824708DF823A08A208DF802
:20438000220020460521C1464246012300F042F9002815DB00208DF826008DF82500149858
:2043A0008DF823008B208DF8220001208DF82400204605214A46012300F02CF9002810D5D7
:2043C0006FF00201411A18BF01213143C90767D107981DF02CFF012600280DF12204C5D0CC
:2043E0005BE0069D022D30DBCC208DF822000DF1220001214246052300F00CF90028DDE93D
:2044000004791ED4691E149A019E91400AEB010B052856D1484631463A4607F0C9FEB944F3
:20442000022D36DDBA44013DCC208DF822000DF1220001214246052300F0ECF80028E7DABC
:204440000026DDF80CB08EB12AE0DDE904790DF12200CD218DF8221001214246052300F092
:20446000D9F80028DDF80CB020DACEB9C11C17D15D4518D002988144AAEB070A0135079808
:204480001DF0D5FE012600280DF122043FF465AF03E000260125DA46D9E70120C8F2000098
:2044A0000BB0BDE8F08F6FF00200F9E7052808D1484601993A4607F07BFEABEB05000130F2
:2044C000EEE74FF0FF30EBE72DE9F04F85B0984692460E9B012909D0002954D10F98009056
:2044E00050464146002200F053F84CE084208DF80B00C62041F28005C1F208058DF80A00F5
:20450000286AC4180DF10A060DF110090DF10B0B474600BF304601214A4602231DF05EFEF2
:20452000022808D19DF81100C00604D5286A201A0128EFDA25E05AF8040B04908DF80C00EA
:20454000010E8DF80F10010C8DF80E10000A8DF80D0000BF584605214A4601231DF03EFEDC
:20456000012809D19DF81000000704D5286A201A0128EFDA05E0013F286A17B1201A002814
:20458000C8DCA8EB070040EAE07005B0BDE8F08F2DE9F04F83B08A4606466FF03A00002A23
:2045A00008BF01388DF80B000C98012141F28004C1F2080401FA00F9206AC5180DF10607C9
:2045C000781C00900DF10B0BD04600BF584601213A46052325F07CFA012804D1206A281A11
:2045E0000028F3DC0EE005280FD136B1304600994A4607F0DDFD4E4400E00026206AB8F1A7
:204600000108ECD1AAEB080001E06FF0010003B0BDE8F08F2DE9F04782B0984616468A4696
:20462000054625F055FA012817DB0446652740F20109C8F2000900BF307810F0C00F0FD1C5
:2046400000072BD5013F0DD0284651463246434625F03EFA04460128EEDA6FF001041DE047
:204660004C4601E06FF0020400208DF8070006208DF8060088208DF805000DF1050528465D
:204680000321002200231DF0A9FD02208DF8060028460321002200231DF0A0FD204602B0B8
:2046A000BDE8F0872DE9F04F89B0994692468B460746C620069006A805AA012102231DF04E
:2046C0008DFD022840F01981059810F400780AD00220009003A8012101221423FFF758FF43
:2046E000012840F00A8146F6FD00CFF6173015F063FD002800F1018148F21E40C0F6400003
:2047000015F05AFD002800F1F88041F2E320CFF22E6000F02FF9002800F1EF8002240094CD
:2047200007A8012101221423FFF732FF012840F0E48046F6FD20CEF2723015F03DFD42F638
:204740001260C0F2FB3000F015F9009408A8012101221423FFF71CFF012840F0CE8000256F
:204760001BF8016B0F2E05D8022E1AD0012E1AD1089889E0192E12D038694FF6FF71C0F62E
:204780001051884209D06FF07241884205D04FF6FF71C0F6205188420CD1182E0AD1059526
:2047A00073E0079870E041F2E300CFF62E6040EA062057E0182E0BD8304625F05BF941F688
:2047C000FD71CEF2023101F5964141EA005006901B2E06D01A2E0DD141F6FD70CEF20230BF
:2047E00039E07869D8B141F6FD70CEF2023000F5801030E01B2E10D978690028CFD0A6F19A
:204800001C000428CBD8DFE800F00311161B220041F6FD70CEF2023016E006981CE041F632
:20482000FD70CEF2023000F5001014E041F6FD70CEF282300FE041F6FD70CEF28230D6E748
:2048400041F6FD70CEF2823000F5401003E046F6FD20CEF2D230069015F0AEFC42F6126010
:20486000C0F2FB3000F086F8009405A8012101221423FFF78DFE01283FD11B2E0DD178696E
:2048800018B90598000400BF059005984AF8040BB9F101097FF464AF34E012980028F4D080
:2048A000132EF2D1CDE90045384644F60011C0F20801012204ABFFF72FFD01281DD19DF8D5
:2048C00010008007E1D505980138059047F2FD31C0F2090141EA006015F06EFC0598000A5C
:2048E00000F1385015F068FC40F2F530C0F20330043000F03FF80028C7D54FF0FF3009B054
:20490000BDE8F08FB8F1000F1AD041F6FB60C4F2840015F051FC4FF60800C0F21200039906
:2049200040EA016015F048FC0398000A00F1385015F042FC40F2F530C0F2033000F01AF804
:20494000089841F2FB2141EA004015F035FCBDF8220040F0085040F47B0015F02DFC0798EC
:2049600015F02AFC4FF22E40C0F2033000F002F80020C4E7F0B583B08E218DF807108DF81B
:204980000800010E8DF80B10010C8DF80A10000A8DF809000DF1070001AA052101231DF015
:2049A0001DFC012812D165260DF1070401AD00BFBDF8040000070CD5013E27D0204605216E
:2049C0002A4601231DF00AFC0128F1D06FF0010020E0C6208DF8070041F28006C1F20806FA
:2049E0000DF10704306A00F5FA7701AD204601212A4602231DF0F2FB0228E7D1BDF804004E
:204A0000400706D5306A381A0028EFDC6FF0020000E0002003B0F0BD2DE9F04F8FB01446E6
:204A2000B2F5037F02DAA4F5037056E38946054608464FF4037107F0E1FB2946687A11F8E0
:204A4000082F42EA00208A78C97842EA012140EA014049464FEA102A41F8040F4FEA104BF5
:204A60002A682B7B002B64D04FF6FE73C0F613539A4216DD4FF6FE73C0F616539A4227DD49
:204A80004FF6FE73C0F630539A4243DC4FF6FF73C0F616539A4249D04FF6FF73C0F617538A
:204AA00042E04FF6FE73C0F60C539A4221DC4FF6FF73C0F609539A4238D04FF6FF73C0F616
:204AC0000A539A4232D04FF6FF73C0F60B532BE04FF6FF73C0F613539A4227D04FF6FF7368
:204AE000C0F614539A4221D04FF6FF73C0F615531AE04FF6FF73C0F60C539A4216D04FF62A
:204B0000FF73C0F60D539A4210D04FF6FF73C0F60E5309E04FF6FF73C0F631539A4205D0F8
:204B20004FF6FF73C0F630539A4202D10123C9F80832C9F8A82100228DF83820CDE90C224A
:204B400009F50373CDE905130892A4F50371CDE90A3121EAE17103EB510207924908C9002A
:204B60000991C0F1020000F007074FF0FF3000FA07F65020B84060EA060107F1080505AC16
:204B800020462A461DF08BFBC9F8D00109F5B671204625F0B1FA8820B84060EA0601204678
:204BA0002A461DF07CFB09F5BC71204625F0A4FA8A20B84060EA060120462A461DF06FFB7D
:204BC00009F5C271204625F097FA2046022108221DF065FB09F59E71204625F08DFA204603
:204BE00000210122032316F02BFD5FFA8BF5EE4356FA8AF7C7F1050000F00700C11920464E
:204C000000F02AFF09F59271204625F075FA204600210022082316F013FD09F5C871204609
:204C200025F06AFA2046862108221DF038FB09F1C401204625F060FA204600210122012322
:204C400016F0FEFC204600210022012316F0F8FC204600210022012316F0F2FC20463946E7
:204C600000F0FAFE65B105AC2046294600F0F4FE8046204600210122012316F0E1FC06E071
:204C800005A800210122012316F0DAFC80465FFA8AF0049005AC204600210022012316F072
:204CA000CFFC204600210122012316F0C9FC204600210122012316F0C3FC09F5CE7120465A
:204CC00025F01AFAC9F8E881CAF1000000F00701204600F0C1FE2046394600F0BDFE5FEAE0
:204CE0000B60CDE901600ED005F11F0105AC204600F0B2FEC9F8D401204600210122012323
:204D000016F09EFC08E005A800214FF00042202316F096FCC9F8D401039705AE0024304664
:204D200000210122012316F08BFC09F59871304625F0E2F9304600210122082316F080FCAA
:204D400030464FF4487100F087FE30460021D022082316F075FC09F5A471304625F0CCF9DE
:204D60003046882108221DF09AFA0DF1340A304651462022002324F03DFFC9F8D80130463B
:204D800000210122032316F05BFC049800F11E01304600F061FEC9F8DC010898C0F10400E8
:204DA00000F00701304600F057FE304600210D22042316F045FC09F5AA71304625F09CF9D3
:204DC000304651462122002324F014FFC9F8E00109F5B071304625F08FF93046892108221B
:204DE0001DF05DFA304651462122012324F002FFC9F8B80109F14001304625F07DF930469A
:204E0000402108221DF04BFA09F1A001304625F073F93046502108221DF041FA09F58C71CF
:204E2000304625F069F900BF304651462122002324F0E0FE24B1012C08BFA0EB080B00E01A
:204E400080460134102CEFD109F14C0105AC204625F052F9C9E97B8B2046882108221DF09F
:204E60001EFA0DAE0027204631462022002324F0C1FEC9F8F40120468A2108221DF00FFA1C
:204E800080208DF83700204631462022002324F0B1FEC9F8F8012046502108221DF0FFF9F1
:204EA00009F13401204625F027F900BF204631462022002324F09EFE27B1012F08BFA0EB1D
:204EC000080B00E080460137102FEFD109F11C0605AC2046314625F00FF9C9E97F8B09F165
:204EE0002801204632461DF026FD2046A12108221DF0D5F90DAE204631462022002324F03D
:204F000079FEC9F8AC0109F19401204625F0F4F82046302108221DF0C2F909F1AC01204600
:204F200025F0EAF82046202108221DF0B8F909F1B801204625F0E0F82046A62108221DF081
:204F4000AEF909F1D001204625F0D6F82046A42108221DF0A4F909F58071204625F0CCF869
:204F60002046A02108221DF09AF909F58671204625F0C2F8204631462022012324F03AFE87
:204F8000C9F8C40109F1DC01204625F0B5F8204631462122012324F02DFEC9F8C80109F185
:204FA000E801204625F0A8F8204600210122032316F046FB039801280CDB01980499461897
:204FC00005AC00BF204600210022012316F038FB013EF7D1029898B105AC20460021002217
:204FE000202316F02DFB0646013DB5FA85F0420920460021012316F023FB002DF4D107E09F
:2050000005A800214FF00042202316F019FB064605AC0025204600210622032316F010FBDC
:20502000C9F8CC6109F1F401204625F065F88DF837502046AC2108221DF031F90DAD2046FB
:2050400029462122002324F0D5FDC9F8B00109F16401204625F050F82046AD2108221DF096
:205060001EF9204629462122002324F0C3FD09F17001204625F040F82046A82108221DF086
:205080000EF9204629462022012324F0B3FDC9F8B40109F17C01204625F02EF82046A9214C
:2050A00008221DF0FCF8204629462022012324F0A1FD09F18801204625F01EF8DDE90A10E4
:2050C0000C9AC9F80010A0EB420001EB4201494201F003010228C8BF401A0FB0BDE8F08FEF
:2050E0002DE9F84F1E469146884605460368D0F83C01D5E950121DF0BFF80A9F284641460D
:205100003A4600F051F88046002844BF4046BDE8F88F012000FA07FB05F5B67A0024CDF803
:2051200000903A463019022A08BF10F003010DD0375D012A0BDB417847EA012707D08178BB
:20514000C07847EA014141EA006700E03759D5F8D001C21C2846514615F046FB002848BFAC
:20516000BDE8F88F28463946424600F087F8002816D45C44B9F101090A9AD3D1D5F8D001D3
:20518000C21C2846514615F02FFB002808D42B6805F59E7207CA1DF06FF80098BDE8F88F53
:2051A0004FF0FF30BDE8F88F2DE9F8439046894604460368D0F89400D4E926121DF05CF8F8
:2051C0002768D4F8AC11384626F0F6F941F28002C1F208020146126AC0070FD1D4F8040286
:2051E000101A652840F20100C8F2000044DB11F0C00F1CBFC4F80422BDE8F88304F5AA722A
:2052000007CA3B4624F0E4FC2368D4E97601091A103100271A4600BFC60800F00705965D22
:20522000EE40F60708D002EBD0024819FF074FF00107F1D0002700E0012704F5BC7207CA16
:2052400024F0C6FC204649463A4600F017F8002848BFBDE8F883236804F5C27207CA24F018
:20526000B7FC4FEA887120463A4600F007F80028B8BF4FF0FF373846BDE8F883F8B51546BA
:205280000446D0F83001D4F8D42124F09BFC236804F5927207CA24F09BFC23686426182707
:2052A00004F5C87207CA24F093FC236823F0030017EAC302016806D0D14082F01F02406855
:2052C000400090400143C8B2FF2805D0013E04BF4FF0FF30F8BDE3E704F5987207CA24F02D
:2052E00077FC2DB1236804F5A47207CA24F070FC0020F8BD2DE9F0471E4690468946D0E98E
:205300007B4A00276FF00F05E00804F0070119F80000C840C00706D0611C484626F04CF92E
:2053200048F8040B013754440135EDD34EB1D6E9020100EB8700B060884202D33168304667
:2053400088473846BDE8F0872DE9F04F87B09A469346884611F00306DDE91057059023D012
:2053600000210DF11809CDE9009128F003010422534624F04BFC044617B1069800BA069070
:2053800009EB0601C6F104065E4588BF5E462846324606F00DFF042C40F080803544B0440E
:2053A000ABEB0609059800E0D94639F00302069258D00021CDE903A5CDE900514146534618
:2053C00024F024FC8246002F41D02C46A80706980DD00021B1EB900F39D08008294600BFDA
:2053E0000A6812BA013841F8042BF9D12FE018F0010118BF0134461A08EB0100800707D528
:20540000022E05D32078617860702170023E02342546042E0FD300BF20461EF071FDE870C4
:20542000010AA970010C000E697005F8040B043E0434032EF0D8012E06D92078617868707E
:2054400005F8021B023E02340EB1207828700698824523D1A9EB0009DDE903A5054480445C
:20546000119F0598B9F1000F1AD0002206A9CDE9001241460422534624F0C8FB824617B1F6
:20548000069800BA069006A928464A4606F090FEBAF1040F18BF4FF0FF3B01E04FF0FF3B85
:2054A000584607B0BDE8F08F2DE9F04FADF6442D0DAE45F60071C1F6002130464FF4807220
:2054C00006F07CFE002100BF705CFE2902D80131FF28F9D045F60061C1F600210027096881
:2054E0008DF810100A0E8DF813200A0C8DF812200A0A8DF81120FF283A4608BF023A0131C4
:205500000129914698BF6FF00209FF2808BF914604A8043020211FF0F1FA002800F1EF8061
:20552000054609F008F952AC20461FF05BFE52982A1D036904A92046984752984DA943693F
:20554000204614229847529881692046884709F0F2F80DF67C10CDF874094AF24870C1F668
:205560000120CDF86C09CDF87879CDF87079CDF88049CDF884494FF40270CDF87C09042128
:2055800004F502702060013901290446F8D8002404600DF66C15CDF8A0590DF51A60043028
:2055A000142106F02BFECDF888590DF688100430142106F023FE4BF27C50C1F6012007F0FE
:2055C00035FD00F1060ABAF1100F2746C0F0A280CDF8B049CDF8AC490DF51A6040211FF02B
:2055E000B9FD0746002800F18D804FEADA00039006F1FC0B6FF0030800260DF51A6500BF0E
:205600005BF8040902BA28463146F3F7D1FF013608F10408B8F1FC0FF2D3002F4BF27C55DD
:20562000C1F601256ED40DF688100DF51A6108F01EF9002865D405F118010DF688100DF616
:205640006C132A46F4F7C8F800285AD40DF51A60DDF80CB059461FF07DFDBBF1000F28D072
:20566000DDF8A409584400215D460023DDF894798F4286BFDDF88C79FF580027042D2A4634
:2056800028BF0422561E032E0ED8DFE806F00B08050200F8017D3F0A00F8017D3F0A00F825
:2056A000017D3F0A00F8017D0131043D04335B45DCD3DDF8A4594BF27C50C1F6012007F00A
:2056C000B5FCBAF1D00F18D30BEB050111F8011CBC2912D1DDF88C79461E384629465A46EF
:2056E00006F066FD2AF00700801B41F6D371C1F60321095C3878014218D0002702E0FC43B7
:205700000FE007460DF51A6008F07BF80DF6881008F077F8002FC8BF0124B9F1000F18BFF9
:205720004C4620460DF6442DBDE8F08FCDE90017BBF1150807EB0800029042D000250DF57E
:205740001D660DF6B817DDF804A028BACDF8CC0930461FF047FDDDF8D0090299036930460B
:2057600014229847DDF8D0090DF6CC110369304604229847DDF8D00939464369304614221A
:205780009847DDF8D009816930468847B8F1140F04D2B8F1000F14D0002003E0A8F114005F
:2057A0004FF014080135394611F8012B9AF800305A40B8F101080AF8012BF5D100288046B4
:2057C000C3D1DDE9000280F0FF00117801401170BBF11A000CD000298FD1ABF11B0101329D
:2057E000002729B1013912F8013B002BF9D089E7019F385C01287FF480AFABF119060DF508
:205800001D6528461FF0EEFCDDF8D00942F256210369C1F60421284608229847DDF8D009D9
:205820004DA90369284614229847DDF8D009B9190369284604229847DDF8D0090DF6B816A5
:2058400043692846314614229847DDF8D00981692846884730460299142226F053FD0546D5
:205860003846594606F0CAFCB5FA85F0470949E770B5A0B1044643F65915C1F208054BF247
:20588000AC56C1F6012600BF287800EB4000012256F82010002015F039FD013CF4D170BD73
:2058A00038B543F64405C1F208052B68002B3CD043F62340C1F2080000780A2833D8DFE81C
:2058C00000F01B0632320635321B3232060043F24470C1F2080043F24071C1F208010268B1
:2058E000096843F2487043F63464C1F20804C1F208002468006814E043F24470C1F2080073
:2059000043F24071C1F208010268096843F2487C43F63460C1F20800C1F2080C0468DCF882
:2059200000006468A0470020286038BD43F24470C1F2080043F24871026843F63460C1F29B
:205940000800C1F208010468086864680021E9E72DE9F84F99B316460F46834643F6440545
:20596000C1F2080523B1286810B90120FFF780FF43F6591AC1F2080A4BF2AC51C1F6012120
:205980009AF8000000EB400001EB800043F2FE52C1F20802816814880320042215F0B6FC17
:2059A000A01BC21B11D043F66C10C1F208000078012807D10020002115F0A8FC05E04FF077
:2059C000000846E0104615F023FDD5F80080012F18DB01244FF00009781E04FA00F100209C
:2059E000092FB8BFC8B2002E18BF4846082F3D46A8BF08251BF8011B2A4615F087FC7F1BDC
:205A0000002FE9DCBEB143F67010C1F208000078012806D1701E012101FA00F010213246F3
:205A200007E0022E02DB701E15F0F2FC01200121012215F06BFC9AF8000000EB40004BF225
:205A4000AC51C1F60121012251F82010012015F05DFC4046BDE8F88F70B5C56851B10C46FD
:205A6000064600BF304600210022012315F0E8FD013CF7D1284670BD38B50D4604460829F9
:205A80000CDB00BF2046FF210022082315F0D8FDA5F108000F2D0546F4DC00E02846012847
:205AA000B8BF38BD451C00BF204601210022012315F0C6FD013D012DF6DC38BD38B543F26F
:205AC000D050C1F2080008F07DFE43F26C70C1F2080000240068002528B1D0E900108D428A
:205AE00038BF0D46F8E743F2D050C1F2080008F0A7FEB5F1080038BF204638BD38B50C4691
:205B0000054643F2D050C1F2080008F05BFE43F26C70C1F20800006888B105F10F0121F055
:205B2000070143F26C72C1F2080200BF03688B4207D80DD0024652F8040F0028F6D1002422
:205B40000CE05B1A43504318136042685A6001E043681360C0E9001400F1080443F2D05011
:205B6000C1F2080008F06CFE204638BD0022C0E9001243F26C72C1F20802116831B343F26E
:205B80006C72C1F20802814202D9134606E000BF0B4653F8041F09B18142F9D941601860A7
:205BA0001068A0B1014651F8042F82B1D0F800C00CEB0003934207D1D2E900320A6003EBB2
:205BC0000C010160EEE700BF1046EBE71060704770B582B00B2501AC43F6AA66C1F2080636
:205BE0000A21224619F022FD9DF8041030317155013DF5D202B070BD2DE9F0479EB00DF19D
:205C0000070001211CF0A6FF9DF80700112800F22481DFE810F0120015001B0022012201EF
:205C20001D002A002C0022016700810099009D00A100A300AE00CB00CF0043F6E67001E0B4
:205C400006F0EAF9009024F0C9FA06E10220AEE0052024F05BFB002800F1FF8040F6971069
:205C6000C1F6042024F072FBF7E0062071E002A808211CF06FFF43F22C34C1F20804DDE913
:205C80000267A56C002F41F28008C1F208081ABFD8F8200000EB07094FF00009206C811CA8
:205CA0002164295A01F01F004AF2C87AC1F6012A5AF8202020469047002840F0BD8016B141
:205CC000013E01D1B7E000262FB1D8F82000B9EB000000F1B080206C811C2164295A01F03F
:205CE0001F00E5E702AC20460C211CF033FF201D04211CF092FE43F22C31C1F20801886CFA
:205D0000002800F08A804B6DDDE902218F189F4200F2848010449EE002AC20460C211CF023
:205D200019FF43F22C31C1F20801886C002879D04B6DDDE902218F189F4274D80434104497
:205D400024F034FA204674E00B2024F0DFFA84E00C2024F051FB80E00D2028E068460421D7
:205D60001CF0F8FE00991F293AD802A824F01EFA3CE00AA808211CF0EDFE0A9800EBC0001D
:205D800042F66471C1F2080101EB800080690B994269914239D2026983188058184424F06A
:205DA00005FA0B98002833D4002033E0102017F063FA52E00AA80C211CF0CCFEDDE90A0292
:205DC00000EBC00042F66471C1F2080101EB80000C998069104424F0E9F90C98C01719E097
:205DE000084617F033FA00208DF8080002A824F0ADFA0A9043F22C30C1F20800D0E90F0160
:205E0000CDE90B100AA80C2125E0084617F01EFA4FF0FF30029002A80BE00399084617F0DA
:205E2000C9F91AE00399084617F010FA00200090684604210FE000200B904C200A900AACC2
:205E400004F1080043F22C31C1F20801482206F0B5F9204650211CF0E0FD1EB0BDE8F0873F
:205E60002DE9F04F00EBC00042F66473C1F2080303EB800C1CF8200F00286AD18E46D16828
:205E80000EEBC10303F1200431B30026002500BF23783BB1671C0023F85C01330028FBD196
:205EA00001E000BF0023581C23181C46871914F8010B40B158783C180344A71C13F8020F1B
:205EC0000028F7D15C1C01357E1C8D42E0D116F003001CBF201A041D9069B8B304EBC008B0
:205EE00000214BF2C85AC1F6012A894654F8390008EB000B002600BF0AEBC6005F464568FC
:205F000015F8013B17F8010B08B19842F8D0984208D001360C2E04BF6FF00700BDE8F08F52
:205F2000EAE700BF106904EBC90370445B68C718C55C05F070058335C554BE70300AF8701B
:205F4000797009F1010990698145CFD301208CF800000020BDE8F08FF0B5036844F250373D
:205F6000C3F25627BB421DD1D0F80CE0BEF1010F15DB203000EBCE0C002300BF0468644496
:205F80000D4600BF15F8016B14F8017B0FB1B742F8D0B74217D0013308307345EED14FF06B
:205FA000FF3012E040F69710C1F6042010F8013B11F8017B0FB19F42F8D0F81A18BF4FF0AE
:205FC000FF30042101E04168002002B11160F0BD2DE9F8430068411E0020212988BFBDE884
:205FE000F883DFE801F011161B20252A737C8A8E92969F7171717171717171A37171717100
:20600000717171717171AAB143F67000C1F2080097E043F6B000C1F2080092E043F67400E1
:20602000C1F208008DE043F6B400C1F2080088E043F67800C1F2080083E0002403200021F1
:20604000042215F063F943F64400C1F2080043F200010568C0F225510020202215F056F900
:2060600040F27F2015F0D4F901200121012215F04DF901200021012215F048F90C3543F2AB
:206080004478C1F2080845F2532900BF2E19F710FFF706FCD8F8000000EBE601C05D4A7848
:2060A00040EA022016F007021EBF8978C0EA0140D04080B2484504BF2046BDE8F88301346F
:2060C0004FF420708442E1D1BDE8F88343F62740C1F20800007880F00100BDE8F88343F2BC
:2060E000E070C1F2080044F6D351C1F262010068A0FB01018809BDE8F88324F0FBFEBDE8B9
:20610000F8831DF074FDBDE8F88324F0D7FEBDE8F88346F20010C4F20F000068C0F3002015
:20612000BDE8F88306F04BFBBDE8F88343F62340C1F208000078BDE8F88343F2B070C1F2EC
:2061400008000068BDE8F88343F22C30C1F20800806C0088BDE8F8832DE9F04143F66C10D3
:20616000C1F208000078012840D143F2E070C1F208004FF61844C0F2E7340068A04240F08A
:20618000DD801CF077FB43F62345C1F2080541F28831287818F028FC1F200021062215F07E
:2061A000B5F803200021042215F0B0F810201021052215F0ABF81F200021062215F0A6F8C0
:2061C00003200021042215F0A1F810201021052215F09CF801200021022215F097F81CF090
:2061E00049FB2878214618F0FFFBCEE043F62340C1F208000078072840F0C280FFF750FBF3
:2062000043F63467C1F208073868D0E9070580474AF23060C1F60120386043F2E070C1F248
:20622000080044F6D351C1F262010068A0FB010140F2FF1000EB9110400A642100FB01F84D
:20624000002600BFB8F1080F444628BF08244FF0FF300021224615F059F82644652E02D3DD
:20626000FFF71EFB0026B8EB0408EBD100200021012215F04BF8FFF713FB24F0A9FD0120F3
:2062800008F04AFB24F0D8FD012008F045FB24F0EBFD012008F040FB032400BF1DF07BFCC5
:2062A000012008F039FB24F0C7FD012008F034FB013CF3D100200021042215F027F80020C5
:2062C0000021042215F022F800200021182215F01DF8FFF7E5FAA8476FF001040D2000214D
:2062E000052215F013F80134F8D319200021062215F00CF80120012118F0C0FD0320092187
:2063000018F0BCFDFFF7CCFAA8474AF20C60C1F6012038600720002118F0B0FD00200021BB
:20632000012214F0F3FFFFF7BBFAA8471B200021062214F0EBFFFFF7B3FA26E01F2000212F
:20634000062214F0E3FF03200021042214F0DEFF10201021052214F0D9FF1F2000210622F8
:2063600014F0D4FF03200021042214F0CFFF10201021052214F0CAFF01200021022202E06D
:206380001F200021062214F0C1FFFFF789FA0020BDE8F08180B50068002243F61B4CC1F2F0
:2063A000080C0121C0F200111CF80230062B04D00132082AF8D14FF08071002201F0B8FA76
:2063C000002008BD70B543F64002C1F2080246681268002A32460BD000680C18354600BF10
:2063E0002046294618F0AAFE2D1A0444F8D10022B01A70BDF0B5026801251324C0F2800405
:206400001378A3F10906172E05D805FA06F6264201D00132F4E74FF0000C1C4602EB0C0E36
:20642000A4F13005EDB20A2D0BD3A4F14105EDB21A2D06D3E5B25F2D03D0613CE4B21A2CD5
:2064400004D29EF801400CF1010CE7E70C7834B14E1C0025775D0135002FFBD100E00025B5
:20646000654519D1BCF1000F18D00125A3F16106F6B21A2E38BF203BDBB2A4F16106F6B250
:206480001A2E38BF203CE4B29C4205D1AC4505D0535D4C5D0135E9E70120F0BDC0F800E08C
:2064A0000020F0BD70B582B0144643F62342C1F2080205461078012804D070B981B11DF0CB
:2064C000BDFB0FE0002914BF45F004002846214602B0BDE8704001F09DB86FF0010426E054
:2064E0001DF0B9FB600F8DF80700600D8DF80600600B8DF8050060098DF80400E00040EAF7
:2065000045008DF8030000240DF1030528461CF005FA06460820FFF7ABF930461CF0CCF9B6
:20652000C00704D00134652CF0D14FF0FF34204602B070BDF8B50C46054600260F4600BFFE
:2065400055F82610002C224618BF3A46304624F0BFF904370136082EF2D1F8BDF8B5144664
:206560000D460646D0E90110C243521804D4A242B8BF1446F16804E0F1680A44A242B8BF77
:206580001446326811440F1ABC42B8BF274629463A4605F00DFE3268D6E902013844531875
:2065A000834208BF1046B060E41B3D44EAD1F8BD2DE9F04786B0002943F64801C1F208010F
:2065C0000446086840F00100086001D0182104E06846182105F012FE082168461CF0BAFAF7
:2065E00042F6082AC1F2080AA4EB0A0904F10808002600BFB14517D00AEB0600056B9DB14A
:20660000296889B12F697FB15AF80610226891420AD101792279914206D1083041460422A3
:2066200025F070FE002845D04436B6F5AA7FE1D1256B286940B11CF0B2F928681CF0AFF98D
:206640002846242105F0DAFD019800EB4000C60030461CF091F92860E8B1314605F0CEFDCD
:20666000FFF72CFA4CF6CD41CCF6CC41A0FB01018E0830461CF080F960B19DE88C0000216E
:2066800085F82010C5E90132C5E90370C5E90500EE6109E0286808B11CF081F9206B2421C1
:2066A00005F0ACFD6FF00101084623F097FD06B0BDE8F08738461CF072F94FF00009C5F81A
:2066C0001090286818B11CF06AF9C5F800902846242105F093FDABE72DE9F04F89B01D464A
:2066E000CDE901208946064640F2080AC2F2000A002400BF304621462A46012300F016F953
:206700000746CDE9045401192A1A3046002300F00DF90028394618BF0839082FD8BF394625
:206720000391002900F098808B46083918BF01210022082FC8BF0122B0FA80F040091043D0
:2067400040EA01000CBF25210021CDE9060160B9A01CC11000F0070019F8011021FA00F055
:20676000C007079808BF032007904FF0000800BF4FF0010C43F6DB36C1F20806BBF1190F01
:206780005846A8BF10200022012815DB002141F2C805C1F2080500BF6318DF1003F0070382
:2067A00019F8077027FA03F303F001038B401A4301318842F0D103E041F2C805C1F20805BB
:2067C000012181F31088069B002B00F00101014404BFDDF81C8002310023CAF8043008AB55
:2067E000CAE90236CAE904180892BFF35F8FCAF800C0ABEB000B00BFDAF800100029FBD1EC
:20680000002181F31088B8F1000F1DD0317819291AD80021C5E9001172185278531F142BE4
:206820000CD80C2A07D301F00702CB080CFA02F2EF5C3A43EA5401314029EDD143F6E4021F
:20684000C1F2080200211160BBF1000F04D00444022005F0E6FE8BE7DDE90454DDE902605F
:2068600004442D1A304621462A46002300F05EF8002855D043F6E401C1F2080104950F689C
:2068800041F2C801C1F2080101EBD702019901EBD40312F8011BCDE9054707F0070721FAD6
:2068A00007FE04F00701C7F10807079005464FF0FF3000BF00FA01F66C1800FA04F404F5A1
:2068C0008078F443C1F1080CAC4584BF68EA0604AC461E7812F8018B04EA060B08FA07F617
:2068E00046EA0E0606FA01F1A14341EA0B0103F8011B26FA0CFEA7EB0C0101F10807002145
:20690000B5EB0C05D6D1DDE9061043F6E402C1F2080201441160DDE904542D1A0444029E64
:20692000002D7FF4E7AE09B0BDE8F08F10B5012ABCBF002010BD8446002000BF01EB000E4A
:206940004FEAEE040EF0070E1CF8044024FA0EF404F001049C4218BF10BD01308242EDD153
:20696000104610BD2DE9F04F99B014468B4600211191042813D8CDF83CB0DFE810F00500D4
:2069800017004B00710019011F20129043F62C60C1F208000068426912A800F00ABC4FF6E1
:2069A000FA60CFF6FF70119000F007BC4FF0FF3043F62C6AC1F2080A1890DAF80000082150
:2069C000426812A890479DF848009DF849109DF84A209DF84B309DF84C6040EA012040EAEC
:2069E000024040EA0363D81DC208251FABF1080806F00300C6F34117032800F0B181022895
:206A000040F01282002F00F0FF81012F40F00C820820FBE14FF0FF3043F62C65C1F2080529
:206A2000189028681821426812A890479DF848009DF8491040EA01209DF84A1040EA01403A
:206A40009DF84B1040EA0160C71DFE08042CABF1180940F0EC80286881684846884794E1FD
:206A600043F2A055C1F208052868002800F0518168685845C0F09581A2462868594623F055
:206A8000C9FB0020E86043F62C66C1F208064BF2B871C1F60121316043F28468C1F208088A
:206AA00042F2C854C1F208040DF1480998F80110C1EBC10104EBC1010A695AB1496900295F
:206AC000ABEB0101A9600BD00A1AFF2AEEDD002707E000BFC5F808B00127594601E000BF79
:206AE0000127091A0C2931D330680C214268484690479DF84C009DF84D1040EA01209DF88B
:206B00004E1040EA01409DF84F1040EA0161D5E90220121A8A4217D39DF849009DF8502087
:206B20009DF8513042EA03229DF8523042EA03429DF8533042EA0362FFF714FFD5E90210E4
:206B4000091A0B29D0D801E00C38E860B0EB0B0118BF0121FA430A42A8D14FF00009CDF81A
:206B6000609030680421426918A8904743F29055C1F20805A96821B128681BF0B0FFC5F862
:206B8000089023F031FB4BF2D870C1F60120306043F2A050C1F20800002123F051FF43F298
:206BA0009050C1F20800002123F04AFF544602E343F62C68C1F208080821D8F8000042680B
:206BC00012A890479DF848009DF849109DF84A209DF84B309DF84C509DF84D609DF84E7084
:206BE0009DF84F9040EA012040EA024040EA036143F2A050C1F2080023F022FF18900028F8
:206C0000C0F2A18045EA062040EA074040EA096143F29050C1F2080023F012FF1890002883
:206C200080F29B8043F2A050C1F208008FE09DF85D0010909DF85C000E909DF85E000C90C8
:206C40009DF85F0008909DF859000D909DF8580003909DF85A00CDE90A409DF85B00079027
:206C60009DF8550002909DF854809DF8560005909DF8570006909DF851A09DF850B09DF87D
:206C800052409DF8530004909DF84C500996B9F1000F484618BF012006FA00F0FF304FF673
:206CA0000071C7F6FF7110EA010608BF4FF4807630461BF061FE002858D00146CDE9007197
:206CC00010980E9A42EA00270D98039A42EA0022029848EA00284BEA0A2040EA044405F0C7
:206CE00010000E90B9F1000F2B4665D043F62C60C1F208000D4600689246426808464946ED
:206D00009946904752464B4605EB560010900D9555E043F2A050C1F208004FF4405123F010
:206D20008FFE002836D443F29050C1F208004FF4007123F085FE00287FF59AAE43F2A05071
:206D4000C1F208002AE043F29050C1F20800002123F076FE6FF483701890D8F8000026E220
:206D6000002F5AD0012F5FD1082058E043F62C65C1F2080528688168484688476FF4837044
:206D80001890DDF83CB0DDE9096428688169304688470BE243F29050C1F20800002123F0A7
:206DA0004FFE584616F052FA201F16F003FA6FF4837023F013FAFEE100200D901091DDE9DB
:206DC0000B1047EA004042EA0141DDE9046248EA024244EA0669C3F341160C9603F00305D0
:206DE0000E9E7EB9032D009F00F01B81022D40F030810C9E002E00F01A81012E40F01F81E3
:206E0000082616E1009F24E14FF4807046F20021C4F20F01C1F8800006E04FF4807046F2CD
:206E20000021C4F20F0108600D9255EA080000F0A6800C95FEF742FE0546DDF83490814587
:206E400038BF4D46B5F5807F98BF4FF480754FF60070C1F6FF70B5F5805F88BF0540284612
:206E60001BF08AFD002800F09B80CDE908670A94B8F1000F4446804618BF4FF000080C9ABE
:206E80000B94002A18BF0122002C214618BF0121114018BF00EB5508002C079018BF04464F
:206EA000002918BF6D08B9F1000F5ED02F4648460E9500BFB84238BF07463CB18146DAF84D
:206EC00000003946C268204690474846C01B10904FF0000BB4B100BFDAF800000068804754
:206EE000391AA1EB0B0108B1FF29F5DDFF290D46C8BF25F03F05002808BF0D4604EB0B005D
:206F000008E000BFA7EB0B05B5F5007F28BF4FF400750020B8F1000F43F63461C1F20801FE
:206F20004646096818BF5E44D1F80490EB0000213246C8472EB1DAF800002946C26930462A
:206F40009047AB44BB45C5D1B8F1000FDDF83CB007D000BFDAF800000069804718900028F4
:206F6000F8D110980E9F0028A4D1DDE90C5018904FF00009DDE90A4807AFC4CF15E043F6B5
:206F80003460C1F208004FF0000900680021D0F804C000200022E0470D981890002204E089
:206FA0006FF48370189000220C9D06F00C000C2806D0082819D147B1012F16D1082006E0C5
:206FC00067B1012F11D108200AE04FF4807046F20021C4F20F01C1F8800006E04FF48070D1
:206FE00046F20021C4F20F010860B9F1000F11D0B8F1000F06D0DAF800001646816848463D
:207000008847324635B1DAF8000081694846914688474A4612B110461BF0C1FCDAF8000010
:20702000C5E00C9E6EB1012E12D108260BE04FF4807646F20025C4F20F05C5F88060022593
:2070400007E04FF4807646F20025C4F20F052E6003250B95089E40EA066A079841EA006524
:20706000069842EA006B1098814403F00C0427F007071EF0CFFA80460E9858B943F6346025
:20708000C1F20800109A0068002146680D983B46B0474BE00B98032807D002281BD10C98AD
:2070A00048B1012817D1082007E00C9860B1012811D108200AE04FF4807046F20021C4F2A3
:2070C0000F01C1F8800006E04FF4807046F20021C4F20F01086043F63460C1F20800109A95
:2070E0000068002146680D983B46B0470C2C07D0082C1BD10C9848B1012817D1082007E050
:207100000C9860B1012811D108200AE04FF4807046F20021C4F20F01C1F8800006E04FF4E9
:20712000807046F20021C4F20F0108601EF072FAA0EB080648461CF0E3FE00EA0B00A8426B
:2071400004D05645FFF698AF4FF0FF36DDE90E0B43F62C65C1F2080518960999F0B90C2C76
:207160000C9806D0082C19D140B1012816D1082006E060B1012811D108200AE04FF4807007
:2071800046F20022C4F20F02C2F8800006E04FF4807046F20022C4F20F0210602868C2692F
:2071A0001098904701981BF0FAFB0A9C2868426918A804219047119898B143F62C69C1F2A7
:2071C0000809D9F80000816858468847D9F800008169201F8847D9F800000421426911A854
:2071E000904719B0BDE8F08FF8B591B30D4643F29057C1F208070446D7E90010BA68861ACD
:20720000AE4288BF2E4688182146324604F0D0FFD7E901013144B96081421AD138681BF0D8
:207220005EFC0020B860AD1B13D0344479688D4209D300BF20461BF052FC79680C446D1AD7
:207240008D42F7D22DB1386821462A4604F0B0FFBD60F8BD70B588B004466D4628462021C3
:2072600004F0CCFF2026202C38BF264628463146FFF7BAFFA41BF5D108B070BDF8B543F27A
:207280006C50C1F2080043F64801C1F2080100220B6843F008030B6043F67C17C1F208076D
:2072A0004FF6FF743B780121002B18BFC0F20F044AF65015C0F2AB051EBF30214AF6000500
:2072C000C5F2D455C0E90051C0E902420261284618F0ACF943F6CC56C1F20806B169814270
:2072E00088BFB06128462146002218F09FF9B169814238BFB061306838B1D6E90312914292
:2073000020D01BF04CFB00203060306960B9FEF7D5FBA0F500706FF30800B0F5007FBCBFF6
:207320004FF0FF30F8BD30614CF2C661C1F6032122F00AFF3169F1600144C6E90001002836
:2073400000F0AA801DF0A8FB3168326943F68803C1F20803B069196043F68403C1F208039D
:207360004EF200141A6043F68003C1F20803CEF20004196043F67C01C1F208010A603978FB
:2073800001294AD19C21C4F2050140F60002C0F600120A6041F20851C4F205010A6842F0D9
:2073A00003020A600A68D207FCD042F20041C4F20501D1F8002142F00302C1F8002100BF5C
:2073C000D1F80021D207FBD046F2B801C4F208017222C1F85C2243F20411C4F205010A6D27
:2073E00002F0807282F0807282F480520A6000BF0A6DD204FCD541F20405C4F2080503278D
:20740000AF6005F006FB012068606F602860002084F818034FF080703BE09C21C4F20501AD
:2074200040F60002C0F600124A6041F20851C4F205018A6842F003028A6000BF8A68D207BD
:20744000FCD042F20041C4F205010A6842F003020A6000BF0A68D207FCD046F2B801C4F29F
:20746000080171220A6042F20405C4F208050327AF6005F0CEFA0020E860012169606F60EE
:207480002A6929604EF21941CEF2000108704FF0007020603068B0600020F8BD2DE9F84FF4
:2074A000044642F60820C1F20800A4EB000A42F66479C1F2080909F10C0841F2800BC1F276
:2074C000080B00BFFEF7FAFAB0F50076D8BF0026B0F5905FC8BF4FF480569EB1304642F2EC
:2074E0009A71C1F6042122F02FFEE8B30746E0693946C36A204632469847002822D538462F
:207500001BF04DFADBF820104FF0FF3000225346454600BF3BB135F8027C27B12F688F42CC
:20752000BCBF10463946443B24350132052AF1D1002819D400EBC00009EB80004089F7F714
:20754000EBFABFE7311A384622F012FE0020A0842062E0692761006830B14CF2D161C1F6AE
:20756000032122F0F1FD2062BDE8F88F43F6A000C1F2080001680029FCD04FF0FF30704722
:2075800043F6A000C1F2080001680029FCD04FF0FF30704743F6A000C1F2080001680029AE
:2075A000FCD04FF0FF30704743F6A000C1F2080001680029FCD04FF0FF307047F0B583B0EB
:2075C0000D4600248DF80B408DF80A408DF809408DF80840400001308DF807000DF10706F2
:2075E00030461BF09BF907460820FEF741F938461BF062F9C00705D00134652CF0D14FF08C
:20760000FF3404E01DB1F81C1BF056F92860204603B0F0BD2DE9F04F87B0002442F2D6729D
:20762000C1F604228DF80340105C8DF80200039181EA114080EA102080EA101080EA900044
:2076400080EA500000F001008DF8100041F28005C1F2080543F63466C1F20806286A00F15B
:2076600064070DF1020B43F6B769C1F208090DF1060A00BF30684946D0F804805846524601
:207680000D23C0479DF8070000F00700022804D1286A381A0128EDDA11E0012812D0042825
:2076A0001DD04FF0FF30012C29D843F62841C1F20801097819BB23F03DFC0134DAE76FF0ED
:2076C00001001CE0306843F61861476803A8C1F208010DF106022123B84700200FE030685D
:2076E00043F6D161476843F6C560C1F20800C1F208010DF116023023B8474FF0FF3007B00E
:20770000BDE8F08F2DE9F04F87B0009100238DF8153042F2DE71C1F60421002201928DF8A2
:207720000930085C8DF8080041F28004C1F2080443F63466C1F20806206A00F1640A0DF12E
:20774000080B43F6BE69C1F2080903AF30684946456858463A460D23A8479DF80D8008F015
:207760000700022805D1206AAAEB00000128EDDA13E0042814D0012823D04FF0FF30019DC8
:20778000012D30D843F62841C1F20801097851BB23F0D0FB01350195D8E76FF0010022E0FD
:2077A000306843F6D161476843F6C560C1F20800C1F208010DF116023023B8474FF0FF306C
:2077C00011E0306809F1020147680DF1110003AA2123B847009A2AB1C8F3C100039940EABE
:2077E00081001060002007B0BDE8F08F2DE9F04F85B000248DF80D409F218DF80C108DF837
:207800000B40FF218DF80A1041F28005C1F208050190286A00F1640943F63466C1F20806D1
:207820000DF10C080DF10A0B02AF00BF30685946D0F804A040463A460D23D0479DF8090025
:2078400000F00701022905D1286AA9EB00000128ECDA11E0012912D0042916D04FF0FF309C
:20786000012C22D843F62841C1F208010978E1B923F060FB0134D9E76FF0010015E0019916
:20788000C0F3C100086000200FE0306843F6D161476843F6C560C1F20800C1F208010DF178
:2078A0000E023023B8474FF0FF3005B0BDE8F08F2DE9F04F8BB0074600266D4643F6346993
:2078C000C1F2080943F65D6AC1F2080A43F63C6BC1F2080B01AC00BFF00703D023F04CFBE9
:2078E0000AE000BFD9F800005946D0F80480504622464FF48473C04700202946FFF702FF5E
:20790000009801466FF31F31A1F27742B2FA82F25209A1F6EB21B1FA81F1490951403143F8
:207920000126C907D8D007B138600BB0BDE8F08F2DE9F24F82B0904643F66111C1F20801B3
:207940008146087808B90120087043F64006C1F2080643F23C7A3068C1F2080A88B143F68C
:207960005515C1F2080500BF287818B1012006F0D3FFF9E7DAF8000008B1F1F737FA002028
:20798000306043F25855C1F20805B8F1000F286808BF4FF4807820B11BF001F800202861ED
:2079A00028604CF2E467C1F60327C3460BF10100394622F0C9FB2860ABF58071C34502D97E
:2079C00000288B46F2D001F2011043F23054C1F208042861206840B9812020614CF2F361B2
:2079E000C1F6032122F0B0FB2060FF21002743F61B43C1F20803FF2213F80780A8F1050B77
:207A0000BBF1020F38BF3946B1F1FF0B18BF4FF0010B08F0FD08B8F1040F08BF3A46B2F1C2
:207A2000FF0818BF4FF0010818EA0B0F03D1072F07F10107E0D143F28C73C1F208031960DE
:207A400043F28871C1F208010A604AF29451C1F60121CAF80010C4E901002A68C5E90122F5
:207A6000EA606FF00201CAB1C0B1306808B10138306043F61950C1F60320009043F6A54228
:207A8000C1F6032243F6D743C1F603234846029905F090F8306801303060002143F67E10F3
:207AA000C1F208000122027043F2FD50C1F2080000220270084603B0BDE8F08FF0B591B09A
:207AC00010A804211BF046F8109F6D463C4600BF402F3E4628BF40262846314622F066FB45
:207AE000A41B2846314617F029FB3F1AB04203D1002FEDD1002702E0204615F0A7FB1098ED
:207B0000C01B109022F06AFB11B0F0BD2DE9F8430646C06840B3894606F1240789CF716B28
:207B2000FD435C1948BF0C449442A8BF1446A0460844C51BA845B8BF4546384649462A4624
:207B400004F036FB2F44706A716B4218974208BF0746B8EB0508A944EAD1F762012C04DBD3
:207B6000304623F0C1FB00E000242046BDE8F8832DE9F047994617468A468046089DBDB104
:207B800041F28006C1F20806346A00BF404651463A464B461EF03AF910B3F6F7BDFA306A9E
:207BA000001BA842F2DD4FF0FF3720E0F6F7B4FA404651463A464B461EF028F90028F5D196
:207BC00002E000BFF6F7A8FA404608F0E4FC0028F8D10CE0316A091BA94207DCF6F79CFA2A
:207BE000404608F0D8FC0028F4D100203F1A3846BDE8F08770B582B043F2F054C1F20804A4
:207C000045F25530C5F24230206043F6D815C1F2080500262878009621460D220023FFF70E
:207C2000A7FF0D2818BF10F10100F3D102B070BD2DE9F041069CA4F1010C4FF0FF3E4FF0A7
:207C4000FF0800BFC2F1080551F8046B26FA05F5457096402F0CC7702F0A87700EFA02F79E
:207C60000478BC4334430679047008FA02F43440BCF1000F44EA1564047108BFBDE8F081FE
:207C80001A4400EBD20002F00702ACF1010CD9E730B500EBD10011F0070C11D061F0070175
:207CA0000B44FF2101FA0CF1047824EA010E12F8011B01FA0CF444EA0E0400F8014B00E03F
:207CC0000021082B39D3CCF1080EDC08202B27D312F8045B41EA052121FA0EF5090A00F865
:207CE000045B12F8035C41EA052121FA0EF500F8035C090A12F8025C41EA052121FA0EF50C
:207D000000F8025C0D0A12F8011C45EA012525FA0EF500F8015C043C032CD9D85CB100BF17
:207D200012F8015B41EA052121FA0EF5090A00F8015B013CF4D103F0070353B1127841EA4F
:207D40000221CCF10802D1404FF0FF329A409143017030BD40B1C10709D10021013142087C
:207D600080071046FAD503E04FF0FF3100E000210846704711F8012BA2F141031A2B38BFB7
:207D8000203210F8013BA3F1410CBCF11A0F38BF20330BB19342EDD0981A704700B549B3E4
:207DA000844600201CF801EBAEF13002D3B20A2B0FD3AEF16102D2B2052A03D8AEF15702E4
:207DC00007E000BFAEF14102D2B2052A08D8AEF137020301013953FA82F008BF00BDE1E767
:207DE00043F25C4CC1F2080C4FF6F861CFF6FF71CCF82C10002000BD70B504460026002575
:207E0000022E09D0A05D1CF03EF8A9B200EB011501360028F4DA0025A8B270BD70B543F28B
:207E20007424C1F20804206950B1606D002500BF46681AF0B4FD0135206985423046F7D381
:207E400000202061606570BD2DE9F04F9FB098468A46814613B10020C8F800004FF0FF3460
:207E6000002000BF19F800102E2901D009B902E004460130F6E7611C08BF0446071B09EB3A
:207E800004001CBF0130013F0D9012F0080005920E901FD10CB34FF0000B082CD8BF032FC0
:207EA0001DDC4D46264600BF15F8010B23F03EFC98B9013EF8D16FB10D9D3E4615F8010BE5
:207EC00023F034FCB0FA80F14FEA511B38B9013EF4D104E04FF0010B01E04FF0000B4FF011
:207EE000FF30402CD8BF402F02DD1FB0BDE8F08FBAF1000FCDF810A01CD0CDF8088043F272
:207F00007420C1F208000025D0F82C80B8F1010FC246D8BF4FF0010A12AE00BF2846314673
:207F200023F01AFC129840B10135AA45F6D10020039009E00020039029E0B8EB050018BFBA
:207F400028460390A8EB0500DDF8088043F27423C1F20803DDF810A0197D0AEB4122013AF3
:207F60004902B2FBF1F18842C0F234810191D86A451E1DAE2846314623F0EEFB1D9810B19D
:207F8000013DF7D103E00198281A01300390BBF1000F27D00E9800284FF020008DF8720083
:207FA00042F22000ADF870004FF02030CDE91A0055D1082C2246A8BF08221AAD28464946E2
:207FC000234600F053FA4FB1032F3A46A8BF032205F108000D993B4600F048FA1AA817F09D
:207FE0003BFD45E00220002F08BF012039190D1868001EAA1A2117F019FB1E99002943F2D9
:208000007421C1F2080118BF0130CA6806904FF6F071C0F2FF7111EA021B0E9500F0BC8090
:2080200000250026B24600BF4FF6FF70C0F27F0000EA1A10002100F0D3F9002800F0AD8023
:2080400005F4F071405CE52803D0002800F0A580013620350AF1010AD345E5D19DE00B2CF9
:208060002246A8BF0B221AA84946234600F0FEF9039FBDF87000ADF840009DF872008DF82B
:20808000420000250F95DDE91A9617F009FD0446C0F31610012100F0A3F9002855D004F040
:2080A0000F014A0100EB411400F80290300A60714FEA1960E0704FEA1940A0704FEA19207A
:2080C00060702046032200F8046F310EC170310C817004F1080010A904F06AF80F9804F88D
:2080E0000E0F04F80EAF4FEA1A61E1704FEA1A41A1704FEA1A216170452104F8031C7221A7
:2081000004F8041C04F8055C04F8065C04F8095C04F80A5C010E04F80B1C010C04F80C1C62
:20812000000A04F80D0C04F80F5C04F8105C059804F8110C380A04F8010C04F8027C380E90
:2081400004F8070C380C04F8080CBAF1000F21D043F27424C1F20804DDF80490E16A09EBDD
:208160000700884211DC4FF0FF353846216B05FA01F2461CB9F1010F314608BFD14323F051
:2081800097FAB9F101093046F0D1B8F1000F18BFC8F800700020A8E60026ABEB0600DDF85F
:2081A00018B0584516DD20208DF8720042F22000ADF870004FF02030CDE91A006CB1062C19
:2081C0002246A8BF06221AA84946234600F04EF90E9D04E04FF0FF3087E60E9D2846CDF86F
:2081E00008801AAC7E2121542044312141704FB1032F3A46A8BF032204F108000D993B4654
:2082000000F034F9204617F027FC0020002700BF215CFAB2FB0143EA52028F1801300B28FA
:20822000F6D109EB0500A0F1010912AC002500BF20461A21FF2203F0E2FF1E981E9500281A
:2082400008BF1A20211819F8012901F8015C01F8022C0238F6D1E079217A627A8DF8422074
:20826000BDF85420BDF8523043EA024240EA0120ADF840009DF84E000990BDF84C000890E8
:20828000BDF860000790BDF85E80DDF848A0BDF856000C909DF85800CDE90E029DF859009A
:2082A0000D90BDF85A000B90BDF85C000A9017F0F7FB06464FF6FF70C0F27F0000EA161092
:2082C000012100F08DF8002866D0DDE9082142EA0141079A48EA0248069A93455A4606F021
:2082E0000F034FEA431C08BF42F0400200EB431600F80C2071714FEA1A40F0704FEA1A20E9
:20830000B07086F801A032464FEA1A6002F8040F080CD070080A907006F1080010A90322A3
:2083200003F046FF0F9806F80E0F0A9A06F80E8F4FEA1861F1704FEA1841B1704FEA1821CC
:208340007170110A06F8031C06F8042C0B9A110A06F8051C06F8062C0C9A110A06F8091CE3
:2083600006F80A2C010E06F80B1C010C06F80C1C000A06F80D0C06F80F7C06F8105C0F201F
:2083800006F8110C06F8015C06F8025C0D9806F8070C0E9806F8080CBBF1010B7FF448AF7B
:2083A0009DF872008DF84200BDF87000ADF8400000250F95DDE91A9617F072FB04464FF6A3
:2083C000FF70C0F27F0000EA1410012100F008F80028DDF810A0DDE902877FF460AEB4E6C6
:2083E0002DE9F04743F27425C1F208050446E868A04238D9286959B3A04229D805F1540942
:2084000000274FF69D48C1F603284846BA4600BF0668B6B94FF40270414621F095FEB0B1BE
:20842000064604304FF4017103F0E8FE06F108003060002F484618BF381D0660286901308E
:2084400028610AF1010A301DA2453746E0D92869A04208D9686D14B1013C4068FCD110B1C2
:208460000068BDE8F0870020BDE8F0872DE9F84391460D4680465C1E002700BF15F8016B22
:20848000304623F053F910B908F8016B013714B1013C4F45F2D13846BDE8F8832DE9F04F4E
:2084A00089B043F27424C1F20804A06D08B11AF076FA206D18B11AF072FA00202065FFF750
:2084C000ADFC2046602103F099FE4020207545F245500221C4E90201052003220123002759
:2084E000C4E90F73C4E91112E0640C2040F2551245F24057C4E90831C4E90A72C4E90C03DB
:20850000FFF78CFCA06D08B11AF049FA606B400240F6DF11C1F6042121F016FEA065002869
:2085200000F0D880616B490203F068FE206B012505FA00F0A0F10801002023F0B9F8206BDA
:20854000A91E01FA00F0C143012023F0B1F843F28070C1F2080084F85D50076807F5806034
:20856000602103F04BFE1BF03CFD00284FF09A004FF6EB31C1F6032142F6E602C1F60422C0
:20858000C7F80024C7F80414C7F8080400F0A380D7F8F404002806DA411C00F0E78010F5BB
:2085A000807F40F3E380012607F58C606C2103F025FE4FF0000A40F6080502AC47F2017888
:2085C000C5F275380020019081462046294610221AF047F80298404508D047F20371C5F214
:2085E0007531884244D0002861D16BE00399BAEB513F67D10498BAEB503F63D1059A104452
:20860000BAEB503F5ED141F2FC70471A1D2F28BF1D27C34643F2807AC1F2080A09EBC908BE
:20862000DAF8000000EB880000F58C6001F604013A461AF016F8DAF800004FF0000A00EB7A
:208640008801D84601F58C6200EB061002F807A0C0F804A4C0F80024DDE90423C0F80834D0
:2086600002F60400C1F88004013609F101091EE00398BAEB503F25D10499BAEB513F21D1FF
:20868000059A1144BAEB513F1CD141F2FC710F1A0B2F28BF0B2700F604010DF1180B5846EE
:2086A0003A4619F0DEFF0BF807A001200190B9F1020FD8BF052E05DCB5F5FF5F05F110057F
:2086C0007FF683AF0198B8B106A843F27424C1F2080419E0FEE71B2042F6F201C1F6042197
:2086E0004FF68542C1F60322C7F81024C7F81414C7F81804022603E043F27424C1F2080446
:208700004FF69740C1F60320002128220023FFF79BFB43F28070C1F20800A663006800F503
:208720008061E161012E0FDB00F20C4555F80C0C38B155F8041C21222B46FFF785FB0028AD
:2087400002D41035013EF1D1012084F85C00E06804010025C5F316100021FFF741FE10B19D
:208760000135AC42F6D109B0BDE8F08F002940F6EC11C1F60421C7F810144FF6AF45C1F626
:2087800003250CD04BF66801C1F6012101F10802516831B152F8083B8342F9D102E029464E
:2087A00000E00021002943F6EC04C1F2080418BF0D46206840B940F6F511C1F60421802044
:2087C00021F0C2FC206040B14FF6C142C1F6032280212B461CF042FF256843F28070C1F271
:2087E00008000768C7F8145415F8010B28B10020295C01300029FBD100E00020C7F8180443
:208800000226D1E62DE9F04F85B01E4614460D4680460846092103F0F1FC0020E070A07040
:20882000607020700E9F06B130600FB100203860B8F1020F56DB43F2742AC1F2080A0020C9
:20884000DAF80C90B0EB091F42D083460021FFF7C7FD00283DD0CDE9014603954FEA091510
:20886000D94604AC4FF0FF3B09F00F0100EB4116F07A00F03F000F281AD03078C0B1E52885
:2088800016D0708BA0B100BF0746214622F064FF049840B1DAF830100BFA01F120EA01021B
:2088A000C9438A42F0D1474502DB708B40451CDD09F10109A9450FD0C9F316100021FFF773
:2088C0008FFD0028D0D1039D0E9F4FF0000B00E004E085F800B001E0039D0E9F17B1287825
:2088E00000B13E6005B0BDE8F08F029901B10860039DD6E900012A46287002F8041F0B0EFD
:20890000D3700B0C9370090A6971010EE970010CA970000A687006F10801019C2046032275
:2089200003F046FC00200E9F295C202903D001300828F9D101E0002129540020215C202904
:2089400003D001300328F9D1C8E700212154C5E72DE9F0418046002543F24457C1F2080769
:20896000E908786805F00702415CD140C90701D001351FE0691C00BFB1F5806F09D0CA0820
:2089800001F00703825CDA400131D207F4D04C1E01E04FF48064661B3968B86828444A1992
:2089A0003146434617F082FE7868294632461BF0B2FA2546B5F5806F28BFBDE8F081CFE7FB
:2089C0002DE9F04F85B09A4690460D46814600F049F9002800F1DF8043F23014C1F208045B
:2089E000BAF1000FE06B08BF814402AF002D00F0B9804846394601AA17F090FF002800F178
:208A0000B3808246DDF808B0CB454FD1484604A903AA17F083FF0646C0106168085C06F0EE
:208A20000701C840C00741D000270020012122F0C5F8606D38B103284F4604D0012814BFD0
:208A40004FF0FF37E76B0120394622F0B7F8A06D48B10328494602AF07D0012814BF4FF06B
:208A6000FF31E16B01E0002102AF022022F0A6F8E06D40B10328494606D0012814BF4FF0EC
:208A8000FF31E16B00E00021032022F097F8A16C062000F083F8002878D11BF084FB0028D4
:208AA00074D160683146012222F0D2FDA068616B019ACDF80080ABEB0903D618AE42A8BF93
:208AC0002E4601440020324600231AF093FFB0424DD10320494622F071F87110042022F092
:208AE0006DF8206E40B10328494606D0012814BF4FF0FF31E16B00E00021052022F05EF8BD
:208B0000606E48B10328494607D0012814BF4FF0FF31E16B01E000BF0021062022F04EF807
:208B2000A06E48B10328494607D0012814BF4FF0FF31E16B01E000BF0021072022F03EF8B6
:208B4000E16C042000F02AF870B91BF02CFB98B96068514601221BF0DEF9AD1BB044B144D1
:208B60007FF444AF002016E06FF4817013E04FF6FA60CFF6FF700EE002286FF481704FF6AE
:208B8000FA61CFF6FF7108BF881C04E04FF6FA60CFF6FF70043005B0BDE8F08FF8B50C4617
:208BA00043F23017C1F2080705463868010E4FF0FF300E2955D8012202FA01F144F24A0218
:208BC000114208BFF8BD7E6B10204FF0807121F0F5FFF8688119112021F0F0FF71190F2094
:208BE00021F0ECFF42F60827C1F20807F9694A69B2B13869CB6C012163B19847F9693869E8
:208C00004A69012190470546F9693869CA6C0021904701E09047054615B9002087F842007A
:208C200041F28005C1F20805286A0444002021F0EBFF40B9286A8442F8DA002022F010F86A
:208C40004FF0FF30F8BD69460F2021F091FFB01E0099081A18BF0120891B18BF012108400C
:208C60004042F8BD70B582B043F23016C1F2080696F8760008B10025D1E017F073FD0028F8
:208C800036D44BF634113046C1F6012140F8301F002180F8471050F81C1C49688847002856
:208CA00028D4044696F8770018B91BF083FA002820D4002021F0A8FF20B9002021F0D0FF43
:208CC000012817D14FF48071726C706D02F2071222F0070202F12003C6E9023231610328B6
:208CE0000BD84BF69811C1F6012151F8200006E005468FE06FF0FF058CE04FF0FF30B16D6A
:208D0000032906D84BF69812C1F6012252F8211001E04FF0FF310843F16D032906D84BF6C5
:208D20009812C1F6012252F8211001E04FF0FF310843316E032906D84BF69812C1F601222B
:208D400052F8211001E04FF0FF310843716E032906D84BF69812C1F6012252F8211001E0F3
:208D60004FF0FF310843B16E032906D84BF69812C1F6012252F8211001E04FF0FF31084335
:208D80004FF6FA65CFF6FF7516D40020A6F87400306C012812DBF16E01F10802002100BFED
:208DA00032F80C3B19440138FAD1A6F87410082010FA81F0C00802E0043D2BE001200121E3
:208DC00081F3108842F66A11C1F6042121F0BCF97060002181F31088706830B1B6F874203A
:208DE00000212CB122F034FC04E06FF4807511E01BF091F8716B726C306F00900020002346
:208E00001AF0F8FD002805D40C204FF47A71FFF7C5FE38B196F8760008B922F07FFD284695
:208E200002B070BD1BF0BFF90028F3D4012086F8760020E72DE9F04F83B091460C4682460C
:208E4000D0F864810F7BD1E901063146002216F0EDFB009720FA07F5FEF77CFF07462068A1
:208E6000CDE9015085B30025E808029A05F00701105CC840C00718BF002E05D10135019820
:208E80008542F1D120E000BF009805FA00F44FF0000B00BF0BFA07F040EA0401D8F82420B7
:208EA0005046904750464FF45A3122F00FFE5046494622F00BFE20B90BF1010B5E45E9D144
:208EC000DCE74FF0FF3006E001980730C108029803F094F9002003B0BDE8F08F2DE9F04388
:208EE00083B01C46154688468146012702AE00BF18F8010B02900097484631462A4600F0AC
:208F000007F80435013CF3D1002003B0BDE8F0832DE9F84F14468A4680464BF6EF69CDF684
:208F2000AD690A9D6E4640F2A91B00BF5AF8047BA7F1110040280BD2009098F8291111B32E
:208F4000D8F84411B0EB810F28D1D8F82C012CE0D8F84411404617F023FDBFB1A7F2611073
:208F6000FF2825D898F8FC00022860D8A7F2122006284FD898F8FF00A7F21121814256D17B
:208F8000D8F834012AE000F00F0220E098F8FC000328484624BF002020601FE0890041F040
:208FA000010188420ED1D8F830012060002713E0A7F16100FF2819D840463946224622F0DB
:208FC000ABFD08E04046314617F0F6FD009A404621461BF0D0F907460FB1002020600434CA
:208FE000013D04BF0020BDE8F88F9FE7A7F151000F28F2D840463946224622F08DFD4AF66B
:209000000070CFF6FF7000EB07204021C0F2FA01014327E0A7F22320052808D898F8FF00C9
:20902000A7F22121814202D1D8F83801D6E7B7F5137F0ADC5F4521D0B7F5D57F21D040F21D
:20904000C91087424846C9D004E0A7F24D2002284846C3D349F60070CFF6FE7000EB07201B
:2090600040F44031404622F031FD0028B5D407464046214600221BF07EF9ADE7D8F83C0155
:20908000ACE7D8F84001A9E72DE9F04383B01C46154688468146012702AE00BF18F8010B1B
:2090A00002900097484631462A4617F0F9FD0435013CF3D1002003B0BDE8F0832DE9F041A9
:2090C00082B0D0F86461804672690221904741F28004C1F2080401AD206A00F1640700BF6D
:2090E0007268404629469047002807D49DF80400C00606D4206A381A0128F1DA4FF0FF3050
:2091000003E040461BF0C6F8012002B0BDE8F08170B5144614F8042B054614F8030C14F808
:20912000023C14F8016C42EA002040EA034040EA0662D5F85C01436D0E465B69012198473A
:20914000D5F85C0147F2F002416D4B6903219847013E00BF14F8040B14F8021C14F8032CD7
:2091600014F8013C40EA022040EA014040EA0362D5F85C01416D4B6902219847013EE9D1D9
:20918000002070BD2DE9F04714460E468146D0F8A401B9F8B0218F2122F05CFFB9F8B21140
:2091A000D9F8A40100EBD10001F0070247F2E00122F014FAD9F8600109F5D2730ECB1BF0F0
:2091C000F7F9D9F8A401B9F8B0218C2122F042FF751E0027D9F8600109F5D2730ECB1BF094
:2091E000E7F9B9F8B011D9F860A15046012200F059F80646B9F8B2115046202200F052F87F
:2092000044B12070010EE170010CA170000A6070043400E000243743013DDBD1D9F8A4015B
:20922000B9F8B0218A2122F015FFD9F8600109F5D2730ECB1BF0BCF9B9F8B0A1D9F8606139
:2092400030465146012200F02DF88046B9F8B2113046202200F026F844B12070010EE170E4
:20926000010CA170000A6070B9F8B0A1D9F8A4018821524622F0EEFED9F8600109F5D273CA
:209280000ECB1BF095F9B9F8B011D9F86001012200F008F848EA0701084318BF4FF0FF30DB
:2092A000BDE8F08700B54FEAE10C01F0070310F80CE02EFA03FEC3F1080393420ADA604483
:2092C000013000BF10F8011B99404EEA010E08339342F7DB4FF0FF3090402EEA000000BD65
:2092E0002DE9F84343F66419C1F2080999F80000012818BFBDE8F88343F62060C1F208007E
:20930000802143F63045C1F2080501602868012867D8EFF31088012181F31088286830B1CC
:209320000124012814BF4FF48076002601E0002600244427C4F20507386840F001003860EC
:2093400040F60000C0F20E60386000BF57F8040CC007FBD03868386040F60000C0F600103B
:20936000B86200BFB96A01F0F851B1F1106FF9D1386400BF396C01F0F851B1F1106FF9D1A7
:20938000386200BF386A00F0F850B0F1106FF9D140F2DC50EEF784FF386820F44070304313
:2093A000386000BF57F8040CC007FBD064B940F2DC50EEF775FF386840F08000386000BFEA
:2093C00057F8040CC007FBD043F63840C1F208004EF21401CEF200010068086088F3108837
:2093E0002868002189F8001042F22E71C1F60421085C43F63061C1F208010860BDE8F8830A
:20940000ADF6480D43F2AC15C1F2080544F21970C1F60320E860002242F63A60C1F60420EE
:209420002864686A10A9696243F25C71C1F2080185F866200E684BF6D827C1F60127C6F836
:2094400098709146139241F22D71C1F60321CDE910010DF2747101F11000059001F1340A6A
:2094600001F12C000D900DF26F1000F10C0B0DF2BB1008300B9001F144000E9006F18C00B7
:2094800006904FF48078CDE907B6CDF83CA000BF0DF2747420469C2102F0B0FE4BF61C30F1
:2094A000C1F60120CDF89C07CDF89877CDF8947701208DF891074FF4B270ADF8800713A83E
:2094C000CDF87C0741F6FD00C1F60320CDF878074AF26520C1F60120CDF87407CDF8AC8721
:2094E0000DF27460CDF8A807CDF8A0470020C1F62160CDF88C07E86918B10DF25310CDF888
:2095000008084FF49660CDF8C8070B98CDF8C4070DF27470CDF8B807CDF8F8B7CDF8BC07D8
:20952000E86C08B94020E864686D08B90C2068652A6D5C463AB10DF26F110844841A696B7A
:20954000204602F035FE4AF24070C1F60120CDF80408CDF8FC47CDF8D8870DF15300CDF8A9
:20956000D007002F00F002860D98002104F096F90128C0F25E86504642F27641C1F6042108
:2095800004F0CEF930B14FF00108002401200C901CE000BF504640F2EE71C1F6042104F054
:2095A000BFF920B102200C900124A0460EE0504640F2F371C1F6042104F0B2F980460028D6
:2095C0001CBF03204FF001080C9001240DF50166504631460822002304F0FAF90128C0F2FF
:2095E000E885CDF800685046F0F77AFCEE69B6FA86F04009204308D171685046002204F057
:2096000027FA10BB3668002EF6D12F6A97B10024A346002679685046012204F019FAA04234
:20962000C2BF3E464FF0010B04463F68002FF1D102E000BF0026B3466FEA0800B6FA86F1B0
:209640004909084203D000F0A2BD4FF0020B0E980021F0F765FCCDF84468EA6C0B2AC0F045
:20966000DB85DDF8D4170F9849B1DDF8E027012304F0AEF90128C0F2CF85EA6C0F98DDF88D
:20968000F817002304F0A4F9CDF83C08002840F3C385DDF8F8070C998DF820180E99CDF8B9
:2096A0001C18CDF818086C6A0DF6180A34B100BF6168504688472468002CF9D1BBF1000F87
:2096C00012D1DDF8F847204640F23951C1F6042102F00CFD40B9204641F6C871C1F60321F0
:2096E0000B2202F065FD00BFDDF8A807DDF8B077DDF8B417DDF8F827CDF8EC27441820467C
:209700004CF2A631C1F6032106223B4604F0E2F9CDF83C08B84200F07F850444A079312830
:2097200040F07A85207A302805D0312840F074856E208DF8800701270E980121F0F7F0FB55
:209740006E698EB1DDF8F8774FF000080DF6380A7068514602683846904740B93668002E30
:20976000F6D10026012707E00026B04604E0307A002800F0548300279DF880079DF88117E4
:20978000643818BF0120B1FA81F1490908408DF80E08CDF8E407BBF1000F03D0CDF8CC878D
:2097A00054E000BF002F00F04583EA6842B1DDF8FC0705999047DDF8840708B1CDF89407C4
:2097C0009DF8900701280DD1DDF8040850B103680E990DF2747022469847CDF83C08002807
:2097E00040F01A850F98F0F77BFB0D98002104F055F8CDF83C08002800F10E8503280F9C04
:2098000021DBDDF8B01701291DDBDDF8A877DDF8AC27DDF8B4379E1AB8BF1E46BF5D3F2F15
:2098200011D101339A1AB8BF1A460139CDF8B01708BF0A46CDF8B427421E0DF27470214660
:209840002023F0F781FB204604F0DBF90D98012104F024F8CDF83C08002800F1DD840228B0
:209860000AD1DDF8B007012800F25A820020CDF8B007814664E200BF4FF000080026002095
:20988000CDE90900B146DDE90E0ACDF81808DDF8C06700BFD6B3B4685046214604F040F8C6
:2098A00010B93668F6E700BF0746DDF8B007B84203D20021CDF8B0170CE0DDF8AC17DDF8F7
:2098C000B4273A44511AB8BF1146C01BCDF8B00708BF0146CDF81C48CDF8B41771680DF6FC
:2098E00018008847022840F0A680DDF8AC07DDF8B0173944814209DCCDF8B017DDF8B4178C
:20990000C91B48BF0144CDF8B41700BF504642F27A41C1F6042104F003F838B1DDF8B017F3
:20992000814205D20022CDF8B0270EE04E4637E0DDF8AC27DDF8B43703449A1AB8BF1A46FC
:20994000091ACDF8B01708BF0A46CDF8B427DDF83C18081ACDF83C085046F0F7C1FADDF840
:209960003C18081ACDF83C0803284E4618DB00BF50461BF017FD6FF02F0151FA80F00928C7
:2099800000F24A8406EB860100EB4106DDF83C080328A0F10100CDF83C08DDF83CA0E7DC0A
:2099A00050464CF2AD31C1F6032103F0B9FF002800F01081DDF8B017814203D20022CDF8AB
:2099C000B0270CE0DDF8AC27DDF8B43703449A1AB8BF1A46091ACDF8B01708BF0A46CDF8FF
:2099E000B427DDF83C18081ACDF83C085046F0F777FADDF83C180C1ACDF83C48032CC0F2D1
:209A0000E9802868E8B1036850460DF6180122469847CDF83C0848B928680DF618014368EF
:209A200050460DF2747298475FFA80F8B8F1000F40F0D0802FE30446504604F0E2F84E466F
:209A400058E150464FF6BD21C1F6032103F068FF002800F0BF80049600268DF81868DDF8EE
:209A6000B017814203D20022CDF8B0270CE0DDF8AC27DDF8B43703449A1AB8BF1A46091A80
:209A8000CDF8B01708BF0A46CDF8B427201ACDF83C085046F0F724FADDF83C180D1ACDF890
:209AA0003C584FF0000A062D58DBDDF8A847DDF8AC770DF5046000BFBAF11C0F4ED8DDF8B1
:209AC000B0C7BCF1040F12DB0022DDF8B41700BF635C83540131B942A8BF31460132042ADF
:209AE000F6D1CDF8B417ACF10400CDF8B0079DF8400803F048FF80469DF8410803F043FF02
:209B0000000340EA88489DF84298484603F03BFF48EA80169DF84388404603F034FF3043D7
:209B20000DF61802010C02F80A10B9F13D0F01D1012109E002EB0A01020AB8F13D0F4A7061
:209B40001ABF88700321022100260DF504608A44092DA5F10405CDF83C58ADDC0DF61800C1
:209B600043F2AC1500F80A60DDF89C87C1F20805D8F804604EB382463068002800F0738134
:209B8000DDF8F8474FF00009B768D7B1017839B1411C00228B5C0132002BFBD101E000BF2F
:209BA0000022214622F0AEFB30B93846514602F09DFA50B14FF0010956F8100F0028E3D147
:209BC00051E1B9F1000F40F04E814FF00108DDF83CA0049EE86878B39DF8910760BB9DF8A8
:209BE000900748BB286C38B30DF274700E9940F2F872C1F604220DF63C0303F09DFF002157
:209C0000CDF8CC17C0B1017839B1411C002400BF0A5D0134002AFBD100E0002440F60901B2
:209C2000C1F604210422234603F054FFA0421CBF01208DF80F0800BF504642F2A641C1F6D2
:209C4000042103F06DFE28B19DF80D0840F020008DF80D08BBF1020F20D0BBF1010F2DD1AD
:209C60000A9858B90DF274700E9942F2D642C1F604220DF63C0303F05FFF0A900998E8B90F
:209C80000DF274700E994FF6E122C1F603220DF63C0303F051FF099010E000BFA868DDF864
:209CA000F8170768009150460DF274710DF63C020DF64403B847002840F0AE82DDF8B0077D
:209CC000DDF83C18884205D20020CDF8B407CDF8B0070EE0DDF8AC27DDF8B4370B449A1A45
:209CE000B8BF1A46401ACDF8B00708BF0246CDF8B42702240D98012103F0D0FDCDF83C0852
:209D0000002800F1898202287FF4BCADDDF8B007012800F284810020CDF8B00781468EE19B
:209D2000A0F10209CDF8B097DDF8AC07DDF8B4170231081AB8BF0846B9F1000F08BF48462B
:209D4000CDF8B407002400260020CDE90900DDF89C87B246D8F80460D6B13068C0B1DDF8D1
:209D6000F87700BFB16899B1017839B1411C00228B5C0132002BFBD101E000BF002239461E
:209D800022F0C0FA00286ED056F8100F0028E9D15646BBF1010F23D0BBF1020F00F00B82BD
:209DA0009DF890070C99012908BF012800F0CB800C99032940F01681DDF8AC07864200F3A2
:209DC0002B8200BFB14580F2E5800D981BF002FBCDF83C080128C0F21F82DDF8B097F1E724
:209DE0000020CDF8CC07DDF84408DDF8F8178768DDF8002809988DE84300DDE90D010A9BE8
:209E0000B847CDF83C080028DDF83CA0DDE907B64FF480783FD10E9803F0AAFC3BE08DF8B4
:209E20000E8864208DF88007CDF8E487BBF1000F7FF4B4AC95F8650000284FF0010018BF0D
:209E40008DF8F4077068DDF8F8274768DDF838180E9C20464DF62F33C1F60123B8472046ED
:209E600003F086FC10E00020009040F2911001900E9842F28A41C1F604214CF2BC32C1F605
:209E800003224346EFF74CFF089EDDF83CA0DDF81CB04FF48078DDF8E407012817D19DF84A
:209EA000F40730B9DDF8BC07DDF8EC170022EFF731FE0020CDF8E4070E9C204642F2DE41E4
:209EC000C1F6042103F0BEFC204603F051FC0E980221F0F725F89DF881079DF882170843F0
:209EE00040F0A7819DF88007642800F0A2810022ADF8F427CDF8F027CDF8C027DDF8D40735
:209F000000B102700598C0E90022C0E9022264208DF880078DF80F288DF80D28DDF898076F
:209F2000DDF80418CDF8940701208DF891070020C1F62160CDF88C0709B1CDF8DC274FF021
:209F40000009FFF711BB0E9803F046FE9DF8F507DDF83CA00028DDE907B64FF480789AD1C6
:209F6000DDF8F8170DF27470F0F786F8002892DA002000904FF4CA7001900E9840F60E0178
:209F8000C1F6042140F62702C1F604220023EFF7C7FE80E7DDF80408C0B14768DDF8F8277F
:209FA0000096B1460DF274700E992346B847CDF83C080028DDF83CA0DDE907B64FF4807882
:209FC0003FF469AF01304E4600F026819DF80D080F9900F020030DF274703246EFF7B4FF81
:209FE0009DF89007012801D10E9839E79DF80F08DDF81CB0002878D0DDF8FC87DDF8F8078B
:20A0000098F8001011B308F101014FF0000A00BF11F80A200AF1010A002AF9D118E0A0F123
:20A020000209CDF8B097DDF8AC07DDF8B4170231081AB8BF0846B9F1000F08BF4846CDF8F4
:20A04000B407B8F1000F7FF4A4AE80E64FF0000A95F8661079B1C244286C1AF8016C00785B
:20A060000AF8010CDDF8940701684046884704460AF8016C38E0B8EB000238BFA0EB0802A1
:20A08000296CE86C0B78DBB14F1C0023FE5C0133002EFBD115E0DDF89C370DF6180000906A
:20A0A00040F2911001900E9842F28A41C1F604214CF2BC32C1F60322EFF732FE089EE6E62B
:20A0C000002310445A1C02EB0A0383420DD808EB0A0002F06DF8DDF894070168404688476D
:20A0E0000446002008F80A0054B900208DF80F08DDF89417DDF8FC0709688847044600B38E
:20A100000C98089EDDF83CA0C0074FF480780FD09DF8910710B10E9803F05EFD9DF8F507F0
:20A1200030B99DF891270DF27470214603F076FD0E9803F01DFBDDF894074168204688473A
:20A14000A9E6002000904FF4CA7001900E9840F60E01C1F6042140F62702C1F6042200238C
:20A16000EFF7DEFD089EDDF83CA092E640F2F710CDE900900E984CF26931C1F6032140F245
:20A18000DA62C1F604220023EFF7CAFD51E040F2F510CDE900900E984CF25F41C1F60321C9
:20A1A00042F2E642C1F604220023EFF7B9FDDDF81CB0089E3BE00C9801282DD19DF80D08D0
:20A1C00000F01F001F2827D19DF880076E2823D3DDF84408DDF80818C0689DF80C28076813
:20A1E0001C2000900E980B46B847012814DB8DF80C08DDF84408AA68816852680DF2747033
:20A200009047DDF844080E9CC068DDF87C17426820469047204603E001208DF882070E9807
:20A220000221EFF77DFEDDF83CA0DDE907B64FF48078D6F89C00002450B1C6F89C4030686A
:20A240007169C6E90100C6E90611069803F070FEBFF34F8F4FF00009C6F8A040D6F8987063
:20A26000FFF716B92DE9F84F43F25C75C1F208052C688046D4F89C0000284FD18A460020FC
:20A28000009000BFBAF1000F2ED0B8F1000F3DD06069D8B3D4E90617FA43561844BF616A4B
:20A2A0000E44564528BF56464FF00009B34600BF08EB0901626A1044C51BAB45B8BF5D4627
:20A2C00038462A4601F074FF2F446069616A01448F4208BF0746BFF34F8FE761BBEB050B6D
:20A2E00006D0A9446069E3E74FF0000A0EE000BF46B1BAEB060A0098304408BFBDE8F88F67
:20A300000090B04443F25C75C1F20805286880301BF0D2F8D4F89C000028B3D04FF0FF305D
:20A32000BDE8F88F2DE9F04104460068866891B188464BF6A430C1F60120051D002700BF05
:20A3400055F80C0B4146FDF715FD18B10137032FF6D100E037603068002848BFBDE8F081BE
:20A36000606840F2BD42C1F604220021EFF7D2FB40F66F21C1F60421204603F063FA306843
:20A3800018B93046214621F0A1FE2046BDE8F04103F0EEB953CB011A694B031A794B031A9E
:20A3A000894B031A73CB011A00000000A7CB011A13CD011A2FCE011A994B031AA94B031AA1
:20A3C000B94B031AABCE011A00000000F7CE011A37CF011AC94B031AD94B031AE94B031A04
:20A3E000F94B031A094C031A194C031A00000000294C031A6987001AE187001A5D88001AEB
:20A40000D988001A5189001A57CF011A394C031AC589001A00000000000000000F00000073
:20A42000000000000F00000009000000000000000D000000000000000F00000008000000E0
:20A44000000000000C000000000000000F0000000A000000000000000600000001000000D0
:20A460000F000000010000000000000004000000000000000F0000000B00000000000000AE
:20A48000000000000000000003000000010000000500000000000000000000000D000000A6
:20A4A000030000000000000002000000050000000F0000006BD0011ADFD0011A794C031A81
:20A4C0000000000097CF011A000000000000000000000000000000000000000000000000FB
:20A4E000A58C001A0000000000000000B1C8011AE9C8011A15C8011A00000000354D031A1A
:20A5000000000000000000007D4C031A8DC7011A15C8011A00000000A94C031A00000000DC
:20A5200000000000614E031A71C9011A01CA011A00000000CD4D031A0000000000000000DD
:20A540008D4E031AD5CA011A41CB011A000000001FD1011A00000000B94E031ADD4E031AAB
:20A5600081CB011A61CB011A0000000063D2011A000000000000000047D6011ACD4E031A6D
:20A5800061CB011A000000006FD4011A0000000000000000FD4E031AB5CB011AED8D001A7F
:20A5A000014F031A59B1031AA13C031AA33C031A5DB1031A9F3C031A00000000954F031AED
:20A5C00021CD011A298E001A000000000000000000000000994F031A59B1031AA13C031A7B
:20A5E000A33C031A5DB1031A9F3C031A00000000000000000000000000000000E803000051
:20A6000000000000BD4F031AC94F031AB182001AB382001AE54F031A00000000E94F031A9A
:20A6200014B8011A00000000B9CE011A3150031AD94F031A3DCE011AE54F031A0000000037
:20A64000E94F031A14B8011A00000000B9CE011A3150031AD150031A05CF011A45CF011A22
:20A66000000000004D50031A00000000000000000000000088A6011A0100000001000000D5
:20A68000000000000100000001000000140000000000000000000000F551031AF598001A9A
:20A6A00059D6011A0DD7011A3E24041AFFF9031A4224041A09FA031A4624041A50C3031A60
:20A6C000AE06041A50C3031A4A24041A13FA031A4E24041A21FA031AB306041A21FA031AEB
:20A6E0005224041A21FA031A5624041AB806041A5A24041A5BC3031A66C3031AC106041A18
:20A700005E24041A2BFA031A00000000000000000E24041A1224041A1624041A1A24041AFF
:20A720001E24041A2224041A2624041A2A24041A2E24041A3224041A3624041A3A24041AA9
:20A740000D54031A2DA1001A2BE8011A0FE9011A7BE9011A5956031A01000000E625041ADD
:20A76000AFC4031A000000002959031A000000001BF5011A27F6011ACBF6011A7559031A80
:20A780007959031A9559031AB159031AC7F7011A29A4001AB7F8011A7BF9011A000000007F
:20A7A000F1F2011ABDF4011A99F5011A91A4001A3D5A031A515A031AF55A031ADD5B031A9A
:20A7C000955C031AE9F6011A4F09021AD5BA001A3162031A4D62031A9309021AA562031AFC
:20A7E0008F0D021A6501021ABD62031A3163031A4563031A6163031A7963031AA963031A6A
:20A800002F0E021A2F0E021A4F09021AD5BA001AB963031A4D62031A1B11021AA562031AF8
:20A820009F12021A39BB001ABD62031A2F0E021A2F0E021A2F0E021A2F0E021A2F0E021A44
:20A840002F0E021A2F0E021A000000000D9C031A0323031A6DBB001A79BC001A7DBD001A58
:20A8600000000000D563031AB101021A00000000000000007DBE001A9903021AE105021AA6
:20A8800055C1001A0000000000000000F714021A0000000000000000000000000000000061
:20A8A000000000000000000000000000000000000D9C031A0323031AF912011AA113011A9A
:20A8C000E555021AE183031A7582031AFBB6021A000000009BD1021AC112021A7185031A36
:20A8E0005986031A0515021A0168031A000000000000000000000000373F021A6588031A04
:20A90000000000000000000073D2021AE188031A000000000D9C031A0323031AF912011A21
:20A92000A113011AE555021AE183031A7582031AFBB6021A000000009BD1021A5D68031A26
:20A940007185031A5986031A00000000E916021A17D2021A00000000000000004741021A24
:20A960006588031A000000000000000073D2021AE188031AAD73031A8D73031ADDF4001AA1
:20A980005D3A021A4379021AF573031A1574031A4574031A45F5001AE5F5001AF569031A68
:20A9A000F969031A156A031AAB44021A296A031A456A031AF99E031A796A031A4346021A9C
:20A9C0006918021A411A021A5349021AF95B011AD16A031AD91A021AF569031AF569031ADF
:20A9E000FD6A031A256B031A7B49021AF569031A8735031A1D1E021AD5E2001AD16B031A71
:20AA0000A9DF021AA16C031AF569031AE9E3001AF569031A35B2031AF569031AF569031A92
:20AA2000F569031AF569031AF569031AF569031A8920021A75E6001A79E7001AD1E7001AA4
:20AA4000D1F6001A7176031AEB79021A534D021AE16C031A39AE031A973B031AFDAD031AB1
:20AA6000613B031A6751021A8F52021AFF54021A95E8001A2121021AF569031AF569031AF2
:20AA80003755021A7755021ACF55021AF569031AF569031AF569031AD1AD031A69AE031AA6
:20AAA000E359021A0B5B021A8125031A719E031A256D031A3911021AF569031AF569031AC2
:20AAC000F569031AA77A021AB35B021A435C021AAB5C021A756D031A5F5D021A9DE6021A40
:20AAE000F569031A1B5F021AF569031A3122021AC96D031A4D25031A5B60021AD56D031A43
:20AB0000B32F021ADF32021A89E9001A1335021A9F3D021AF569031A390E021A5D9E031A2C
:20AB2000F569031AF569031AE1E9001AF569031ABF7BFFB9A9EB001ADD6D031AB364021A86
:20AB40004B66021A1368021A852C021AF5EC001AE768021A216E031A916E031A4B6A021AC5
:20AB60000000000000000000000000000000000000000000DD6E031A0970031A5D70031AED
:20AB8000FB6A021A55EE001A2971031AAB6B021A8571031AD171031A7B6C021A736D021A7D
:20ABA0001D72031AB92E021AC52F021A7572031A1761021AFB63021AA929021AF132021A97
:20ABC000AB70021A3771021A5372021A0573031A1573031A2573031A3D73031A8373021ACB
:20ABE0005173031A01000000E625041A75C5031A0000000021EF001AFB73021AD538021A16
:20AC00000DF2001A5573031A6573031A5375021A7573031A8573031A8973031AAD73031AED
:20AC20008D73031ADDF4001A5D3A021A4379021AF573031A1574031A4574031A45F5001A2C
:20AC4000E5F5001A6574031A8975031A7B78021AC174031A59B0021AF5E4021A2577031ABB
:20AC6000E13B021A11F8001A7977031A9977031AA9FB031A05000000B977031AAFFB031A65
:20AC800005000000BD77031AC2C5031A06000000C177031AC9C5031A06000000C577031A55
:20ACA000FA25041A0B000000C977031AD0C5031A0E000000FF7B021A0626041A130000003C
:20ACC0003B7D021AAFC6031A19000000CD77031AE77F021A85FA001A0110C0E4B210C0E062
:20ACE000015EA0EC74EE150F00453BD574EE350F20453BD510EE150E000533D564EE350FAF
:20AD000020451BD564EE150F00451BD500531CD5000318D5200318D5400318D500EE150EAE
:20AD2000000513D510F8011B0114403830F8021B0124407800EE151E010513D500F8011B30
:20AD40000114003820F8021B0124007810EE151E010533D5CFA7021A000000000000000003
:20AD600027A8021AFD80031A800000000D9C031A0323031AD104011A954D021A9D7F031A9E
:20AD8000AD02011A6D51021AA799021A0000000027A2021AAFAC021AE509011A9552021A4B
:20ADA000A17F031A5FAE021A0000000000000000050D011AC180031ABFA4021A0000000023
:20ADC000000000009FA6021AE580031A290E011AAD81031A800000000D9C031A0323031A6A
:20ADE000D104011A954D021A9D7F031AAD02011A6D51021AA799021A0000000027A2021A47
:20AE0000BFAE021AE509011A9552021AA17F031A53B0021A0000000000000000050D011A14
:20AE2000C180031ABFA4021A00000000000000009FA6021AE580031A510E011AB181031A89
:20AE4000000000000D9C031A0323031A513F021AA9FD001AA578031AD144021AF543021ABE
:20AE60005978031A00000000F38B021A790E011A6146021AADFF001A517A031ACFB2021A9A
:20AE8000000000003BB3021A097A031ACF92021AEF8A021A0000000000000000EF97021A54
:20AEA000797B031A9510011A3111011A000000000D9C031A0323031A513F021AA9FD001AEF
:20AEC000A578031AD144021AF543021A5978031A00000000F38B021A4BB4021A6146021A4D
:20AEE000ADFF001A517A031A03B6021A0000000000000000097A031ACF92021AEF8A021A1D
:20AF00000000000000000000EF97021A797B031A0555021A4555021A000000000100000051
:20AF20000300000002000000000000005915011ADD15011AF7D6021A7189031A8160021A79
:20AF40004516011A57D7021A9589031AF3D7021A77D9021ACD89031A73D6021AB116011AEA
:20AF60001961021AEBD9021A9FDF021A63E0021AA3E4021A5D8A031AEBE4021A37E6021A97
:20AF80006BE6021A33E9021AE7E9021A7BEE021A7D8A031A73D6021A651A011AFD1B011A45
:20AFA00003EF021A000000000D9C031A0323031A916A021A2D1F011A496B021AAD1F011A45
:20AFC000F16B021AF96C021A00000000818A031AED1F011AF16D021A0D21011A0000000066
:20AFE00000000000000000008FF0021A0000000000000000000000000000000000000000B6
:20B000000000000000000000000000000D9C031A0323031AFD73021A1928011AC58A031AD3
:20B02000092A011AB92C011AB98D031A00000000ABF1021AF12D011AD530011A3933011AC7
:20B040009D75021A00000000000000000000000000000000000000000000000000000000C2
:20B060000000000000000000000000000000248C000044ACFFFF6324FCFF601404002124F3
:20B0800020FF043C08008000000000000000248C000044ACFFFF6324FCFF601404004224CB
:20B0A00020FF043C0800800000000000000000000D9C031A0323031AC538011AED38011A48
:20B0C00077FA021AC991031A2184021ABFF9021A00000000000000005F07031A5BF7021AE6
:20B0E000C3F8021A5590031A8FFD021AF991031A0000000000000000FD91031A000000007D
:20B100001183021AC183021A00000000E7FA021A000000000D9C031A0323031AC538011A01
:20B12000ED38011A77FA021AC991031A2184021ABFF9021A00000000000000004308031ACE
:20B140005BF7021AC3F8021A5590031A8FFD021AF991031A0000000000000000FD91031AAE
:20B16000000000001183021AC183021A00000000E7FA021A0992031A00000000E308031A02
:20B180008709031A1188021A1992031A2D8B021A1539011AE709031A2306031A7F06031A53
:20B1A0000000000000000000000000000000000000000000000000000000000023285040B4
:20B1C0008322C0406F00C03FE0B1011AF0B1011A00B2011A10B2011A832280406F00004036
:20B1E0000324004123808200938212006F00803F0324004123908200938222006F00803F6B
:20B200000324004123A08200938242006F00803F0334004123B08200938282006F00803F6A
:20B2200030B2011A40B2011A50B2011A60B2011A8324004103840400232880406F00803F0E
:20B240008324004103940400232880406F00803F8324004103A40400232880406F00803F66
:20B260008324004103B40400233880406F00803F7370047B0F1000006F00C03F7360047BA1
:20B28000736440F1232680106F00803F070E031A0594031A413B011A730E031A9710031ABE
:20B2A0001194031AF98B021AE992021AF597021A2306031A7F06031A7B12031A7D94031A2D
:20B2C0005314031A9594031AE994031A3F15031A2995031A00003200000036000000330023
:20B2E000000037000910340000002200000026000000230000002700091024002598031A21
:20B3000000000000000000007B1B031A6998031A6999031A8B20031A9199031AB999031ABF
:20B32000C599031A00000000000000000000000000000000D199031A813D011A153E011AC4
:20B34000FD99031A8D3E011A1D9A031ADD99021A8D9C021AF53E011A9120031A3D9A031A99
:20B360000A000000020000000C000000090000000800000019000000180000000B00000068
:20B38000030000000A0000000A0000000A0000000A0000000A0000000A0000000A00000064
:20B3A0000D000000000200000D9C031A0323031A9D9A031A1540011A599E021A9941011AA9
:20B3C0006542011AE320031A00000000000000000D21031A1943011A499F021A00000000C5
:20B3E000AD9A031A0000000000000000C944011A000000005B21031A000000000000000028
:20B4000000000000C19A031AFD173100FD178100FD179100000200000D9C031A0323031A2A
:20B4200000000000000000000000000000000000000000000000000000000000000000000C
:20B44000194A011A51A2021AE150011AF9A4021A259B031A0000000000000000A5A6021A16
:20B4600000000000399B031A000000000000000000000000B59B031A2917FF4F29D896AD9C
:20B480006A0C9FCDFD494F44C806EAC048C9039EF4278E801D85C13B90A85054AF61682B81
:20B4A0007401AE0BBA15E9F3796EF2B456279568EBDC58CABCDA99E584D93F525DC12BB0C8
:20B4C00099F2ECE7F8E62C16CE713A664EA968E4D5A0310F019B718A5107474F9FAEDAD794
:20B4E00079EC70E864D4C9560A9786A7018DA515D4F0813438471B37E485CFA11BBAC0EF7B
:20B500000A552F51839971A235E1AF0CB1C07FC88088023512DEB50A33BF91C7E4908ED387
:20B52000C510B59352EB7DC491C959A3D87DC3B68D257FDE5B21C6F53D13DFC21C60923BCC
:20B5400016244B02D2CC69B602754773589D7F847F38D5692A59C62C56C6DC1BFE59495F02
:20B56000EDB35C747D7B0860B43684BCC7760C6A1FA0991B98F487AE0100010000000000E8
:20B5800078B4011A400000004000000000000000010000000000000078B5011A010000009A
:20B5A000010000000000000001000000000000000000000000000000010000000700000081
:20B5C0000F000000C8B5011A032C031A38C6031A292C031A4E27041A4F2C031A6227041A19
:20B5E000C9A2031A4BC6031A752C031A5AC6031A832C031A7627041AE1A2031A6DC6031A23
:20B60000992C031A74C6031AA32C031A7FC6031AAD2C031A8AC6031ABB2C031A95C6031AC4
:20B62000F5A2031A7E27041A81A4031A99A4031AB1A4031ABDA4031AE5A4031AFDA4031AA3
:20B640008DD5021A09A5031AC92C031A15A5031A21A5031A35A5031A49A5031A81D6021A60
:20B660005DA5031A69A5031ADB2C031AF92C031A79A5031A0B2D031A95A5031A19D7021A27
:20B6800069D7021AD1A5031A112D031A372D031A5D2D031A31A6031A61A6031A832D031A53
:20B6A000752C031AC9A2031A11D8021AD15F011A91A6031A91A6031AB12D031A95A6031AF9
:20B6C000A5A6031AB5A6031A5961011A91A6031A91A6031AB72D031AC1A6031A91A6031A34
:20B6E00091A6031A91A6031A91A6031AFD2E031A272F031A95D9021AD5DA021ACDA6031AAE
:20B70000F9A6031A9563011A4D2F031A29A7031AC563011A572F031A35A7031A692F031A40
:20B7200041A7031A832F031A51DB021A91A6031A4DA7031A9D2F031A9D2F031AFDDD021AC0
:20B740009D2F031A9D2F031A9D2F031A9D2F031A9D2F031A9D2F031A9D2F031A9D2F031AA1
:20B760009D2F031A91A6031AA72F031A9D2F031A9D2F031AB12F031ADB2F031A59A7031A86
:20B7800069A7031AFD2F031AAB30031A9D2F031A9D2F031A9D2F031A9D2F031A9D2F031AAE
:20B7A0009D2F031A15A8031A41A8031A9D2F031AB930031A9D2F031A99AA031AD935031A5D
